:020000040800F2
:1080000000800120C14F01088DFF00088FFF00088C
:1080100091FF000893FF000895FF00080000000092
:1080200000000000000000000000000097FF0008B2
:1080300099FF0008000000009BFF0008F581000880
:1080400005500108055001080550010805500108B8
:1080500005500108055001080550010805500108A8
:108060000550010805500108055001080550010898
:108070000550010805500108055001080550010888
:10808000055001080550010805500108119200082B
:10809000A99000085D9100080550010805500108ED
:1080A0000550010805500108055001080550010858
:1080B0000550010805500108055001080550010848
:1080C0000550010805500108055001080550010838
:1080D0000550010805500108318F0008658C000823
:1080E0000550010805500108055001080550010818
:1080F0000550010805500108055001080550010808
:1081000005500108055001080550010805500108F7
:1081100005500108055001080550010805500108E7
:1081200005500108055001080550010805500108D7
:1081300005500108055001080550010805500108C7
:1081400005500108055001080550010837A2000834
:1081500005500108055001080550010805500108A7
:108160000550010805500108055001080550010897
:108170000550010805500108055001080550010887
:04818000055001089D
:1081880010B5054C237833B9044B13B10448AFF349
:1081980000800123237010BDB405002000000000FA
:1081A800EC5501080C4B43B10C4810B50C49AFF322
:1081B80000800C48036823B910BD0A48036833B926
:1081C8007047094B002BF7D0BDE810401847064B05
:1081D800002BF5D0184700BF00000000EC5501083F
:1081E800B8050020B405002000000000684620F013
:1081F80007018D4601B51B4B19781A4600292ED068
:108208005B681949013353600B6801330B60174BE6
:10821800196811B1196801391960154B196811B13C
:1082280019680139196000231370124B1A683AB1A2
:108238001A68013A1A601B6813B901220E4B1A70AA
:108248000E4B1A683AB11A68013A1A601B6813B9DA
:1082580001220B4B1A70BDE8014085467047012288
:108268001A70E2E7D0050020406200203C58002048
:108278004058002044580020485800203858002012
:108288004958002041F64B52094B10B55A60F0226C
:10829800084C6FF0040084F8232000229A6007221B
:1082A8001A600AF0B7FA302384F8233010BD00BFF3
:1082B80010E000E000ED00E0014B5868704700BF97
:1082C800D0050020000000002DE9F34101210846F7
:1082D8000024022509F06CF8012748F21343814E67
:1082E8006946304600938DF805508DF804708DF876
:1082F80006408DF8074008F0A1FE48F21103758387
:1083080033834FF480736946304600938DF80450E8
:108318008DF805508DF806408DF8074008F08EFE60
:1083280021464FF4800008F099FF2846394609F0A5
:108338003FF84023DFF8BC816946404600938DF83A
:1083480005508DF804408DF806408DF8074008F078
:1083580075FE41F2B4034046694600938DF8055016
:108368008DF804708DF806408DF8074008F066FE19
:108378008423A8F81A3041F230033946A8F8183097
:10838800042009F015F84EF2C233694656480093A6
:108398008DF805508DF804408DF806408DF807409B
:1083A80008F04CFE3946082009F002F84FF48E73A5
:1083B80008F500684046694600938DF805508DF829
:1083C80004408DF806408DF8074008F037FE4FF658
:1083D80080634046694600938DF805508DF8047017
:1083E8008DF806408DF8074008F028FE8023A8F88D
:1083F8001A304FF47E433946A8F81830102008F098
:10840800D7FF45F6FF734FF4005869463748009385
:108418008DF805508DF804408DF806408DF807401A
:1084280008F00CFE694630468DF80550CDF80080FE
:108438008DF804708DF806408DF8074008F0FEFDB1
:108448004FF480433046694600938DF805508DF807
:1084580004408DF806408DF80740454608F0EEFDCB
:108468000A22234630464FF47A71758300BF0139DA
:10847800FCD10169A6F818804F044FF47A7158BFEF
:10848800013300BF0139FCD10169490448BF0134F7
:10849800013AE8D10A2B164B21D10A2C1FD101220F
:1084A8001A704FF4C04300240093022369460D4814
:1084B8008DF804308DF805308DF806408DF80740AA
:1084C80008F0BCFD22460D21064808F041FE224670
:1084D8000E21044808F03CFE02B0BDE8F0810022FD
:1084E800DEE700BF00000240000802400010024022
:1084F8007C59002000040240F7B5104B1B78D3B11B
:1085080010210F4B0F46012000241E460D4D5F839E
:1085180018830194019AAA4209D93183708301947E
:10852800019AAA42F3D8019A01320192F8E7019A16
:1085380001320192EEE703B0F0BD00BF7C59002084
:10854800000002403F0D03000022802110B5074BB8
:10855800074C072022801983114601F067F921781A
:108568000122BDE81040072001F060B9000C02406C
:1085780022580020032110B5094C400001FA00F0F0
:108588002188002221EA000121800720090A01F040
:108598004DF921780122BDE81040072001F046B9C5
:1085A80022580020022110B5094C40008140208843
:1085B8000022014389B221800720090A01F036F917
:1085C80021780122BDE81040072001F02FB900BF33
:1085D8002258002038B50546002445FA04F3DB0785
:1085E800E0B205D5FFF7DEFF0134082CF5D138BD20
:1085F800FFF7C0FFF8E708B507282ED8DFE800F036
:10860800040D12171C1E2328002001F089FAB0F56A
:10861800006F34BF0020012008BD114B1869C0F35A
:10862800400008BD0E4B1869C0F3800008BD0C4B14
:108638001869C0F3C00008BD0420E6E7084B1869B4
:10864800C0F3401008BD064B1869C0F3801008BD80
:10865800034B1869C0F3C01008BD002008BD00BF57
:108668000008024007282CD8DFE800F004090E13A0
:10867800181D2227144B1888C0F340007047124B6E
:108688001888C0F3C00070470F4B1888C0F340101B
:1086980070470D4B1888C0F3C01070470A4B1888F4
:1086A800C0F340207047084B1888C0F3C0207047BB
:1086B800054B1888C0F340307047034B1888C00B2F
:1086C80070470020704700BF2258002038B50020AE
:1086D800FFF791FF041C18BF0124144D2B699A075A
:1086E8002B6948BF44F002045B072B6948BF44F07C
:1086F800040418074FF0040048BF44F00804FFF7CB
:108708007AFF08B144F010042B6999062B6948BF19
:1087180044F020045A062B6948BF44F040041B0665
:1087280048BF44F08004204638BD00BF000802401E
:108738001022064B10F0010F14BF1A835A8320220F
:1087480010F0020F14BF1A835A83704700040240C6
:1087580008B5082001F0E4F9592805D9064B1A781C
:108768000AB901221A7008BD082001F0D9F9542865
:10877800F9D80022004BF5E7D8050020034B1878FC
:10878800013801288CBF002001207047D80500203F
:10879800034B187801280ABF022200201A7070477C
:1087A800D8050020052822D8DFE800F003080D12BC
:1087B800171C104B186900F0010070470D4B186921
:1087C800C0F3800070470B4B1869C0F30010704766
:1087D800084B1869C0F380107047064B1869C0F33E
:1087E80000207047034B1869C0F3802070470020B1
:1087F800704700BF00100240154B18691A6980F4D1
:10880800004051041A69C0F3C03058BF40F002005C
:108818009204104A58BF40F00400116949071169D1
:10882800126958BF40F00800090758BF40F010000F
:10883800D1061A691B6958BF40F02000920558BF3D
:1088480040F04000DB0558BF40F08000704700BF93
:1088580000080240000C0240034B10B1034ADA60E2
:108868007047034AFBE700BF00ED00E00400FA058B
:108878000100FA0500224FF0FF31930003F1604335
:10888800013203F56143082AC3F88010C3F8801148
:10889800F3D1002319460448C2180133F02B82F89B
:1088A8000013F9D1704700BF00E100E0C0B207F043
:1088B800C7BAC0B207F0B2BA2DE9F743484D04462B
:1088C80005EB8015EB690BB16E8B96B93821204604
:1088D80006F0CEFE382120F48062204606F098FE8D
:1088E8004FF480323A21204603B0BDE8F04306F049
:1088F8008FBE07F038F8C0F1080006FA00F00BF058
:10890800AFFDED69064685EAE570A0EBE5700F4618
:108918000BF0A6FD02460B46304639460BF030FFF9
:10892800304B002206460F460BF000FE6A46804692
:1089380089460CF0BBFB002200230CF05FF8A0B1C5
:10894800494640460CF08CF8002D06464FF0380199
:10895800B8BF4642204606F08BFE382120F48062DC
:10896800204606F055FE3246BCE7304639466A4690
:108978000CF09CFB002D06460F46DDE9000118DDD2
:108988000CF06EF814A3D3E90023050439463046E9
:108998000BF0CCFD0CF064F805433821204606F0B6
:1089A80067FE382140F48062204606F031FE2A46F0
:1089B80098E70CF055F808A3D3E90023C5433946D6
:1089C80030460BF0B3FD0CF04BF8C0F51C502D04ED
:1089D8001030E1E7AFF30080000000000088C340DA
:1089E800845600200000F040392106F041BE0A46B6
:1089F800392106F00DBE10B50024E0B20134FFF7AE
:108A08005BFF062CF9D110BD022803D80130C0B293
:108A1800FFF7F1BD052801D80230F8E700207047BC
:108A280018B1012806D000207047054B1869C0F31B
:108A380000207047034B1869C0F38010704700BFCF
:108A4800000C024000040240064B1B69DB0541BFD5
:108A5800054B186980F04000C0F3801058BF012012
:108A6800704700BF000C024000040240012907B50E
:108A78001BD004D3022926D003B05DF804FB88B9C3
:108A88004FF48043009300238DF804300222694696
:108A980011488DF806308DF805208DF8073008F05C
:108AA800CDFAE9E74FF48053ECE70B4A40B94FF4AD
:108AB80080435383009301238DF804300023E5E7B6
:108AC8004FF48053F5E7044A18B94FF480431383F1
:108AD800F0E74FF48053FAE70010024070B50646FD
:108AE80088B0584809F064FC01214FF4802008F050
:108AF80083FC0121022008F05BFC02244FF4806310
:108B0800002502A9504802938DF80C408DF80E50AC
:108B18008DF80D408DF80F5008F090FA4FF400636F
:108B28000293012302A948488DF80F308DF80C40B4
:108B38008DF80E508DF80D4008F080FA07220A21B2
:108B4800414808F005FB404807220B2108F000FBCC
:108B580004A809F0DFFC0B2E71D8DFE806F07006D8
:108B680055585B5E6164676A6C6E4FF4615304A983
:108B78003648049309F074FC2723002401258DF856
:108B88000430062301A88DF805308DF806408DF8CD
:108B9800075009F0F5FD40F2FF312C4809F0BAFD05
:108BA80022462821294809F097FD2A4640F22771D4
:108BB800264809F091FD2A4640F22661234809F02B
:108BC8008BFD2A4640F22551204809F085FD2246B2
:108BD80040F224411D4809F07FFD224640F6460137
:108BE8001A4809F079FD224640F66A11174809F03B
:108BF80073FD22466021154809F06EFD2946134889
:108C080009F0A9FC08B070BD4FF49643AFE74FF4E4
:108C1800E143ACE74FF41643A9E74FF46143A6E7F5
:108C28004FF49633A3E74FF4E133A0E74FF46133F1
:108C38009DE7074B9BE7074B99E7074B97E74FF4EF
:108C4800165394E700100140000402400048004019
:108C580090D0030020A1070040420F00684620F092
:108C680007018D4619B522480388990614D5214B6A
:108C78001A6859680132202A08BF00228A4205D0A2
:108C8800196880881944C0B208721A600A211A4A01
:108C980011609A6A194B1A60154803881A0612D58A
:108CA800164B1A687AB9134BDC6A196B8C4219D0C7
:108CB800196B4C1C1C63194491F834108180196B92
:108CC800202900D11A630A4803885B0606D540F2BA
:108CD800266109F043FD074B1A6BDB6ABDE81940B2
:108CE8008546704740F2277109F0F6FCEBE700BFB4
:108CF80000480040DC050020445800203C58002073
:108D08000A4AD36A116B0133202B08BF00238B4218
:108D18000AD0D16A114481F83400D36240F2277135
:108D28000122034809F0D8BC704700BFDC050020C9
:108D380000480040094B59681A6891420CD05A689B
:108D4800511C59601A44127A02705A68202A01D1BB
:108D580000225A600120704700207047DC0500207F
:108D6800014B9862704700BFDC050020044B1A785D
:108D780002F0FF0012B1002201201A70704700BFF4
:108D88004858002072B60022024B5A601A6062B638
:108D9800704700BFDC05002010B5441E14F8010F11
:108DA80000B910BDFFF7ACFFF8E770B5064688B00C
:108DB800584809F0FDFA01214FF4003008F01CFB77
:108DC8000121084608F0F4FA02240025042302A928
:108DD800514802938DF80C408DF80E508DF80D40D7
:108DE8008DF80F5008F02AF908234B480DEB0301C2
:108DF80002938DF80C408DF80E508DF80D408DF8CB
:108E08000F5008F01BF907222146434808F0A0F943
:108E180041480722032108F09BF904A809F07AFBCE
:108E28000B2E74D8DFE806F07306585B5E61646742
:108E38006A6D6F714FF4615304A93648049309F0C1
:108E48000FFB2623002401258DF80430062301A8F2
:108E58008DF805308DF806408DF8075009F090FC24
:108E680040F2FF312B4809F055FC224628212948B9
:108E780009F032FC2A4640F22771264809F02CFCFA
:108E88002A4640F22661234809F026FC2A4640F289
:108E98002551204809F020FC224640F224411D4873
:108EA80009F01AFC224640F646011A4809F014FC5B
:108EB800224640F66A11174809F00EFC2246602146
:108EC800144809F009FC0222134B29465A83114819
:108ED80009F041FB08B070BD4FF49643ACE74FF47E
:108EE800E143A9E74FF41643A6E74FF46143A3E72C
:108EF8004FF49633A0E74FF4E1339DE74FF4613325
:108F08009AE7064B98E7064B96E7064B94E74FF42B
:108F1800165391E7004400400000024090D003003F
:108F280020A1070040420F00684620F007018D4647
:108F380019B52D4803889C0604D52C4B5B69990705
:108F480036D58388284803881A061BD5284B1A6803
:108F5800C2B9284BD3F88040D3F884108C423ED055
:108F6800022422490C83D3F884104C1CC3F8844093
:108F7800194491F888108180D3F88410202901D1F0
:108F8800C3F88420184803885B060DD540F2266193
:108F980009F0E4FB174BD3F88420D3F880309A42C9
:108FA80002BF0222114B5A83BDE81940854670471B
:108FB800104B5A6D996D0132202A08BF00228A424F
:108FC80006D0596D80881944C0B281F85C005A6592
:108FD8000A21094A1160DA6F054B1A60B2E740F2BC
:108FE800277109F079FBCDE70044004000000240FA
:108FF80040580020DC050020385800200C4AD2F8E0
:109008008030D2F884100133202B08BF00238B4214
:109018000CD0D2F88010114481F88800C2F8803052
:1090280040F227710122034809F056BB704700BF80
:10903800DC050020004400400A4B996D5A6D9142AE
:109048000DD09A6D511C99651A4492F85C200270F3
:109058009A6D202A01D100229A65012070470020CC
:10906800704700BFDC050020014BD867704700BF80
:10907800DC050020044B1A7802F0FF0012B1002230
:1090880001201A70704700BF4958002072B60022AC
:10909800024B9A655A6562B6704700BFDC0500202E
:1090A800684620F007018D4631B5264C264B2568C9
:1090B8001B680135082D08BF00259D4286B03BD0AE
:1090C80001AA0021214807F0A4FB9DF80C30226872
:1090D800042B1F4B03EB021227D101215170226888
:1090E800029903EB021251609DF80D20022A0CBF71
:1090F80001210021226803EB0212917022689DF879
:109108000E10120199540022216801A8104403EBA3
:1091180001111144C07A0132082A0872F4D125607D
:1091280006B0BDE83140854670470021517022687D
:10913800019903EB0212D6E70021044807F0B3FBBC
:10914800EEE700BFD85800204C58002000640040CB
:1091580058580020684620F007018D4631B5264C46
:10916800264B25681B680135082D08BF00259D4240
:1091780086B03BD001AA0121214807F04AFB9DF89F
:109188000C302268042B1F4B03EB021227D101215C
:1091980051702268029903EB021251609DF80D206C
:1091A800022A0CBF01210021226803EB02129170F0
:1091B80022689DF80E10120199540022216801A816
:1091C800104403EB01111144C07A0132082A0872D5
:1091D800F4D1256006B0BDE83140854670470021CE
:1091E80051702268019903EB0212D6E70121044865
:1091F80007F059FBEEE700BFD85800204C58002074
:109208000064004058580020684620F007018D4649
:109218002C4B11B52C4A1968126887B0914209D1B4
:1092280000220121294807F0C1FB07B0BDE8114021
:10923800854670471968264A02EB0111497801F002
:10924800FF00002931D004218DF80C100021019174
:10925800196802EB011149680291196802EB0111C2
:10926800897801F0FF0049B302218DF80D101968C3
:109278000901515C8DF80E100021186802EB0010EE
:109288000844047A01A8084401310829C472F4D1B9
:109298001A6801A901321A601A680C48082A04BF22
:1092A80000221A6007F021FABFE719688DF80C0050
:1092B80002EB0111496802900191CEE78DF80D008B
:1092C800D5E700BF545800205058002000640040E3
:1092D800DC580020F0B501388BB00E461546022345
:1092E800072800F22181DFE810F017010F010D01B6
:1092F800070105010301FB000800ADF80C300B2342
:109308008DF8103001238DF8113000239D488DF819
:109318000F3007F093F801214FF0007008F06CF857
:109328000121082008F044F80323002401930223B4
:109338000127012108208DF808308DF809308DF8B3
:109348000A408DF80B4008F033F801A98E4807F061
:1093580075FE092221468C4807F0FAFE09220121F0
:10936800894807F0F5FE03A986488DF80E408DF868
:1093780012408DF813708DF814408DF815408DF853
:1093880016708DF8177007F073F8B6F5006F8DF842
:1093980022408DF823408DF8247080F2C780730135
:1093A800ADF818304FF6FF73ADF81A40ADF81C3021
:1093B800ADF81E30ADF820408DF8257006A807F0EE
:1093C800C1F8012300228DF822308DF823208DF872
:1093D8002430002D00F0B980B5F5006F80F2B5801B
:1093E800ADF81A204FF6FF726901ADF81810ADF804
:1093F8001C20ADF81E20ADF820308DF8253006A8C9
:1094080007F0A0F802238DF822307313F60046F017
:10941800040600270124ADF81A604FF6FF7606A867
:10942800ADF818308DF823708DF82440ADF81C6025
:10943800ADF81E60ADF820708DF8254007F082F871
:109448000323BD428DF822308DF823708DF8244017
:1094580040F38A806B13ED0045F00405ADF8183031
:10946800ADF81A50ADF81C60ADF81E60ADF820409C
:109478008DF8254006A807F065F801240726002581
:10948800142368468DF800308DF801608DF802507D
:109498008DF8034009F074F9152368468DF80030FB
:1094A8008DF801608DF802508DF8034009F068F9D5
:1094B800132368468DF800308DF801608DF802504E
:1094C8008DF8034009F05CF9224602212D4807F087
:1094D8006DFA224610212B4807F068FA0BB0F0BD50
:1094E8000323ADF80C300F238DF8103002230AE760
:1094F8000623F6E70C23F4E70F22ADF80C208DF8CD
:10950800102000E71E23ECE73C23ADF80C300F23B6
:109518008DF810300723F6E67823ADF80C300C23CD
:109528008DF810300323EEE60823DAE74FF6FF73D1
:10953800ADF81840ADF81A40ADF81C30ADF81E3043
:10954800ADF820408DF8254038E74FF6FF71ADF8AB
:109558001820ADF81A20ADF81C10ADF81E10ADF8A3
:1095680020308DF825204AE70423ADF81870ADF8AF
:109578001A30ADF81C60ADF81E60ADF820408DF8CB
:10958800257077E700640040000C0240F0B543788E
:1095980087B004464268002B39D004238DF80C307C
:1095A800002302920193A37803B102238DF80D30B2
:1095B800234613F8081B06AA02F80A1D04F1100135
:1095C80013F8010B8B4202F8010FF9D101A91348D6
:1095D80007F08BF8042817D1114F124B3D681B6810
:1095E8000135082D08BF00259D4215D03B680E4E59
:1095F80006EB031694E80F0086E80F0001220748DF
:1096080011463D6007F0D2F9012007B0F0BD8DF892
:109618000C3001920293C6E70020F6E70064004090
:109628005058002054580020DC58002030B50C4B0E
:109638000C4C054622681B689A420FD02268531CBE
:109648002360094B03EB02130FCB85E80F00236857
:10965800082B01D100232360012030BD002030BD3C
:10966800D85800204C580020585800202DE9F047C1
:10967800012188B04FF4805007F0CAFE0121002470
:10968800E0230226664D084601938DF80A408DF8BE
:109698000B408DF808608DF8096007F089FE01A974
:1096A800284607F0CBFC05222846114607F050FD56
:1096B80028460522062107F04BFD4FF4827A4FF425
:1096C80000794FF0100828460125564F052207213A
:1096D80007F03EFD03A93846ADF80C40ADF8104040
:1096E800ADF81A40ADF81C40ADF80EA0ADF8126008
:1096F800ADF81450ADF81690ADF8188007F08EFF4D
:109708002946384608F023F829464FF4804007F0E8
:1097180073FE4FF4604307F55447294630460193DA
:109728008DF80A408DF80B408DF808608DF80960B7
:1097380007F03EFE01A9384607F080FC38460522AE
:109748000D2107F005FD384605220E2107F000FD22
:10975800052238460F21A7F5E63707F0F9FC03A9DB
:109768003846ADF80C40ADF81040ADF81240ADF8F1
:109778001A40ADF81C40ADF80EA0ADF81450ADF885
:109788001690ADF8188007F049FF2946384607F0CB
:10979800DEFF29464FF4004007F02EFE4FF4E05359
:1097A80007F5E8372946042001938DF80A408DF81B
:1097B8000B408DF808608DF8096007F0F9FD01A9E4
:1097C800384607F03BFC384606220A2107F0C0FC61
:1097D800384606220B2107F0BBFC062238460C212E
:1097E80007F0B6FCADF80C40ADF81040ADF81A40E3
:1097F800ADF81C400C4C03A92046ADF80EA0ADF8FE
:109808001260ADF81450ADF81690ADF8188007F056
:1098180005FF2946204607F09AFF08B0BDE8F08703
:109828000000024000300140003C0040F8B504460A
:109838000E461546072800F28280DFE800F004444F
:109848007174777A7D264FF400425D4B5A835D4FE1
:109858000221384608F009F80028F9D0314659485D
:1098680007F0D0FF574E0121304607F0FEFF0028D1
:10987800F9D0002D00F08D804FF40042504B1A8330
:10988800504807F0BCFFC0B2F8BD4FF480524E4BB1
:109898005A834E4F0221384607F0E7FF0028F9D0D7
:1098A80031464A4807F0AEFF484E0121304607F0DE
:1098B800DCFF0028F9D0002D6BD04FF48052424BCA
:1098C8001A834248DDE74FF48062414B5A83414F87
:1098D8000221384607F0C9FF0028F9D031463D4833
:1098E80007F090FF3B4E0121304607F0BEFF0028ED
:1098F800F9D0002D4DD0072C4BD801A353F824F0F4
:1099080081980008719900087D99000883990008DA
:10991800899900088F99000895990008C39800084C
:109928004FF40062D1E74FF48052CEE74FF4005273
:10993800CBE74FF48042C8E74FF40042C5E7072859
:10994800D7D801A353F820F057980008D7980008F3
:10995800D7980008D7980008D7980008D798000823
:10996800D79800089B9800084FF48062184B1A8318
:10997800184886E74FF40062F8E74FF48052F5E79D
:109988004FF40052F2E74FF48042EFE74FF4004201
:10999800ECE7072C12D801A353F824F089980008A3
:1099A8007999000879990008799900087999000847
:1099B8007999000879990008CB9800080020F8BD2B
:1099C80000000240003C0040000402400038004013
:1099D800000C0240003001402DE9F04101219CB00B
:1099E8004FF4800007F0E4FC01214FF4807000245C
:1099F80007F00EFD0326112301A9444801938DF8B1
:109A08000B408DF8086007F019FB01A94048DFF802
:109A18000C818DF80B4001968DF8086007F00EFB5D
:109A280001214FF4800007F0C3FC01214FF480703E
:109A380007F0EEFC404607F08FF8364B01250E93F1
:109A4800354B04270F934FF4806313934FF400634F
:109A580014934FF4005315934FF4807316934FF4F7
:109A680000330DA9404617930D941094129418943E
:109A78001A941B941197199507F0F6F82946404651
:109A880007F02DF903A8039404940594069406F0AE
:109A980059FB079409940A940B9404F1804404F543
:109AA800903407A920468DF820508DF821508DF864
:109AB800307006F018FB2946204606F005FC2B46B8
:109AC8002A4620460A2106F089FB2B462046022218
:109AD8000E2106F083FB2B4632462046082106F06D
:109AE8007DFB2B463A462046092106F077FB29469E
:109AF800204606F0F2FB2946204606F03DFB2046AC
:109B080006F0B2FB1CB0BDE8F08100BF00080240BF
:109B1800000402404C2001408406002010640240EA
:109B28000A2819D8DFE800F0061818180A181818B3
:109B38000D181500094B188880B27047074B5888D4
:109B4800FAE7064BD88883B240F26B1058430013EB
:109B58007047024B9888EFE7002070478406002082
:109B68000C4BC0EBC000184490F800380B7090F80C
:109B780001384B7090F802388B7090F80338CB702E
:109B880090F804380B7190F805384B7190F8063846
:109B98008B7170478C06002038B500214FF40063A4
:109BA800224A99540133B3F5804FFAD14FF4006437
:109BB800012206210020FFF739FE00220521104668
:109BC800FFF734FE002101220846FFF72FFE800729
:109BD800F3D5002202211046FFF728FE0022C4F325
:109BE80007211046FFF722FE0022E1B21046FFF7D8
:109BF8001DFE0025A5F13F014A424A4100210135D9
:109C08000846FFF713FE402DF4D100220521104627
:109C1800FFF70CFE002101220846FFF707FEC307E5
:109C2800F3D44034B4F5804FC2D138BD8C0600203F
:109C3800F7B50022C0EBC00000F500650C461046E1
:109C48000321FFF7F3FD0022C5F307211046FFF7B4
:109C5800EDFD0022E9B21046FFF7E8FD00221146AB
:109C68001046FFF7E3FD0022074611461046FFF7AE
:109C7800DDFD0022064611461046FFF7D7FD0022FB
:109C8800054611461046FFF7D1FD00228DF8030066
:109C980011461046FFF7CAFD00228DF80400114650
:109CA8001046FFF7C3FD00218DF805000122084684
:109CB800FFF7BCFD23788DF80600BB420ED1637810
:109CC800B3420BD1A378AB4208D1DDF80300D4F836
:109CD8000330C31A5842584103B0F0BD0020FBE7D7
:109CE80038B504461A4B0D461955012206210020A5
:109CF800FFF79CFD002205211046FFF797FD002184
:109D080001220846FFF792FD8207F3D500220221BF
:109D18001046FFF78BFD0022C4F307211046FFF71A
:109D280085FD0022E1B21046FFF780FD0122294699
:109D38000020FFF77BFD002205211046FFF776FD86
:109D4800002101220846FFF771FDC307F3D438BD8F
:109D58008C06002038B50D46C0EBC00404F5006041
:109D68000978FFF7BDFF697804F60100FFF7B8FF2F
:109D7800A97804F60200FFF7B3FFE97804F60300B8
:109D8800FFF7AEFF297904F60400FFF7A9FF697908
:109D980004F60500FFF7A4FFA97904F60600BDE85C
:109DA8003840FFF79DBF2DE9F84304460F460025CC
:109DB8003E4B0344954233D1012206210020FFF790
:109DC80035FD002205211046FFF730FD0021012254
:109DD8000846FFF72BFD8607F3D50022022110461F
:109DE800FFF724FD0022C4F307211046FFF71EFDEC
:109DF8000022E1B21046FFF719FD002605F1FF38F1
:109E0800B54211D1002205211046FFF70FFD0021B0
:109E180001220846FFF70AFDC307F3D4BDE8F8831B
:109E2800795D59550135C5E7013414F03F09B95D2D
:109E38003AD0A8EB0600424242410020FFF7F6FC68
:109E4800B9F1000F2ED146452CD20022052110462B
:109E5800FFF7ECFC002101220846FFF7E7FC10F0B1
:109E68000100F2D101220621FFF7E0FC00220521C2
:109E78001046FFF7DBFC002101220846FFF7D6FC5D
:109E88008207F3D5002202211046FFF7CFFC0022FB
:109E9800C4F307211046FFF7C9FC0022E1B21046BF
:109EA800FFF7C4FC0136ABE70122C6E78C060020A9
:109EB800014B185C704700BF8C060020002310B5CA
:109EC800044C2044934200D110BDC45CCC540133EF
:109ED800F8E700BF8C060020F7B5002203211046E2
:109EE800FFF7A4FC002211461046FFF79FFC002252
:109EF800444D11461046FFF799FC002443F6FF77BE
:109F08002E46E11B4A424A4100210846FFF78EFCD3
:109F180028550134B4F5804FF3D1002205211046AD
:109F2800FFF784FC002101220846FFF77FFC10F0B0
:109F38007104F2D1FEF7C0F90546FEF7BDF9401BE2
:109F48000028B8BF4042B0F5FA6F20DAC4B12E4BF2
:109F58001B78F3B940222D490020FFF7AFFF4024BA
:109F68002B4D04F1004140392046202205EB4101E8
:109F78002034FFF7A3FFB4F5807FF2D103B0F0BD22
:109F880096F8FF47A4F142035C425C41D5E7002CF8
:109F9800DDD1002140F2FF70FFF7A2FEFFF7FCFDC4
:109FA80040221A490020FFF7FEFE4024194D2046A2
:109FB800202229462034FFF7F6FEB4F5807FF6D13B
:109FC80000234FF4C36402AD45F8043D2046042243
:109FD80029460434FFF7E7FEB4F5FF6FF6D10023F6
:109FE8004FF4A76401932046042229460434FFF75E
:109FF800DAFEB4F5C36FF6D1422140F2FF70FFF7E5
:10A008006FFEA7E78C0600207C5900200400002082
:10A0180084560020C854010870477047122301482D
:10A028000B80704744000020042301480B807047D0
:10A0380056000020002070470020704730B50024EB
:10A04800084B01441A68814203D104B11A60002008
:10A0580030BD3F2A04D805789C18257101240132A7
:10A068000130F0E78C46002010B5044C0A4604483D
:10A07800214609F081F8204610BD00BFE36E00209C
:10A088009D55010810B5044C0A460448214609F0BC
:10A0980073F8204610BD00BFE36E0020AC550108E0
:10A0A80010B5044C0A460448214609F065F82046D4
:10A0B80010BD00BFE36E0020C455010810B5044C64
:10A0C8000A460448214609F057F8204610BD00BF4B
:10A0D800E36E0020CC55010810B5044C0A4604482C
:10A0E800214609F049F8204610BD00BFE36E002064
:10A0F800D7550108202803D021280BD0002070470D
:10A108000C4B0A689A610A791A774A795A778A79D8
:10A118009A77F3E7074A9369180A0B704870180C86
:10A128001B0ECB70137F88700B71537F4B71937F1D
:10A138008B71E3E7440000200020704770477047A8
:10A148007047704770474FF4C053F7B50026032790
:10A1580000930223244C694620468DF804308DF87C
:10A1680005708DF806608DF8076006F067FF2046D9
:10A178000A220B2106F0ECFF0A2220460C2106F0E9
:10A18800E7FF01254FF400736946204600938DF8D8
:10A1980005708DF804608DF806508DF8076006F09C
:10A1A8004DFF0A222046092106F0D2FF4FF48063B2
:10A1B8006946204600938DF806508DF807508DF8B3
:10A1C800057006F03BFF0A222046114606F0C0FF44
:10A1D80029464FF4804007F01BF92946802007F0F4
:10A1E800F3F803B0F0BD00BF00000240432307B5F9
:10A1F80003228DF80430012301A88DF805308DF86D
:10A2080006208DF8073008F0BBFA03B05DF804FBB0
:10A21800782358430723B0FBF3F000230133984217
:10A22800FCD270474FF47A735843FFF7F1BF684682
:10A2380020F007018D4601B5034809F069FDBDE826
:10A2480001408546704700BF385A0020F0B5002607
:10A25800084B094D0144884200D1F0BD1C68621CBE
:10A268001A6010F8017BB2F5006F2F5528BF1E60E9
:10A27800F1E700BF30560020E3660020074B30B5F9
:10A28800196841B100221D1D545D84540132914268
:10A29800FAD100221A60084630BD00BF8C46002063
:10A2A800084B10B51A68082A0AD900221C1D115D2E
:10A2B80081540132092AFAD1002201201A6010BD06
:10A2C800002010BD8C46002007B5064A012102F186
:10A2D8003C0300932032044B044808F0C2FB03B04F
:10A2E8005DF804FB4400002058010020385A002083
:10A2F800014809F0E3BC00BF385A00200000000004
:10A30800002330B519464FF0FF350D4A0D4813703C
:10A318005370141D44F82350C15401332F2BF9D125
:10A32800094B82F8C0101960084B82F8CC101960EC
:10A33800074BC2F8C410C2F8C810196030BD00BF7E
:10A34800D0460020085A0020306200204C620020CD
:10A358003460002038B5184C0546231893F8CD20F2
:10A368004AB3002204EB800483F8CD202521D4F8D9
:10A37800D42005F04DF9D4F8EC202846242105F026
:10A3880047F9D4F804212846282105F041F9D4F8E2
:10A398001C2128462A2105F03BF9D4F83421284607
:10A3A800232105F035F9D4F84C212846BDE838407A
:10A3B8002B2105F02DB938BDD04600202DE9F04FEE
:10A3C800914C8FB0A078052802D96378022B56D11A
:10A3D80000238E498E4A0B54135463780291914698
:10A3E800032B00F23083DFE813F004004D00AE00C9
:10A3F800A5020025874FDFF83482DFF824A2A2786F
:10A40800AA4209D0844B03EB8212527EA2B303EB1B
:10A4180085135B7E93422FD14FF0000B029B09F806
:10A4280005B003F805B0EB5DEEB243B17B4B2721D5
:10A4380053F82520304605F0EBF805F807B015F875
:10A44800083043B15AF825202621304605F0E0F8B7
:10A45800002305F808303046FFF77CFFD4F80320C6
:10A468002D21304605F0D4F80023202101930093D4
:10A478001A46304605F090F80135062DBFD10FB0C9
:10A48800BDE8F08F0025DFF8ACB1DFF88881DFF890
:10A498009CA1A278AA420AD05F4B03EB8212527E9B
:10A4A800002A40D003EB85135B7E93423BD1002703
:10A4B800029B09F805705F5515F80B30EEB2012BB9
:10A4C8003BD034D3022B3AD015F808304BB1534B5C
:10A4D800272153F82520304605F09AF8002305F87F
:10A4E800083015F80A304BB14D4B262153F825207A
:10A4F800304605F08DF8002305F80A303046FFF79E
:10A5080029FFD4F803302D211F443A46304605F080
:10A518007FF800232021019300931A46304605F066
:10A528003BF8404B5F600135062DB2D1A7E72D21DE
:10A53800304605F09DF80746C6E72121F8E7304682
:10A54800FEF752FAF7E7D4F80320142A00F3DE8165
:10A5580010F0400500F06181002301261D460DF131
:10A56800180B40FA03F111F0010114BF0BF8036056
:10A578000BF8031003F1010318BF0135062BF0D1C6
:10A58800012D59DC9DF81830B3B1224D2B7843B119
:10A59800254B2721D3F86421002005F039F8002342
:10A5A8002B70224D2B783BB11D4B26211A680020B9
:10A5B80005F02EF800232B700020FFF7CBFE0025B6
:10A5C8004FF0060A2E46DFF86880A3782B41DF0794
:10A5D80016D5029BEFB25E55D4F803302D210AFB45
:10A5E8000353384658F8232009F8056005F010F899
:10A5F8000023019600961A462021384604F0CCFF25
:10A608000135062DE1D13AE72C6000205256002092
:10A6180078560020585600208456002034480020E0
:10A628000458002044620020D04600201C58002016
:10A63800386000204C48002018230025B54E03FB45
:10A648000266E8B2212105F013F856F82530C01A41
:10A658000028B8BF404208AB43F825000135062D55
:10A66800EFD100234FF0FF321D461BF80310D8B27C
:10A6780031B108A951F823109142C4BF05460A46D2
:10A688000133062BF1D1A44B5A5D03935AB1A34B66
:10A69800272103EB8503D3F86421284604F0B8FF8B
:10A6A8000023039A53559E4E735D43B19D4B26215B
:10A6B80053F82520284604F0ABFF002373550026E5
:10A6C8002846FFF747FEAB000493944BAA0003EB20
:10A6D800020A1BF80630F7B2002B00F09980BD4241
:10A6E80000F0968008AB53F826000AF09BFA049A0B
:10A6F8000EAB1344804653F8180C0AF093FA01463F
:10A7080040460AF097FB8046DAF864010AF08AFAB4
:10A7180041460AF0DBFA0AF029FC272102463846AE
:10A7280004F076FF7F4B53F825000AF07BFA414688
:10A738000AF0CCFA0AF01AFC26210246384604F040
:10A7480067FFDAF8D4000AF06DFA41460AF0BEFA5B
:10A758000AF00CFC25210246384604F059FFDAF8C5
:10A76800EC000AF05FFA41460AF0B0FA0AF0FEFB84
:10A7780024210246384604F04BFFDAF804010AF0B7
:10A7880051FA41460AF0A2FA0AF0F0FB28210246E3
:10A79800384604F03DFFDAF81C010AF043FA414656
:10A7A8000AF094FA0AF0E2FB2A21002814BF0246B4
:10A7B8000122384604F02CFF049A584B1344D3F86E
:10A7C800340105930AF02EFA41460AF07FFA0AF09E
:10A7D800CDFB23210246384604F01AFF059BD3F827
:10A7E8004C010AF01FFA41460AF070FA0AF0BEFB63
:10A7F8000A2802464FF02B01B8BF0A22384604F057
:10A8080007FF0123039A9355454AB354464AB35464
:10A818000136062E7FF45DAFD1E6060642D53E4FDF
:10A82800DFF8FC80DFF8ECA0A3782B41D90735D5F9
:10A838004FF0000B029B09F805B003F805B0EB5D7B
:10A84800EEB243B1394B272153F82520304604F0A6
:10A85800DFFE05F807B015F808304BB1314B26215B
:10A8680053F82520304604F0D3FE002305F80830BD
:10A878003046FFF76FFD0622D4F803302D2102FB86
:10A88800035330465AF8232004F0C2FE0023202147
:10A89800019300931A46304604F07EFE0135062DDA
:10A8A800C2D1ECE5052831D81B4E335C4BB11B4BAC
:10A8B800272103EB8003D3F8642104F0A9FEA378D1
:10A8C800F554A078164D2B5C43B1164B262153F84E
:10A8D800202004F09DFE0022A378EA54A078FFF718
:10A8E80039FD06222D21A078D4F8033002FB03039A
:10A8F800084A52F8232004F08BFE0023A078019325
:10A9080000931A46202104F047FEB8E50422084BBC
:10A918001A70B4E53860002058560020D046002050
:10A928001C580020045800209D470020344800206F
:10A9380044620020D4F80330142BE7DC02064AD521
:10A948000025424FDFF81881DFF81091A3782B41DA
:10A95800DB073AD5EB5DEEB243B13D4B272153F807
:10A968002520304604F054FE0023EB5515F8083036
:10A978004BB1384B262153F82520304604F048FEC9
:10A98800002305F80830A07809EB000393F87C3120
:10A998001BB1012B1DD0002002E02D2104F068FE20
:10A9A8000622D4F803302D2102FB03532A4A52F819
:10A9B80023200244304604F02BFE0023202101937B
:10A9C80000931A46304604F0E7FD0135062DBDD147
:10A9D80055E52121E2E7052898D81C4E1F4D335C28
:10A9E8004BB105EB8003D3F86421272104F010FE56
:10A9F8000022A378F254A078194E335C43B1154B6A
:10AA0800262153F8202004F003FE0022A378F254F4
:10AA1800A078054495F87C311BB1012B11D000209A
:10AA280002E02D2104F024FE0622A578D4F8033094
:10AA38002D2102FB0353084A52F8232002442846DA
:10AA480059E72121EEE7032261E700BF58560020AD
:10AA5800344800200458002038600020D0460020E8
:10AA68001C58002073B5D24EB5783446052D00F237
:10AA7800B3817278A52A00F0BA8300F2CF80142A35
:10AA880000F0878264D80C2A00F0118221D8042AA9
:10AA980000F0CE810AD8012A00F0AB81002A00F02C
:10AAA8009F81022A00F0A981032296E1062A00F07C
:10AAB800EB81C0F0D681072AF6D11021284604F090
:10AAC800D7FD0346F278B078D2080192C3F3072283
:10AAD800E4E1102A00F019821CD80E2A00F0068240
:10AAE80040F2F581B34ED4F8030006EB8503D3F8A2
:10AAF8009C31984724210246284604F089FDA37812
:10AB0800D4F8030006EB8306D6F89C319847C6F8BC
:10AB1800EC00CAE1122AA74E4FEA850300F023820F
:10AB280040F20B823344D3F88431D4F803009847B9
:10AB380023210246284604F06BFDA378D4F80300CD
:10AB480006EB8306D6F884319847C6F83401ACE1A1
:10AB58001C2A00F07F8221D8182A00F04E820FD8D4
:10AB6800162A00F0328240F22C82924BD6F803006B
:10AB780003EB8503D3F8843198473321024632E149
:10AB88001A2A00F0588240F247822846D6F8031065
:10AB9800C9B202B0BDE8704004F036BE7F2A00F0AA
:10ABA800828217D8202A00F05E82212A00F06C8267
:10ABB8001F2A7FF479AF1021284604F059FD024678
:10ABC800F378D1B2C2F30722B07803F00F030191F2
:10ABD800009266E1A22A00F0F88210D88C2A7FF44D
:10ABE80063AFD6F803102846C1F10801C9B204F0D2
:10ABF800E7FDB07802B0BDE87040FDF75DBEA32A5E
:10AC080000F0EC82A42A7FF44FAF2846D6F8031050
:10AC1800C9B202B0BDE8704004F03EBEBC2A00F0E4
:10AC2800898363D8AD2A00F02D831FD8A92A00F0A4
:10AC38000E830DD8A72A00F0018340F2EC82284643
:10AC4800D6F80310C9B202B0BDE8704004F028BFBE
:10AC5800AB2A00F00E8340F203832846D6F803108F
:10AC6800C9B202B0BDE8704004F0F9BEB62A00F0DF
:10AC78002B8311D8B12A00F00E83B52A00F0148373
:10AC8800AE2A7FF411AF2846D6F80310C9B202B035
:10AC9800BDE8704004F0F4BEB92A00F02A830BD84E
:10ACA800B82A7FF401AF2846D6F80310C9B202B01B
:10ACB800BDE8704004F0DEBDBA2A00F02383BB2A49
:10ACC8007FF4F2AED6F803102846C9B204F089FF23
:10ACD8000021B07804F0CCFCD6F803100246B07816
:10ACE800002900F0248342F0040246E2CC2A00F056
:10ACF80033832AD8C22A00F0F98110D8C02A00F07C
:10AD0800228300F2DB81BF2A7FF4CEAE2846D6F834
:10AD18000310C9B202B0BDE8704004F050BFC92AA0
:10AD280000F0F081CA2A00F0FA81C32A7FF4BCAE91
:10AD3800204BD6F8030003EB8503D3F884319847FA
:10AD48001D4B03EB85156860AFE0D52A00F0FD8147
:10AD580010D8D22A00F0EB81D42A00F0EF81D12A52
:10AD68007FF4A2AE2846D6F8031002B0BDE87040C2
:10AD7800FDF73DBEF02A00F0EE811FD8D62A7FF4F9
:10AD880093AED6F8030009F06BFB07A3D3E90023C1
:10AD980009F0F6FC0AF008FB09F062FE11210246F0
:10ADA80021E000BFAFF300802D431CEBE236FA3FF1
:10ADB8002C600020D046002084560020FB2A00F09A
:10ADC800D181FF2A7FF470AED6F80330002B00F053
:10ADD800D981012B00F0E7810422BC4B1A7064E092
:10ADE8002D21D6F80320284602B0BDE8704004F0B3
:10ADF8000FBCD6F803202121F5E7D6F8033020212F
:10AE0800002BC8BF0122284604F002FC0122B578B5
:10AE1800AF4BD6F803005A55AE4B002803EB850319
:10AE2800D3F88431B8BF4042984727210246DAE771
:10AE3800D6F80300A74C002804EB8505B8BF4042AC
:10AE4800D5F8843198472021C5F86401B07804F01A
:10AE58000FFC50BBB078272104EB8004D4F86421A0
:10AE6800C2E700229C4BD6F803005A55994B03EBD6
:10AE78008503D3F89C319847984B262143F8250041
:10AE8800B07853F82020AFE71021284604F0F0FBF3
:10AE98000346DAB2B0780192F278D2080092C3F38E
:10AEA80007430022102104F077FB02B070BD342163
:10AEB800284604F0DDFBD6F803300246B0781BB90B
:10AEC80042F0020234218FE722F00202FAE734212D
:10AED800284604F0CDFBD6F803300246B07813B903
:10AEE80042F00102EEE722F00102EBE734212846A6
:10AEF80004F0BEFBD6F803300246B07813B142F036
:10AF08001002DFE722F01002DCE7724CD6F80300EB
:10AF180004EB8503D3F88431984725210246284657
:10AF280004F076FBB378D6F8030004EB8304D4F876
:10AF380084319847C4F8D400B7E73344D3F89C3138
:10AF4800D4F80300984728210246284604F060FBFD
:10AF5800A378D4F8030006EB8306D6F89C3198470B
:10AF6800C6F80401A1E73344D3F89C31D4F80300B0
:10AF780098472A210246284604F04AFBA378D4F8C9
:10AF8800030006EB8306D6F89C319847C6F81C01E7
:10AF98008BE7504CD6F8030004EB8503D3F88431D3
:10AFA80098472B210246284604F032FBB378D6F89E
:10AFB800030004EB8304D4F884319847C4F84C01A7
:10AFC80073E7D6F803202C210DE7D6F803000028F4
:10AFD800FFF602AF424B03EB85152B7E012B01D008
:10AFE80004F09AFF0028C8BF3E4A4FF01501CCBFB5
:10AFF80092FBF0F23C4AA078F6E63421284604F0A9
:10B0080037FBD6F803300246B07813B142F0080295
:10B0180058E722F0080255E73421284604F028FBB7
:10B02800D6F803300246B07813B142F0040249E77B
:10B0380022F0040246E73421284604F019FBD6F82A
:10B0480003300246B07813B142F400623AE722F4C2
:10B05800006237E72846D6F80310C9B202B0BDE847
:10B06800704004F0E3BB6E21284604F001FBF3783E
:10B07800B57801933379002203F0030300936E211E
:10B08800C0F3074328460EE76E21284604F0F0FA7D
:10B098000246D1B2C2F30722F378B0780191009248
:10B0A8006E210022FFE6D6F80330022B3FF694AE5D
:10B0B800084B1D44F37885F87C31F6E6084B03EB22
:10B0C8008515D6F803302B72EFE600BF44620020E6
:10B0D80058560020D04600201C5800200458002054
:10B0E800845600200024F400B50010009F4BD6F8C9
:10B0F800030003EB8503D3F8843198479C4BAD01DB
:10B108005851D2E63821284604F0B2FAD6F803306E
:10B1180000F4806223F480631A4338216BE7944B70
:10B12800D6F8032003EB85135A83284662E5904B33
:10B13800D6F8032003EB8513DA61F6E78C4B03EBB3
:10B148008515D6F803302B62AFE6894B03EB8515DE
:10B15800F3786B76A9E6864B03EB8515F37885F8CB
:10B168002430A2E60021284604F082FAD6F803101B
:10B178000246B07819B142F01002002134E622F0FC
:10B18800100231E67A4A02EB85121376774B03EB0D
:10B198008505784BC5F88431C5F8B431C5F89C31BC
:10B1A800C5F8CC3181E6724A02EB851213766F4BF3
:10B1B80003EB8505704BC5F88431704BC5F8B43185
:10B1C8006F4BC5F89C316F4BEAE72846D6F8031059
:10B1D800C9B202B0BDE8704004F0CEBA2846D6F82D
:10B1E8000310C9B202B0BDE8704004F031BB284674
:10B1F80004F0D5FBD6F80310B378C9B228B91846BD
:10B2080002B0BDE8704004F085BB184602B0BDE846
:10B21800704004F053BB284604F0C1FBD6F8031075
:10B22800C9B228B9B07802B0BDE8704004F092BA4B
:10B23800B07802B0BDE8704004F05ABB2846D6F892
:10B248000310C9B202B0BDE8704004F069BA2846DC
:10B25800D6F80310C9B202B0BDE8704004F0DBBBF9
:10B268002846D6F80310C9B202B0BDE8704004F011
:10B27800E4BB2846D6F80310C9B202B0BDE8704056
:10B2880004F0B7BB2846D6F80310C9B202B0BDE82F
:10B29800704004F017BC2846D6F80310C9B202B0B3
:10B2A800BDE8704004F09EBAD6F803000028FFF607
:10B2B80093AD2E4B03EB8503D3F8843198472C4B81
:10B2C80003EB85152861F0E5D6F803000028FFF6A2
:10B2D80083AD274B03EB85152B7E012B01D004F0A2
:10B2E8001BFE0028CABF284A284A92FBF0F2142104
:10B2F80081E62846D6F80310C9B202B0BDE870400E
:10B3080004F04CBAD6F803000028FFF665AD184BD8
:10B3180003EB85152B7E012B01D004F0FDFD0028E1
:10B32800CABF194A194A92FBF0F2132163E622F0C8
:10B33800040259E52846D6F80310C9B202B0BDE8A0
:10B34800704004F05EBC2846D6F80310C9B202B0BB
:10B35800BDE8704004F021BC2846D6F80310C9B2F5
:10B3680002B0BDE8704004F0F4BB00BFD046002036
:10B378008456002089FF0008B9FE000821FF000854
:10B38800F9FE000861FF00080024F400B500100071
:10B3980038B5D34BD34C98781D46052800F2E68281
:10B3A8005B78A72B00F0A88200F2B080142B00F085
:10B3B800D98152D8092B00F0A48122D8042B00F09F
:10B3C80071810ED8012B00F05981002B00F05281B9
:10B3D800022B00F05581032B00F05D8103232370BD
:10B3E8004DE2062B00F07081C0F06581072B00F05C
:10B3F8008381082BF2D1352104F03AF9C0F34020BB
:10B4080047E10E2B00F093810BD80B2B00F08681BF
:10B41800C0F07A810C2B00F088810D2BDED134210D
:10B428007DE1112B00F090810BD80F2B00F0858166
:10B43800102BD3D1AC4B252103EB8003D3F8B451A7
:10B4480024E1122B00F08781132BC7D1A64B2321AF
:10B4580003EB8003D3F8B45118E11E2B00F0BC8134
:10B4680025D8192B00F0A6810FD8162B00F0838160
:10B47800C0F07F81172B00F09681182BAED13421B4
:10B4880004F0F6F8C0F3C00003E11B2B00F09E8126
:10B49800C0F096811C2B00F09C811D2B9ED1924BF5
:10B4A80003EB8003D3F8B45103F0CAFDF0E08C2B12
:10B4B80000F0A3810ED8202B00F09481C0F08C817D
:10B4C800212B00F095817F2B88D1874B184490F869
:10B4D8007C3121E1A42B00F0FD8108D8A22B00F0DB
:10B4E800F681A32B7FF47AAF04F059FAD1E0A52BAB
:10B4F80000F0F381A62B7FF471AF04F050FA002816
:10B5080040F0F681A87804F019FAC2E0C12B00F0E7
:10B51800798150D8B52B00F0078222D8AC2B00F0E7
:10B52800F7810DD8A92B00F0ED81C0F0E881AA2B96
:10B5380000F0EB81AB2B7FF451AF04F0D5FAA8E013
:10B54800AE2B00F0EB81C0F0E681B12B00F0E98171
:10B55800B42B7FF443AF6F2104F08AF8C0F30440A2
:10B5680097E0BB2B00F0F08110D8B82B00F0E681F3
:10B5780004D8B62B7FF432AF1421FDE0B92B00F0CC
:10B58800E081BA2B7FF42AAF1321F5E0BE2B00F03F
:10B59800E18107D8BC2B00F0DA81BD2B7FF41EAF08
:10B5A800712168E0BF2B00F0DE81C02B7FF416AF5D
:10B5B80004F045FB6DE0CE2B00F04E8122D8C62B5F
:10B5C80000F03D810CD8C32B00F02A81C0F01F8108
:10B5D800C42B00F03081C52B7FF400AF434B2BE127
:10B5E800C92B00F02E8104D8C72B7FF4F7AE3C217D
:10B5F80041E0CA2B00F02B81CC2B7FF4EFAE04F096
:10B6080010FB46E0D42B00F050810FD8D02B00F06F
:10B618004481C0F02381D12B00F04481D22B7FF4E8
:10B62800DDAE334B03EB8010C36975E0F02B00F0FF
:10B63800468114D8D52B00F03D81D62B7FF4CEAEB1
:10B64800112104F015F808F00BFF23A3D3E9002318
:10B6580008F06CFF09F018FE09F002FA19E0FB2B5C
:10B6680000F03381FF2B7FF4B9AE214B03EB801040
:10B67800037E51E02D2103F0FBFF0AE02121FAE7C8
:10B688002721194B03EB8003D3F8B45103F0F0FFE3
:10B69800A8476060F3E0144B222103EB8003D3F842
:10B6A800B451F3E7104B03EB8000D0F8B431D0F875
:10B6B80064019847EDE70C4B0E4A03EB8003D3F87F
:10B6C800CC3152F82000F4E7102103F0D1FFC0F389
:10B6D8000720C000DDE700BF2D431CEBE236FA3F30
:10B6E8002C60002044620020D046002080590020B1
:10B6F8008456002004580020102103F0B9FFC0B27E
:10B70800E7E7FDF781F9C4E7352103F0B1FF10F051
:10B71800020F0CBF012300236360B0E0352103F062
:10B72800A7FFC04300F00100B3E73421EDE734215F
:10B7380003F09EFFC0F30010ABE78F4B242103EB0F
:10B748008003D3F8CC51A1E78B4B282103EB80036E
:10B75800D3F8CC519AE7884B2A2103EB8003D3F81E
:10B76800CC5193E7844B2B2103EB8003D3F8B451DE
:10B778008CE72C217FE7152103F07AFF0028CBBF47
:10B788007E4B6FF07F4393FBF0F06360AA787C4BAD
:10B79800C8BF606003EB82131B7E002B6FD160680B
:10B7A80004F086FB75E7744B332103EB8003D3F871
:10B7B800B4516BE7342103F05BFFC0F3800068E706
:10B7C800342103F055FFC0F3C02062E704F0D9F834
:10B7D8005FE704F0DDF85CE7102103F049FFC0F3F0
:10B7E800034056E76E2103F043FFC0F3090050E71A
:10B7F8006E2103F03DFF00144BE704F0B4F8C0F1EC
:10B80800080046E75E4B03EB8010037A84E75A4B47
:10B818005B49820103EB8000D0F8B431885848E7CF
:10B82800554A574B03EB801302EB8000D0F8B42144
:10B83800586890472DE7534B53F820306CE7362172
:10B8480019E7382103F014FF20F4806021E74C4BFE
:10B8580003EB8010438B5FE76F21C4E700224A4B5C
:10B868006260195C09B1012161601A54474B1A5C86
:10B878001AB1626842F00202626000221A54444B14
:10B888001B784BB1434B62681A60434B002A6FD157
:10B898001A6842F008021A6038BD6F2103F0E8FE0A
:10B8A800000EF6E6FDF7A0F8F3E6354B03EB801043
:10B8B800036A31E7324B03EB8010437E2CE7304BB1
:10B8C80003EB801090F8243026E7002130E704F0DD
:10B8D8003CF8DEE604F071F8DBE604F060F818B92D
:10B8E800A87804F084F8D4E6A87804F06DF8D0E6D7
:10B8F800A87804F075F8CCE604F00EF8C9E604F070
:10B908001AF9C6E604F0F7F8C3E604F0FBF8C0E657
:10B9180004F0FFF8BDE604F015F9BAE604F000F902
:10B92800B7E604F027F8B4E6134A154B03EB801387
:10B9380002EB8000D0F8B42118697AE704F036F8F1
:10B94800A7E604F009F8A4E604F087F9A1E604F0F4
:10B958008BF99EE6002103F08BFE10F004003FF403
:10B9680098AE0123D8E604F071F992E6042336E58F
:10B978001A6822F008028EE7D04600200024F4005E
:10B988008456002060590020785600205256002026
:10B998003F620020306200203460002038B5C44A7D
:10B9A80093781446022B00F01681032B00F01A81BD
:10B9B800002B40F0438253784D2B00F0C28044D8CE
:10B9C800452B00F0928019D8422B00F0848006D8CD
:10B9D800402B74D0412B79D00322B64B6DE0432B1A
:10B9E8007ED0442BF8D1D2F803301C200422B2496F
:10B9F80041F81C3FBDE83840FEF7D5B9482B00F0A8
:10BA0800818014D8462B75D0472BE5D1AA4DD2F8A2
:10BA1800033029460422082041F8083FFEF7C3F9FD
:10BA28002A69A9686879BDE83840FDF753BC4B2BF3
:10BA380074D000F28180492BCED1D2789E4B002A57
:10BA480067D1DA75D97D17203CE0542B00F09A8035
:10BA58001AD8512B00F0818008D84F2B76D0502B64
:10BA6800BAD1D178944B162099752BE0522B00F05F
:10BA78008180532BB0D1904DD2F80330294604224F
:10BA880041F8103F1020C9E7832B00F093800BD8B2
:10BA9800552B00F08380572B9ED1D37886490122FD
:10BAA80001F8273F2720A5E7852B00F08E80C0F0FE
:10BAB8008780FF2B90D1D278804B1A7038BD40F226
:10BAC800FF70D178BDE83840FEF70AB9D1787A4BD3
:10BAD80000201970F6E7D178774B01205970F1E70B
:10BAE800D178754B04201971ECE7D178724B052099
:10BAF8005971E7E7D2F803306F49042241F80C3F47
:10BB08000C2077E7D3786C49012201F8263F2620DC
:10BB180070E701226749DA754A6093E7664CD17885
:10BB28000320E170FEF7DCF8E078FDF719F9E0781A
:10BB3800BDE83840FDF798BAD1785F4B022099707C
:10BB4800C0E7D1785C4B15205975BBE7D2F80310D4
:10BB5800594BC9B259761920B4E7574D2A7DD207F7
:10BB680004D5E378DB0701D4FEF716F8E178142052
:10BB78002975A7E7D2F803304F49042241F8203F3E
:10BB8800202037E7D2F80330012B00F25781D37811
:10BB98004949012201F81A3F1A202BE7D2F803304D
:10BBA800012B00F24B81D3784349012201F81B3F56
:10BBB8001B201FE7D2F80320414BC3F8E42138BD0E
:10BBC800D2F803203F4B1A6038BDD2F803203C4B13
:10BBD800C3F8E82138BD51783B4BD2F8032043F82D
:10BBE800212038BD53782E2B3FF6F6AE01A252F82D
:10BBF80023F000BFD5BC0008E9BC0008FDBC000864
:10BC0800E1B90008E1B90008E1B90008E1B90008A4
:10BC1800E1B90008E1B9000811BD00081BBD000822
:10BC280025BD00082FBD000839BD000843BD000828
:10BC3800E1B90008E1B90008E1B90008E1B9000874
:10BC4800E1B90008E1B90008E1B90008E1B9000864
:10BC5800E1B90008E1B90008E1B90008E1B9000854
:10BC68004DBD00085BBD000869BD000877BD000830
:10BC780085BD000893BD0008A1BD0008AFBD000840
:10BC8800BDBD0008CBBD0008D9BD0008E7BD000850
:10BC9800F5BD0008FFBD000809BE000813BE000876
:10BCA8001DBE000827BE000831BE00083BBE0008C4
:10BCB8002C60002044620020040000203E62002026
:10BCC800D046002040620020506200205C4BD4F82F
:10BCD80003201A60FCF7F0FA5A4BC3F8EC0138BDA0
:10BCE800574BD4F803205A60FCF7E6FA554BC3F8D3
:10BCF800F00138BD524BD4F803209A60FCF7DCFA07
:10BD0800504BC3F8F40138BDD4F803204C4BDA602B
:10BD180038BDD4F803204A4B1A6138BDD4F8032043
:10BD2800474B5A6138BDD4F80320454B9A6138BD5A
:10BD3800D4F80320424BDA6138BDD4F80320404BD5
:10BD48001A6238BDD4F803303D4ADBB282F8243099
:10BD580038BDD4F803303A4ADBB282F82A3038BD0D
:10BD6800D4F80330364ADBB282F8253038BDD4F82F
:10BD78000330334ADBB282F82B3038BDD4F80330B5
:10BD88002F4ADBB282F8263038BDD4F803302C4A6B
:10BD9800DBB282F82C3038BDD4F80330284ADBB245
:10BDA80082F8273038BDD4F80330254ADBB282F850
:10BDB8002D3038BDD4F80330214ADBB282F8283060
:10BDC80038BDD4F803301E4ADBB282F82E3038BDB5
:10BDD800D4F803301A4ADBB282F8293038BDD4F8D7
:10BDE8000330174ADBB282F82F3038BDD4F803206D
:10BDF800134B1A6338BDD4F80320114B5A6338BD6E
:10BE0800D4F803200E4B9A6338BDD4F803200C4BAA
:10BE1800DA6338BDD4F80320094B1A6438BDD4F866
:10BE28000320074B5A6438BDD4F80320044B9A64A6
:10BE380038BDD4F80320024BDA6438BD0422CCE5BF
:10BE480098590020D04600202DE9F74F2A4E0024AB
:10BE58003746DFF8BC80B278A2420AD0274B03EB02
:10BE68008212527E002A40D003EB84135B7E9342F9
:10BE78003BD14FF00009224BDFF898A004F803905B
:10BE880014F80A3004F808904FEA840BE5B243B17D
:10BE98001C4B262153F82420284603F0B9FB04F84C
:10BEA8000A904FF00109184BD7F8030004F80390E3
:10BEB800164B002853F80B30B8BF4042984727214B
:10BEC8000246284603F0A4FBD7F803302021002BB4
:10BED800D8BF02224FF00003D4BF0192CDF80490DE
:10BEE80000931A46284603F057FB0134062CB2D1BA
:10BEF80003B0BDE8F08F00BF2C60002084560020FE
:10BF08007856002004580020585600205448002035
:10BF1800525600201C5800202DE9F74F2A4E0024C5
:10BF28003746DFF8BC80B278A2420AD0274B03EB31
:10BF38008212527E002A40D003EB84135B7E934228
:10BF48003BD14FF00009224BDFF898A004F803908A
:10BF580014F80A3004F808904FEA840BE5B243B1AC
:10BF68001C4B262153F82420284603F051FB04F8E3
:10BF78000A904FF00109184BD7F8030004F8039012
:10BF8800164B002853F80B30B8BF4042984727217A
:10BF98000246284603F03CFBD7F803302021002B4B
:10BFA800C8BF02224FF00003CCBF0192CDF8049025
:10BFB80000931A46284603F0EFFA0134062CB2D152
:10BFC80003B0BDE8F08F00BF2C600020845600202D
:10BFD8007856002004580020585600205448002065
:10BFE800525600201C5800202DE9F7430024184E13
:10BFF800184FDFF86C80B278A24209D0164B03EBD9
:10C008008212527EF2B103EB84135B7E934219D104
:10C018005FFA84F9484603F005F801230022E35546
:10C028002721484603F0F4FA0025022300950193DE
:10C038002A462B462021484603F0AEFA074B04F85F
:10C048000850E5540134062CD5D103B0BDE8F0837F
:10C058002C60002058560020845600207856002076
:10C068005256002064232DE9F341C249C2480A7898
:10C078000370D1F803302A2A427043600C46054603
:10C0880001F0CB8000F20C81142A00F0538459D8B7
:10C098000A2A00F0398222D8052A00F0248211D811
:10C0A800022A00F0148205D8012A00F0088202232F
:10C0B8002B7009E2032A00F01082042AF7D1FEF758
:10C0C8007DF901E2072A00F01482C0F00F82082AE5
:10C0D80000F01882092AEAD1FFF760FCF4E10F2A80
:10C0E80000F0A68313D80C2A00F03E83C0F0298301
:10C0F8000D2A00F04C830E2AD9D18878002800F048
:10C108006E83022800F07F8304232B70DCE1112A60
:10C1180001F0EB82C1F0E282122A01F0ED82132ACB
:10C12800C5D14978954A092900F2C783DFE811F09B
:10C13800C203CE03D103D403D803DF03E203E5032C
:10C14800FA03DD031F2A00F0EB854AD8192A00F00C
:10C15800A98419D8162A00F08F84C0F00A84172AF7
:10C1680000F08E84182AA2D1854AD2F8C830002B54
:10C1780000F0AA81013BC2F8C83002EB8303D3F870
:10C18800F831C2F8C4309FE11B2A00F0A784C0F040
:10C1980097841C2A00F08F851E2A88D14A78142A91
:10C1A80000F2AD818878052800F28A85062101FB16
:10C1B8000201744C44F82130734B9B7E002B00F035
:10C1C8008381002A00F080811823013A5A4302F53E
:10C1D800C36304EB8101042203EB8000FDF7E3FD58
:10C1E80072E1242A00F09C8611D8212A00F02B86BF
:10C1F800C0F0E985222A00F08B86232A7FF457AF06
:10C208005E4B1B68C1F80330FFF7C8FB5CE1272AC7
:10C2180000F0C3862CD8252A00F0B586262A7FF49C
:10C2280046AF574B554AD3F820121160D3F8241261
:10C23800564A1160D3F82822D3F82C12C3F8C42028
:10C24800534A1160D3F83022524983F8CC20D3F8EE
:10C258003422C3F81C22D3F83822C3F8182293F8E2
:10C268003C22885C08B10120885400225A702BE1D6
:10C27800282A00F0A486292A7FF419AF4B780B2BC3
:10C2880000F2C787DFE813F0390744074F075A075A
:10C29800660774077F079607A107AA07B207BD07B5
:10C2A800442A01F04E8300F28280342A01F0FF8193
:10C2B80033D82F2A27D011D82C2A01F0CB80C1F0EF
:10C2C80033802D2A01F05D812E2A7FF4F0AE2B4BAE
:10C2D8001B68C1F80330FEF771F8F5E0312A01F068
:10C2E800CC81C1F0BE81322A01F0D681332A7FF495
:10C2F800DEAE224B1B68C1F803308B78052B01F2A8
:10C30800D281FFF7A1FD214B1B68A3701B4B1B6853
:10C31800C4F80330FEF752F8D6E0392A01F0128249
:10C328001ED8362A01F0D581C1F0CA81372A01F01A
:10C33800EE81382A7FF4BBAE144B1B68FF2B00F24A
:10C34800C380154A52F823200C4B42601A60104BE8
:10C35800002A41F0E6811A6842F008021A60B3E048
:10C36800412A01F0E68219D8402A7FF4A0AE02F0F3
:10C3780035FBA9E02C6000204462002030620020D8
:10C38800D046002038600020040000204C620020C5
:10C3980034600020085A002050620020422A01F030
:10C3A800CC82432A7FF483AE02F022FB8CE0852AFC
:10C3B80001F004833FD8802A01F0D38221D8462A8D
:10C3C80001F0C782C1F0C182472A01F0C682502A13
:10C3D8007FF46DAEA14AD2F8C810072974D86078E6
:10C3E8000C2871D8DFE810F0BA09CC09DE09F00989
:10C3F800020A140A270A390A4B0A5D0A6F0A810AD7
:10C40800930A822A01F0CC82C1F0B182832A01F01A
:10C41800CD82842A7FF44BAE914A127D920701F1B6
:10C42800C982B3F5006F67D204218C4A82F8C01024
:10C43800C2F8403248E08A2A01F07A831CD8872A59
:10C4480001F04883C1F0C082882A01F0F982892A64
:10C458007FF42DAE4A78BABB8978A9BB40F2D242A4
:10C46800934231D140F2FF70FDF73AFCFDF794FB9F
:10C478000120FCF7F1F927E08D2A01F097830FD806
:10C488008B2A01F06E838C2A7FF411AE4E78002E31
:10C4980001F06D83012E01F07A830323037013E00A
:10C4A800F22A01F0D283FF2A7FF401AE40F2D24291
:10C4B800934209D10122694B83F8742204E08B78F6
:10C4C800052B19D8FFF7C0FC02B0BDE8F0818B78C6
:10C4D800052B11D8FFF720FDF6E78B78052B0BD835
:10C4E800FFF782FDF0E7FEF7BDFAEDE7FEF750FF34
:10C4F800EAE78B78052B02D904232B70E4E70323A2
:10C508002B70E1E78B78F5E78B78022B00F0CC8075
:10C51800032B00F0CE80002B40F00C814B78502B81
:10C5280000F0838028D8462B6CD00FD8422B61D0DE
:10C5380006D8402B45D0412B59D003232B7045E01A
:10C54800442B474B5CD059D95B7955E04B2B63D0D2
:10C558000AD8482B5CD058D3492BEED1404BDB7D11
:10C56800003318BF012347E04D2B5BD057D34F2B27
:10C57800E3D13B4B5B7E3FE0812B68D011D8542B35
:10C588005AD005D8522B364B54D051D91B6933E0B9
:10C59800572B54D0802B56D0552BCED1304BDB7E29
:10C5A8002AE0852B70D005D8832B69D064D92D4B10
:10C5B8001B6821E0FE2B02D073D8F02BBDD12A4B8B
:10C5C80016E040F2FF70FDF773FC6860274B1B789C
:10C5D800002B3FF479AF264B6A681A60254B002A76
:10C5E80040F0AA801A6842F008021A606CE71C4BF7
:10C5F8001B7801E01A4B5B786B60E7E71B79FBE778
:10C60800DB69F9E7164BDB68F6E7154B9B68F3E740
:10C61800134B93F82630EFE7114BDB78ECE7104B20
:10C628009B78E9E70E4B5B7DE6E70D4B9B7DE3E7E7
:10C638001B7DE1E71B6ADFE7094B9B7EDCE7084BC4
:10C6480093F82730D8E7054B93F8C030D4E7034B6D
:10C6580093F8C0301F1F7B427B41CDE7D0460020B6
:10C668000400002040620020EC5900203F620020B6
:10C678003062002034600020A14BD3F8C430BBE7FF
:10C688009F4BD3F8E431B7E743F239019C4A9D4800
:10C69800D2F8E83100FB0313C2F8E83123F0004375
:10C6A800AAE7994B1B785BE74A78984B53F82230F6
:10C6B800A2E74B78282B2ED015D8022B29D006D8E4
:10C6C8002BB3012B7FF439AF914B5B6894E7092BAF
:10C6D800FFF433AF0E2B7FF679AF272B7FF42DAF06
:10C6E8008B4B1B6B88E72B2B1BD007D8292B15D01E
:10C6F8002A2B7FF422AF864BDB6B7DE72D2B16D0E0
:10C7080012D32E2B7FF419AF814BDB6C74E7804B6F
:10C718004EE77F4B7AE77E4B5B6B6DE77C4B9B6B01
:10C728006AE77B4B1B6C67E7794B5B6C64E7784B7C
:10C738009B6C61E7042301E71A6822F008021A607B
:10C74800C2E68B78022B0CD1487837283FF6D7AE53
:10C7580000F5A7706F49800004220144FDF723FB10
:10C76800B2E604230370AFE68B78022B0CD148782D
:10C7780037283FF6C4AE00F5A7706649800004224A
:10C788000144FDF79BFB9FE6042303709CE6887831
:10C7980005283FF6B1AE4B78012B08D004D3022B05
:10C7A80008D003232B708FE602F034FC8CE602F0ED
:10C7B80039FC89E602F03EFC574B68601B78002B79
:10C7C8003FF482AE554B1860554B1A6818B942F0C1
:10C7D80008021A6078E622F008021A6074E64A78BD
:10C7E8001AB91846FBF7A4FF6EE6082A03D1D9B296
:10C7F800FCF73CF968E6092A7FF466AED9B2012055
:10C80800FCF734F960E64878072806D813B9FBF72F
:10C81800B1FE59E6FBF7C6FE56E6FF287FF46FAE79
:10C828005E1C0ABF3D4BD8B21878FBF7D3FE4BE627
:10C838008B78012B31D004D3022B32D00423037020
:10C8480005E04878082811D8FBF7D5FE6860324B18
:10C858001B78002B3FF438AE304B6A681A60304BB7
:10C868001ABB1A6842F008021A602DE60A2805D198
:10C87800FCF7EAF8003018BF0120E7E70D2803D1DC
:10C888000020FCF7CDF8E1E70E2801D10120F8E7F8
:10C89800FF28DCD1FBF71AFFD8E74878FDF740F905
:10C8A800D4E74878FBF7DEFED0E71A6822F00802E2
:10C8B8001A6009E61068184410601268184B002ABC
:10C8C80033D11A6842F008021A60FDE51068C01AF0
:10C8D800F2E710685843EFE7106890FBF3F0EBE7D6
:10C8E800116891FBF3F003FB10131360E5E7106880
:10C8F8001840E1E710681843DEE710685840DBE7A6
:10C90800D04600206D4EC6413E6200205062002095
:10C9180098590020185D00203F62002030620020F6
:10C92800346000201368DB43DFE71A6822F008024E
:10C938001A60C9E5A04A1168A04A8B4213680ADA4E
:10C9480023F0030343F004031360136869B943F049
:10C9580008031360B8E50BBF23F0060323F00503B3
:10C9680043F0010343F00203EEE723F008031360EA
:10C97800AAE54A780C2A3FF6A7ADDFE802F00710CF
:10C9880019222B343E475059626B74008B4A126847
:10C9980015077FF599AD8A4AC2F8C43094E5874AED
:10C9A800126814073FF590AD854AC2F8C4308BE58C
:10C9B800824A1268D0077FF587AD814AC2F8C43031
:10C9C80082E57E4A1268D1073FF57EAD7C4AC2F8FF
:10C9D800C43079E5794A126852077FF575AD784A0F
:10C9E800C2F8C43070E5754A126812F0050F3FF4BA
:10C9F8006BAD734AC2F8C43066E5704A126897078F
:10CA08007FF562AD6E4AC2F8C4305DE56B4A1268C4
:10CA180096073FF459AD6A4AC2F8C43054E5674AEC
:10CA28001268D5067FF550AD654AC2F8C4304BE5AB
:10CA3800624A126894067FF547AD614AC2F8C4306D
:10CA480042E55E4A126850067FF53EAD5C4AC2F880
:10CA5800C43039E5594A126811067FF535AD584A90
:10CA6800C2F8C43030E5554A1268D2057FF52CADBE
:10CA7800534AC2F8C43027E5514AC2F8C43023E506
:10CA88004F4AD2F8C81007293FF61EAD481CC2F815
:10CA9800C800D2F8C40002EB8101C1F8F801C2F85D
:10CAA800C43011E54B782E2B03D80121454AD154C7
:10CAB8000AE5FF2B7FF423AD0122414B1A7003E5F1
:10CAC8004B782E2B03D800213E4AD154FCE4FF2B8F
:10CAD8007FF415AD00223A4B1A70F5E4384D95F8FD
:10CAE800CC2072B90A205F1C04BF334B1B68584323
:10CAF800C5F81802FBF7E0FB0123C5F81C0285F80E
:10CB0800CC306378042B3FF6DFACDFE803F0034456
:10CB18007AA71A00FBF7D0FBD5F81C32C01A0028F8
:10CB2800D5F81832B8BF404298428BBF0023D5F8D9
:10CB3800C43085F8CC3003F1FF3398BFC5F8C43052
:10CB4800C2E4A07802F076FA38B91C4A85F8CC001D
:10CB5800136823F010031360B6E4D5F81832A3B1B4
:10CB6800FBF7AAFBD5F81C32C01A0028D5F81832F2
:10CB7800B8BF4042984208D90023104A85F8CC3003
:10CB8800136843F0100313609EE4D5F8C430013BEA
:10CB9800C5F8C43098E4A078352102F069FD10F496
:10CBA800007411D00023054A85F8CC30136823F0AF
:10CBB8001003136088E400BF306200203460002056
:10CBC800D0460020085A0020D5F818329BB1FBF750
:10CBD80073FBD5F81C32C01A0028D5F81832B8BF34
:10CBE8004042984207D9B44A85F8CC40136843F0CC
:10CBF8001003136068E4D5F8C430013BC5F8C430AD
:10CC080062E4A078352102F033FD10F0010408D069
:10CC18000023A94A85F8CC30136823F01003136069
:10CC280052E4D5F818329BB1FBF746FBD5F81C3215
:10CC3800C01A0028D5F81832B8BF4042984207D920
:10CC48009D4A85F8CC40136843F0100313603BE419
:10CC5800D5F8C430013BC5F8C43035E4A078352197
:10CC680002F006FD10F0020408D00023924A85F86D
:10CC7800CC30136823F01003136025E4D5F818327C
:10CC88009BB1FBF719FBD5F81C32C01A0028D5F860
:10CC98001832B8BF4042984207D9874A85F8CC4035
:10CCA800136843F0100313600EE4D5F8C430013B59
:10CCB800C5F8C43008E40022804B83F8C02003E4A0
:10CCC800FF287FF419AC7E4E42B300254FF00608CA
:10CCD80018276078042208FB00510138784300F5D2
:10CCE800C36000EB850006EB81010135FDF75BF8B9
:10CCF800062DEED1FFF7E8BB6119781904223144FB
:10CD08000435FDF750F8182DF6D11834B4F5FC7F2A
:10CD18003FF4DAAB002504F5C067EDE71824F9E71E
:10CD28004B78142B3FF6EBAB8A78052A1BD80621E3
:10CD380001FB0323624A52F82320624B42601B78AE
:10CD4800002B3FF4C1AB604B1A605B4B2AB91A68E1
:10CD580042F008021A60FFF7B7BB1A6822F008020F
:10CD68001A60FFF7B1BBFF2A7FF4C6AB544E43B33A
:10CD780000254FF0060818276078042208FB0051A8
:10CD88000138784300F5C36000EB850006EB8101AC
:10CD98000135FDF793F8062DEED1FFF795BB611924
:10CDA8007819042231440435FDF788F8182DF6D196
:10CDB8001834B4F5FC7F3FF487AB002504F5C06751
:10CDC800EDE71824F9E74B78142B3FF698AB8878F1
:10CDD80006061BD5002506273C4EDFF8E480B37E07
:10CDE8007BB163786BB1182007FB0351013B5843B3
:10CDF80000F5C360042208EB810100EB8500FCF715
:10CE0800D2FF0135062DEAD1FFF75EBB05283FF6B4
:10CE180073AB2E4A927E002A3FF456AB002B3FF4A8
:10CE280053AB0621182201FB0301013B5343244C59
:10CE380003F5C363042204EB810103EB8000FCF7D4
:10CE4800B2FFFFF741BB4A781F4B0A2A0CD8DFE82C
:10CE580002F006151A1F252D41464B5054001C4957
:10CE68001A6809680A441A601A68134B002A49D1DB
:10CE78001A6842F008021A60FFF726BB14491A68BC
:10CE88000968521AEFE7124A196812684A43EAE732
:10CE98000F491A68096892FBF1F2E4E70C4A18682E
:10CEA800116890FBF1F201FB1202DCE708491A68ED
:10CEB80009680A40D7E700BF34600020D046002048
:10CEC800386000203F62002030620020040000200B
:10CED8004C620020B1491A6809680A43C3E7AF49A0
:10CEE8001A6809684A40BEE7AC490A68D2430A6032
:10CEF800BAE71968A94A1160B6E7A84A196810681C
:10CF08001860F8E71A6822F008021A60FFF7DCBA1E
:10CF1800A34B1B68C1F80330FDF7A4FDFFF7D4BA93
:10CF28004B78052B3FF6D0AADFE803F0030A111867
:10CF38001F269C4A136803F00F031360FFF7C4BA57
:10CF4800984A136823F010031360FFF7BDBA954A97
:10CF5800136823F020031360FFF7B6BA914A1368E9
:10CF680023F040031360FFF7AFBA8E4A136823F02B
:10CF780080031360FFF7A8BA8A4A136823F4807302
:10CF88001360FFF7A1BA49782E293FF6B8AA864A56
:10CF980002EB81025360FFF797BA8A78052A3FF6B9
:10CFA800ABAA4B78142B3FF6AAAA062101FB032350
:10CFB8007B4A11687D4A42F82310FFF785BAFF2B98
:10CFC8003FF782AA4A780B2A00F29380DFE802F042
:10CFD80006111C2733414C57626B737F744AA07843
:10CFE80052F8233052F82010194442F82010FFF765
:10CFF8006BBA6F4AA07852F8233052F82010C91A39
:10D0080042F82010FFF760BA694AA17852F8233035
:10D0180052F82100434342F82130FFF755BA644AD9
:10D02800A07852F8233052F8201091FBF3F142F81F
:10D038002010FFF749BA5E4AA17852F8230052F847
:10D04800214094FBF0F300FB134342F82130FFF733
:10D058003BBA574AA07852F8233052F820101940AA
:10D0680042F82010FFF730BA514AA07852F823301E
:10D0780052F82010194342F82010FFF725BA4C4AFD
:10D08800A07852F8233052F82010594042F8201066
:10D09800FFF71ABA464AA17852F82330DB4342F820
:10D0A8002130FFF711BA424A52F82310A37842F808
:10D0B8002310FFF709BA3E4AA17852F8234052F8E4
:10D0C800210042F8214042F82300FFF7FDB9384A11
:10D0D800A17852F8233052F82110994240F33F8248
:10D0E800304A136823F0030343F004031360FFF787
:10D0F800EBB903230370FFF7E7B989782C4A28486E
:10D1080052F821300068034442F82130FFF7DCB9B7
:10D118008978274A224852F8213000681B1A42F8B9
:10D128002130FFF7D1B98978214A1D4B52F82100E7
:10D138001B68434342F82130FFF7C6B989781C4A77
:10D14800174852F82130006893FBF0F342F8213079
:10D15800FFF7BAB98978164A114B52F82140186876
:10D1680094FBF0F300FB134342F82130FFF7ACB90E
:10D1780089780F4A0A4852F821300068034042F87B
:10D188002130FFF7A1B98978094A054852F82130BA
:10D198000068034342F82130FFF796B94C6200203B
:10D1A8003062002034600020D04600203860002023
:10D1B800506200208978A34AA34852F821300068B9
:10D1C800434042F82130FFF77FB99F4B89781B68AD
:10D1D8009C4ADB4342F82130FFF776B99A4B8A78AC
:10D1E8001968984B43F82210FFF76EB98978954A69
:10D1F800954B52F821001C68186042F82140FFF74F
:10D2080063B9904B8A7853F822208F4B1B689A4257
:10D2180064E703230370FFF757B94A788A4B8B49B1
:10D228000B2A78D8DFE802F006161D242C363D4478
:10D238004B51565FA078834A52F820201868024460
:10D248001A601B68002B69D10B6843F008030B6058
:10D25800FFF73AB9A4787B481A6850F82400121AE4
:10D26800EEE7784AA07852F820001A684243E7E7C8
:10D27800A47874481A6850F8240092FBF0F2DFE7AB
:10D28800A078704A1C6852F8200094FBF0F200FB6A
:10D298001242D5E7A0786B4A52F82020186802405D
:10D2A800CEE7A078674A52F8202018680243C7E7FB
:10D2B800A078644A52F8202018684240C0E7A07855
:10D2C800604A52F82020D243BAE7A0785D4A52F863
:10D2D8002020B5E7A0785B4A1D6852F8204042F844
:10D2E80020501C60ADE7574AA07852F820001A6811
:10D2F80090420A6805DA22F0030242F004020A604A
:10D308009FE70BBF22F0060222F0050242F001025D
:10D3180042F00202F3E703222A7092E70B6823F037
:10D3280008030B60FFF7D0B84B780B2B00F2868010
:10D33800DFE803F006111C2733414C57626B737EFC
:10D348008978404A424852F821300068034442F83C
:10D358002130FFF7B9B889783A4A3D4852F8213068
:10D3680000681B1A42F82130FFF7AEB88978354AB1
:10D37800374B52F821001B68434342F82130FFF72E
:10D38800A3B889782F4A324852F82130006893FBB5
:10D39800F0F342F82130FFF797B88978294A2C4BE7
:10D3A80052F82140186894FBF0F300FB134342F84D
:10D3B8002130FFF789B88978224A254852F8213068
:10D3C8000068034042F82130FFF77EB889781D4A8B
:10D3D8001F4852F821300068034342F82130FFF714
:10D3E80073B88978174A1A4852F8213000684340C0
:10D3F80042F82130FFF768B8154B89781B68114A45
:10D40800DB4342F82130FFF75FB8114B8A7819687F
:10D418000C4B43F82210FFF757B88978094A0C4B90
:10D4280052F821001C68186042F82140FFF74CB8F8
:10D43800044B8A7853F82220054BE7E60323037050
:10D44800FFF742B8506200203062002034600020AC
:10D458004C6200204B780B2B00F28F80DFE803F042
:10D4680006101A242F3C46505A636B76B04A8978C6
:10D47800B04B53F8213011680B441360FFF724B800
:10D48800AB4A8878AB49136851F820105B1A1360CF
:10D49800FFF71AB8A64AA74B897853F821101368E2
:10D4A8004B431360FFF710B8A14A8878A149136865
:10D4B80051F8201093FBF1F31360FFF705B89C4A6D
:10D4C8009C4B8978106853F8211090FBF1F301FB0D
:10D4D80013031360FEF7F8BF954A8978954B53F804
:10D4E800213011680B401360FEF7EEBF904A89782F
:10D4F800904B53F8213011680B431360FEF7E4BFDB
:10D508008B4A89788B4B53F8213011684B40136054
:10D51800FEF7DABF8A78874B53F82230844ADB4318
:10D528001360FEF7D1BF834B8A7853F82220804BD3
:10D538001A60FEF7C9BF89787E4A7D4B52F82100F0
:10D548001C68186042F82140FEF7BEBF794B8A7804
:10D5580053F82220764B1B689A42FFF6C1AD764AF3
:10D5680013680BBF23F0060323F0050343F0010300
:10D5780043F002031360FEF7A7BF03230370FEF70F
:10D58800A3BF4A780B2A68D8DFE802F0060F1821F3
:10D598002B374049525B6761A178664A52F82100EF
:10D5A800184442F82100FEF78FBFA178614A52F86B
:10D5B8002100C01A42F82100FEF786BFA1785D4A13
:10D5C80052F82100584342F82100FEF77DBFA178A8
:10D5D800584A52F8210090FBF3F042F82100FEF778
:10D5E80073BFA178534A52F8214094FBF3F003FB30
:10D5F800104342F82130FEF767BFA1784D4A52F830
:10D608002100184042F82100FEF75EBFA178494A80
:10D6180052F82100184342F82100FEF755BFA178BF
:10D62800444A52F82100584042F82100FEF74CBF06
:10D63800A178404A52F82130DB4342F82130FEF706
:10D6480043BFA1783B4A42F82130FEF73DBFA1789D
:10D65800384A52F8212093427FE703230370FEF7EC
:10D6680033BFFCF74DFE0122344B83F8C020D4F8B9
:10D678000320C3F8C420FEF727BF48782D4951F886
:10D688002020013A002A41F820207EF71DAF2B4ABE
:10D69800C2F8C430FEF718BF294B1B68C1F8033025
:10D6A8008B78FEF715BF04230370FEF72CBE204BC2
:10D6B8001B688B70224B1B68C1F80330FEF704BF50
:10D6C8001B4B1B688B701E4B1B68C1F80330FEF7A1
:10D6D800FBBE174B1B788B70FEF700BF144B1B6803
:10D6E8008B70FDF7BFF9FEF7EFBE114B1B688B700F
:10D6F800FDF74EFEFEF7E8BE0D4B1B688B70104B16
:10D708001B68C1F80330FDF7ADF9FEF7DDBE084A26
:10D718001268FF2A3EF6D8AE064941F82230FEF7D5
:10D72800D3BE1A6822F008021A60FEF7CDBE00BF09
:10D738004C6200205062002034600020D046002057
:10D7480030620020D14B1B68FF2B3EF6BDAED04A9D
:10D758001168D04A42F82310FEF7B6BECE480068DA
:10D7680004077EF5B1AE481CC2F8C800D2F8C40060
:10D7780002EB8101C1F8F801C2F8C430FEF7A4BE7B
:10D78800C548006800073EF59FAE481CC2F8C800AF
:10D79800D2F8C40002EB8101C1F8F801C2F8C43024
:10D7A800FEF792BEBC480068C7077EF58DAE481CE0
:10D7B800C2F8C800D2F8C40002EB8101C1F8F80130
:10D7C800C2F8C430FEF780BEB3480068C6073EF50D
:10D7D8007BAE481CC2F8C800D2F8C40002EB810135
:10D7E800C1F8F801C2F8C430FEF76EBEAA48006856
:10D7F80045077EF569AE481CC2F8C800D2F8C400D7
:10D8080002EB8101C1F8F801C2F8C430FEF75CBE32
:10D81800A148006810F0050F3EF456AE481CC2F847
:10D82800C800D2F8C40002EB8101C1F8F801C2F8BF
:10D83800C430FEF749BE9848006884077EF544AEB8
:10D84800481CC2F8C800D2F8C40002EB8101C1F834
:10D85800F801C2F8C430FEF737BE8F480068800769
:10D868003EF432AE481CC2F8C800D2F8C40002EB3D
:10D878008101C1F8F801C2F8C430FEF725BE864818
:10D888000068C7067EF520AE481CC2F8C800D2F86A
:10D89800C40002EB8101C1F8F801C2F8C430FEF7F8
:10D8A80013BE7D48006886067EF50EAE481CC2F899
:10D8B800C800D2F8C40002EB8101C1F8F801C2F82F
:10D8C800C430FEF701BE7448006845067EF5FCAD1D
:10D8D800481CC2F8C800D2F8C40002EB8101C1F8A4
:10D8E800F801C2F8C430FEF7EFBD6B4800680406C3
:10D8F8007EF5EAAD481CC2F8C800D2F8C40002EBB5
:10D908008101C1F8F801C2F8C430FEF7DDBD6248F4
:10D918000068C0057EF5D8AD481CC2F8C800D2F82A
:10D92800C40002EB8101C1F8F801C2F8C430FEF767
:10D93800CBBD01F05BF8FEF7C7BD01F058F8FEF764
:10D94800C3BD01F056F8FEF7BFBD01F053F8FEF76E
:10D95800BBBD01F050F8FEF7B7BD01F04DF8FEF77A
:10D96800B3BD00224D4B83F8C020FEF7ADBD4A7809
:10D978002AB1012A09D003230370FEF7A5BD0122AD
:10D98800464B83F8C020FEF79FBDB3F5006FBEF489
:10D99800B3AD424981F8C020C1F8C430FEF794BD48
:10D9A80002223E4B83F8C020FEF78EBDFCF7A8FC90
:10D9B800FEF78ABD08230370FEF786BD0022374BA9
:10D9C80083F8C020FEF780BD0125354A354C157017
:10D9D800354AB3F5006F9078207027D2127D12EA8D
:10D9E800050623D118466946FCF7BAF89DF80030B9
:10D9F800267263709DF80130A3709DF80230E370C1
:10DA08009DF8063023719DF8053063719DF8043048
:10DA1800A3719DF80330E3712B46E15C227A013350
:10DA28000A44082B2272F8D1FEF74EBD2B4600227D
:10DA3800E2540133082BFBD123782372FEF744BD4F
:10DA48004B78012B19D005D3022B31D00323037057
:10DA5800FEF73ABD0122124B1A70134B114A9B78FC
:10DA68001370124B196800230139013311F8010FA3
:10DA7800082BD054F9D1FEF727BD18224371C27183
:10DA88000F23462203718271FEF71EBD4C620020EF
:10DA9800306200205062002034600020D046002010
:10DAA80034620020356200200400002000000020BD
:10DAB8000122874B87481A70874B884A9B781370D6
:10DAC80000230133191811F8091C082BD154F8D177
:10DAD800FEF7FABC4B78032B3EF6F6ACDFE803F012
:10DAE80002101E237E4B93F8C020C27193F8CC20FD
:10DAF800D3F8403282711A0A42710371FEF7E4BC0E
:10DB0800774B93F8C020C27193F8CC20D3F8C43077
:10DB180082711A0A42710371FEF7D6BC714B1B68F9
:10DB28004360FEF7D1BC704B1B684360FEF7CCBC6A
:10DB38004A786E4B9AB91A70E3786D4A1370684A3E
:10DB480092F844126B4A117000226B490A706B49B3
:10DB58000A706B4A11780B431370FEF7B5BC0122AB
:10DB6800E9E701225E4B83F84522FEF7ADBC0422AB
:10DB7800694640F2FB70FCF7A1F9009BD4F803203A
:10DB88009A420ABF01236E606B60FEF79DBC8B78DA
:10DB98002A2B07D104225B4940F2FB70FCF703F9FA
:10DBA800FEF792BC03230370FEF78EBC4A78032A63
:10DBB80047D8DFE802F01B0234420021484CD4F871
:10DBC800480204F5137281423EF47EAC52F82150AB
:10DBD8009D4201F1010520D102EB8503043B013888
:10DBE800814214D3C4F84802FEF76EBC3C4AD2F80E
:10DBF800481209298FBF0923481CC2F8480202EBC2
:10DC0800810294BFC2F84C322B70FEF75DBC53F80A
:10DC1800042F013143F8042CE2E72946D3E7002317
:10DC280019462F4AC2F8483202F5137242F82310F7
:10DC380001330A2BFAD1FEF747BC0A234360FEF7EB
:10DC480043BC03230370FEF73FBC4B78812B7EF463
:10DC58003BAC8B78922B7EF437AC8B79A32B7EF47C
:10DC680033AC4B79B42B7EF42FAC0B79C52B7EF4F7
:10DC78002BACCB78D62B7EF427AC8022224B5A8350
:10DC8800FCF736FBFAF718FB0446FAF715FB001BFE
:10DC98000028B8BF4042B0F57A7FF6DB72B60024A0
:10DCA800FAF7E8FD194B21461C60194803F017F8EC
:10DCB800174802F051FF02F009FA03F0D1F84FF0CB
:10DCC800804003F030FE2046FAF7C6FDFEF7FCBBA5
:10DCD8003462002000800008040000203562002023
:10DCE800D0460020306200204C6200207859002085
:10DCF8007B590020FB5900207A590020375A002010
:10DD0800795900202F6000200004024010E000E054
:10DD18001064024000232DE9F74F4FF0FF341946F5
:10DD28006B4A6C4D13606C4AC5F8C43013606B4A7B
:10DD3800C5F8C83013606A4A85F8CC302B706B7010
:10DD4800281D40F82340D15401332F2BF9D100244A
:10DD5800DFF8C4A1634B0AF1300B03EB841262496C
:10DD6800127E4FEA840901F13000002A7AD15F4A15
:10DD78004AF824204BF8242041F824205FFA84F83C
:10DD880040F82420272140460193002601F070FC2A
:10DD9800574F584A47F80900A6542621404601F033
:10DDA80067FC554A42F80900544A4046A654FAF717
:10DDB80083FDA7F19702A6542521404601F058FC9F
:10DDC800A7F1900242F809002421404601F050FCD6
:10DDD800A7F1780242F809002821404601F048FCE2
:10DDE800A7F1600242F809002A21404601F040FCF0
:10DDF800A7F1480242F809002321404601F038FC07
:10DE0800A7F1300242F809002B21404601F030FC0E
:10DE18000134183F062C47F80900019B9DD1384A68
:10DE280033463146904642F823100133B3F5807FDC
:10DE3800F9D1344CA37E93BBE37EA3B3237903F0DB
:10DE4800EF02012A3DD1012385F87532637D002B4D
:10DE58003BD0FAF793FCC0B3012385F8C03003B078
:10DE6800BDE8F08F284A4AF82420284A4BF8242095
:10DE7800274A41F82420274A80E7F11909EB0700CF
:10DE8800042251440437FCF719F8182FF5D1183635
:10DE9800B6F5FC7FD0D0002706F5C069EDE7182657
:10DEA800DFF878A0F7E74FF4A766A6F5A761304634
:10DEB800042241440436FCF701F8B6F5C36FF4D1E7
:10DEC800BCE7212BBFD00023BEE70023C5E700BF76
:10DED80030620020D04600204C62002034600020D0
:10DEE800085A0020845600206C48002089FF00084A
:10DEF8003448002058560020045800201C580020A0
:10DF08005062002004000020B9FE000821FF00082C
:10DF1800F9FE000861FF000854480020386000201E
:10DF2800F7B50F4C07460E4694E803008DE803004A
:10DF38000C498A700022C1F803300B4B0F704E70E9
:10DF48001A70FEF78FF821786368084A82F876120B
:10DF58009DE8030084E80300184603B0F0BD00BF45
:10DF6800446200202C6000203F620020D046002040
:10DF7800014B93F876027047D0460020F7B5044667
:10DF88001F4A63781F4D1370A3780E4695E8030067
:10DF98005370E3788DE80300937023796F4693718B
:10DFA80063795371A3791371E379D3700022164B07
:10DFB8001A70FEF757F8154B1A782B469AB9327033
:10DFC80072702A78B2706A78F270EA793271AA7936
:10DFD80072716A79B2712A79F27197E8030083E85D
:10DFE800030003B0F0BD012AF7D10948721EF11DE4
:10DFF80010F8014F02F8014F8A42F9D1EDE700BF4E
:10E008002C600020446200203F620020346200201F
:10E01800356200202DE9F043A84B8FB01B78A84C3F
:10E0280013B994F877326BB1A64B1B78063BDBB279
:10E03800192B04D8A44A22FA03F3D90702D40023DF
:10E0480084F8443294F84432A04E5A1E012A51D81A
:10E05800012B14BF082307238DF8183094F8783261
:10E068009B498DF819300023CA688DF81A30079239
:10E078003278002A33D18B688DF827208DF820302C
:10E08800944B19788DF8211059788DF82210D97988
:10E098008DF8231099798DF8241059791B798DF80A
:10E0A80025108DF8263006A8FBF770FA002800F036
:10E0B8004784894B1A789846002A00F09981874B43
:10E0C800874F1B78013B062B00F28E81DFE813F0A7
:10E0D8006C016C01EE018C018C018C011502012A86
:10E0E800E1D18048013306AA195C1A44082BD17182
:10E0F800F8D1D8E7032B40D194F87552002DD8D128
:10E10800337883BBDFF8C881724F98F8020098F81B
:10E1180001503B7805441D447B781D44FB791D4420
:10E12800BB791D447B791D443B791D44FAF7E8FD12
:10E1380098F80100FAF7E4FD3878FAF7E1FD787805
:10E14800FAF7DEFDF879FAF7DBFDB879FAF7D8FDCA
:10E158007879FAF7D5FD3879EDB2FAF7D1FD284686
:10E16800FAF7CEFDA5E7012BA3D15E4F785D013507
:10E17800FAF7C6FD092DF9D19BE7042B2BD1002313
:10E188000122534FDFF84C81B8787D7888F8013048
:10E198000544154488F80020C8F80430FAF7B0FDA3
:10E1A8007878FAF7ADFD98F80000FAF7A9FD98F825
:10E1B8000100FAF7A5FD98F80700FAF7A1FD98F80D
:10E1C8000600FAF79DFD98F80500FAF799FDEDB2FB
:10E1D80098F80400C1E7052B42D194F87552002D38
:10E1E8007FF467AF337883BBDFF8E480394F98F862
:10E1F800020098F801503B7805441D447B781D4483
:10E20800FB791D44BB791D447B791D443B791D4432
:10E21800FAF7F4FE98F80100FAF7F0FE3878FAF702
:10E22800EDFE7878FAF7EAFEF879FAF7E7FEB879BA
:10E23800FAF7E4FE7879FAF7E1FE3879EDB2FAF701
:10E24800DDFE2846FAF7DAFE33E7012B7FF431AF1B
:10E25800244F785D0135FAF7D1FE092DF9D128E769
:10E26800062B41D100230122194FDFF86880B878C6
:10E278007D7888F801300544154488F80020C8F8EE
:10E288000430FAF7BBFE7878FAF7B8FE98F8000081
:10E29800FAF7B4FE98F80100FAF7B0FE98F807000C
:10E2A800FAF7ACFE98F80600FAF7A8FE98F8050009
:10E2B800FAF7A4FEEDB298F80400C0E73E62002029
:10E2C800D04600202C600020110200023462002099
:10E2D8000400002044620020375A0020FB59002027
:10E2E8007A59002035620020072B3CD194F875320A
:10E2F800002B7FF4DEAE32785ABB904B9F7893F8B0
:10E3080001808F4B8DF800701D7858784744D97973
:10E318008DF802503D449A798DF80300284493F80B
:10E3280005C08DF80410014493F804E08DF8052029
:10E338000A440CEB020373448DF801808DF806C083
:10E348008DF807E08DF8083009216846FBF77EFF55
:10E35800AFE6012AF8D17B495A5C0DF80320013356
:10E36800092BF9D1F0E7082B7FF4A3AE0023012095
:10E37800734A72495370107053608A7849788DF8DF
:10E3880000200A4402448DF801108DF802008DF82F
:10E3980003308DF804308DF805308DF806308DF88F
:10E3A80007308DF80820CFE7644A397893688DF8EC
:10E3B80036108DF8303080238DF831308A238DF86F
:10E3C8003230002307218DF833308DF834308DF842
:10E3D80035308DF829308DF82A30D3680AA88DF8A1
:10E3E80028100B93FBF7D2F800233B7088F8003015
:10E3F800002384F84432337084F8773294F8743206
:10E4080013B10120FAF728FA94F845324BB194F881
:10E418007532B3FA83F35B0984F87532002384F804
:10E42800453206A8FBF702F9002800F048819DF85C
:10E438001830062B40F24381434B9DF820201A7078
:10E448009DF821205A709DF822209A709DF823206B
:10E458009A719DF824205A719DF825201A719DF80B
:10E468002620DA709DF81930079A84F87832334BF1
:10E478001B699A4204BF012384F87732F9F71CFF1D
:10E488000022324B1860324B1A709DF81830072B57
:10E498000CBF0123022384F8443294F8C0305A1E7A
:10E4A800012A57D9052B55D0012254E0DFF88C906A
:10E4B8003B7899F8020099F8015005440A351D4443
:10E4C800FAF71EFC99F80100FAF71AFC8020FAF70F
:10E4D80017FC8A20FAF714FC0020FAF711FC002038
:10E4E800FAF70EFC0020FAF70BFCEDB23878FAF7D1
:10E4F80007FC2846FAF704FC76E780218DF80E1011
:10E508008A218DF80F1000210C4A8DF810105078D0
:10E5180093783A788DF80C3003440A338DF80D005F
:10E528008DF811108DF812101344092103A88DF8E5
:10E5380013208DF81430FBF789FE55E704000020FE
:10E5480044620020356200202C600020E859002039
:10E558005C5900200022BE4B1A7094F8C030042B7E
:10E5680004D1BC4B19780A0640F1ED8194F8442295
:10E57800082A04D840F25113D340DF0701D4FDF72D
:10E5880071FD94F84432092B74D1F9F795FED4F84B
:10E59800EC31B14DC01A00282A68B8BF40429042F9
:10E5A80009D9AE4B1A78012A04BF02221A70F9F76A
:10E5B80083FEC4F8EC01F9F77FFED4F8F0316A68FD
:10E5C800C01A0028B8BF4042904209D9A34B5A78D4
:10E5D800012A04BF02225A70F9F76EFEC4F8F0014E
:10E5E800F9F76AFED4F8F431AA68C01A0028B8BF4F
:10E5F8004042904209D9994B9A78012A04BF0222D5
:10E608009A70F9F759FEC4F8F401237893B3637844
:10E6180083BB1D46914A9248D15C022940F087810C
:10E6280050F823104E1C00F0818184F83C320023FE
:10E638008C4A1268C4F820228B4A1268C4F8242233
:10E64800D4F8C420C4F8C410C4F82822874A126831
:10E65800C4F82C2294F8CC2084F8CC300123C4F8D8
:10E668003022D4F81C226370C4F83422D4F818225B
:10E67800C4F8382294F84432092B06D194F8C02003
:10E68800022A04BF052284F8C020D4F84822002AB0
:10E6980000F05681092B40F0538194F8C030012BCB
:10E6A80040F04E810023D4F8C410714850F823502C
:10E6B8008D4240F04181052384F8C03040E194F850
:10E6C8007552002D62D103A8FAF734FB00285DD0FB
:10E6D800FAF74CFB08B184F8795294F879229DF83E
:10E6E8000C10531CDBB22244092B84F8793282F8CF
:10E6F8007A127FF432AF002384F879325D4B94F8B4
:10E708007A125A788A4207D093F82720002A3FF4D1
:10E7180024AF91427FF421AF93F827308B4204BF96
:10E72800012384F87732002353495A5C01332A4481
:10E73800082BD5B2F9D194F88232AB4222D1454B9D
:10E7480094F87B221A7094F87C225A7094F87D22EF
:10E758009A7094F87E229A7194F87F225A7194F8EC
:10E7680080221A7194F88122DA70F9F7A5FD434BDB
:10E77800434A186000231370032284F8442284F863
:10E7880079328AE6042384F84432E6E694F875522E
:10E79800002D77D103A8FAF74FFC002872D0FAF7BA
:10E7A80069FC08B184F8795294F879229DF80C1024
:10E7B800531CDBB22244092B84F8793282F87A128E
:10E7C8007FF4CBAE002384F879322A4B94F87A127E
:10E7D8005A788A4207D093F82720002A3FF4BDAE22
:10E7E80091427FF4BAAE93F827308B4204BF0123DD
:10E7F80084F87732002320495A5C01332A44082BD5
:10E80800D5B2F9D194F88232AB421ED1114B94F8AB
:10E818007B221A7094F87C225A7094F87D229A70A0
:10E8280094F87E229A7194F87F225A7194F8802283
:10E838001A7194F88122DA70F9F73EFD0F4B104AED
:10E84800186000231370052297E706239BE700BF93
:10E858003F6200202C60002098590020085A0020B0
:10E86800D4460020306200204C6200203460002032
:10E878001C490020040000204A490020F0590020CB
:10E88800FA59002094F875527DBB0AAE3046FBF762
:10E8980007FD50B32B46F25C01331544082BEDB24B
:10E8A800F9D19DF83020AA427FF46DAF3B4B9DF81B
:10E8B80029201A709DF82A205A709DF82B209A70EA
:10E8C8009DF82C209A719DF82D205A719DF82E20C4
:10E8D8001A719DF82F20DA70F9F7EEFC0022304B00
:10E8E8001860304B1A700723D5E594F8C030013B07
:10E8F800012B3FF632AED4F8C430B3F5006F11D215
:10E90800F9F73CFF70B1FAF79FF858B9D4F8C4008A
:10E918002249431CC4F8C430FBF722F9092384F8C0
:10E928004432C1E5002384F8C03016E6D5540133DB
:10E938002F2B7FF471AE9DE601339A427FF4B6AE79
:10E948000FB0BDE8F08394F84402082804D840F2D8
:10E958005112C240D207F3D4D4F84002124DD3F872
:10E968000330B0F5006F69706B6012D20B49FBF78A
:10E97800F1F90A49D4F84002FBF75AF938B1D4F84A
:10E9880040320133C4F8403265232B70D8E707239F
:10E99800FBE707232B7000238EE600BF2C600020C6
:10E9A800F0590020FA59002044620020704710B541
:10E9B800F9F782FC074C2368C01AB0F5FA7F07D92B
:10E9C800054A536983F010035361F9F775FC206019
:10E9D80010BD00BF506600200000024008B5F9F7DE
:10E9E8000BFF014B586008BD446200207047704718
:10E9F8007047704770477047704700BF73B5134E34
:10EA08000446335C0D463BB1114B262153F82020B8
:10EA180000F0FEFD0023335585EAE572A2EBE572AE
:10EA28002046272100F0F4FD01220A4B002D1A553B
:10EA38004FF00003D8BF02220093019220211A460A
:10EA4800204600F0A9FD02B070BD00BF1C58002090
:10EA580004580020585600202DE9F04F352185B084
:10EA6800044600F005FEC149024689464FEA841B68
:10EA780001EB0B052B7A410813F0400F00F0010061
:10EA88006F681DBF01F00108C1B259F80B005FFAA9
:10EA980080F815BFC0F1000A01F001017F4259F862
:10EAA8000BA01D0603F03F0603920291204632D5C3
:10EAB800F9F7AAFFB0FA80F30299039A5B090A2EC4
:10EAC80000F287810120B04010F4C06F40F004824A
:10EAD80010F4F07F40F00E8110F01E0F00F07981E5
:10EAE800A34D2B5D013B122B00F27381DFE813F07D
:10EAF8001B002A003900460056005F006E007C00AB
:10EB0800AC00CE00D40071017B027101710171016A
:10EB18007101EB018002F9F777FF031C18BF01238D
:10EB2800039A0299CBE73421204600F0A1FD012287
:10EB380005EB84039860023E8E4B96421A551AD80C
:10EB4800022319E005EB84039A6842F0020234219B
:10EB5800204600F05DFD51462046FFF74FFF032396
:10EB68000AE0002900F035812121204600F080FDCF
:10EB7800814B43F8240004232B552AE105EB840339
:10EB88009A6842F001023421204600F041FDCAF1A2
:10EB980000012046FFF732FF0523EDE7B8F1000F2B
:10EBA80000F01781204601F063F90623E4E705EB3E
:10EBB80084039A683421204622F0030200F028FDDD
:10EBC80039462046FFF71AFF0723D5E7B8F1000FAB
:10EBD80040F0FF8041462046FFF710FF794220466B
:10EBE800FFF70CFF0823C7E7B8F1000F00F0F1802A
:10EBF8002121204600F03CFD064600212046FFF773
:10EC0800FDFE5D4A342152F8243020469B1B42F811
:10EC1800243005EB84039A6822F0030200F0F8FC24
:10EC28003A462721204600F0F3FC32462D212046A3
:10EC380000F0EEFC00232021019300931A462046A1
:10EC480000F0AAFC092397E7900540F1C280212132
:10EC5800204600F00DFD494B002118602046FFF7C3
:10EC6800CDFE00222D21204600F0D2FC00222121D9
:10EC7800204600F0CDFC033E00223921204600F05A
:10EC8800C7FC012E00F2B2817942B6E0B8F1000F5C
:10EC980000F09F800B236FE7B8F1000F40F09980D8
:10ECA8002121204600F0E4FC414606462046FFF7B5
:10ECB800A5FE05EB84039A68342122F0030220465E
:10ECC80000F0A6FC3A462721204600F0A1FC0222CB
:10ECD8002D2196FBF2F2204600F09AFC4346CDF82F
:10ECE8000480CDF800801A462021204600F054FC0C
:10ECF8000D2341E71E4D285D0138122869D8DFE849
:10ED080010F0130024003F004B005C0068006B000B
:10ED18006800680093009D008100C20068006800D8
:10ED280068006800E20077010122124B3421204676
:10ED38001A5500F09DFC05EB8403062E98603FF4FD
:10ED4800FFAE082E7FF417AFFAE6062E05D105EBC5
:10ED580084039A6822F00302F7E6082E7FF4FBAEDC
:10ED680005EB84039A6822F00302F0E6845600203B
:10ED7800544900205856002060590020805900202E
:10ED8800721F012A05D821B1062E3FF4F4AE1323D1
:10ED9800F2E6F3B10C23EFE6052E05D105EB84036B
:10EDA8009A6822F00302ECE6072E7FF4F0AE05EB3A
:10EDB80084039A6822F00302E5E6721F012A05D847
:10EDC800B8F1000F02D0052EE1D1B9E6002B7FF48F
:10EDD800FBAE05B0BDE8F08F002BFAD1073E012E3F
:10EDE8000AD905EB84039A68342122F0030242F021
:10EDF8000202204600F00CFC39462046FFF7FEFDD3
:10EE08000A23B9E6002BE4D1073E012E7FF63CAF7A
:10EE180005EB84039A68342122F0030242F00102D0
:10EE2800204600F0F5FB2FE7002BD2D02121204609
:10EE380000F01EFC05EB840318622BE7002BC8D1F9
:10EE480021212046029300F013FC064605EB8408B6
:10EE5800D8F80820342122F00302204600F0D8FB1D
:10EE68003A462721204600F0D3FBD8F820202D2150
:10EE780016440222204696FBF2F200F0C9FB029BE0
:10EE8800019300932FE79105A3D512232121204652
:10EE98002B5500F0EDFB5B4B002118602046FFF777
:10EEA800ADFD204600222D2100F0B2FB20460022B5
:10EEB800212100F0ADFB00223921204605B0BDE834
:10EEC800F04F00F0A5BB342105EB84039A68204677
:10EED80000F09EFB00234FE64B4D2B5D013B122BB0
:10EEE8003FF677AF01A151F823F000BF41EF0008CA
:10EEF80069EF0008DBED00087FEF0008DBED000894
:10EF0800DBED0008DBED0008DBED0008DBED0008B9
:10EF1800DBED0008DBED0008DBED0008EFEF000893
:10EF280097EF0008AFEF0008BDEF0008C7EF000833
:10EF380003F00008F9EF00083821204600F098FB9C
:10EF480005EB8403986340F488723821204600F06A
:10EF58005FFB092E3FF4F4AD0A2E7FF43AAF0AE6C0
:10EF68002A492046F9F743FD59F80B102046FFF7C8
:10EF780045FD0E2300E626492046F9F738FD59F8E5
:10EF88000B1020464942FFF739FD0F23F4E52046D0
:10EF9800F9F72AFD0028FFF61CAF00212046FFF7ED
:10EFA8002DFD1023E8E52046F9F71EFD00283FF760
:10EFB80010AFF2E752057FF50CAF1123DCE52046D0
:10EFC800F9F712FD21210246204600F021FB3A46BE
:10EFD8002721204600F01CFB00222D21204600F0AE
:10EFE80017FB00234CE793057FF5F3AE1223C3E527
:10EFF80000212046FFF702FDF8E705EB84039A6B32
:10F00800382164E78059002054490020003665C43F
:10F0180000CA9A3B024B1A5C0AB901221A5470477B
:10F0280054490020024B1A5C0AB113221A54704743
:10F0380054490020014B185C704700BF5449002018
:10F04800014B53F820007047A44900202DE9F74FE1
:10F058009F4DEB69ABB19F4E347894B9F9F72CF911
:10F068009D4B1B68C01A0028EB69B8BF4042984204
:10F0780007D92046013400F0FBFE062CF9D1012304
:10F0880033702B6AABB1954E347894B9F9F714F90B
:10F09800934B1B68C01A00282B6AB8BF404298429D
:10F0A80007D92046013400F0E3FE062CF9D10123EC
:10F0B8003370F9F7C9FC68B98A4C257E95B1012DE2
:10F0C80000F0D2808022884B5A830122A3F5806306
:10F0D8005A8315E000242046013400F0C9FE062CAE
:10F0E800F9D1E9E72846F9F79BFC05460120F9F72D
:10F0F80097FC854204D0F9F7DFF80123E061237615
:10F10800F9F7DAF894F8383004EB83031B6AC01A6D
:10F118000028B8BF40420A2826DDF9F7CDF821219A
:10F12800074694F8380000F0A3FA064694F83880A9
:10F1380004EB8805E86B301A05F074FD8146286AEF
:10F14800381A05F06FFD0146484605F073FE05F0D4
:10F1580099F95DA3D3E9002305F0E8F905F080FCEF
:10F168002F6244F82800EE63352194F8380000F047
:10F178007FFA10F0400706460FD094F8380000F0E8
:10F1880077FE012194F83830584AD154584A0F3341
:10F19800D15C012904BF0221D15494F83800554D9F
:10F1A80005EB80131B69002B77D0222100F060FA51
:10F1B80094F83880002805EB88131B69B8BF4042D3
:10F1C80098426AD904EB080393F854307BB9342188
:10F1D800404600F04DFA342140F48062404600F089
:10F1E80017FA012294F83830234483F8542094F80D
:10F1F8005A30DFF808B173B998465FFA88F0F9F722
:10F20800FAF90BF8080008F10108B8F1080FF4D171
:10F21800012384F85A304FF027084FF000090222E2
:10F228003549DFF8CCA05FFA89F08DE80600F9F7D8
:10F23800E2F99DE806001BF80930834267D009F11E
:10F248000C0351F823300BF80900022B58D0032B7C
:10F2580003D0012B5BD1002859D01AF80830012BB4
:10F2680008BF0AF8082052E0F9F726F8E369C01A3F
:10F2780040F6FC030028B8BF4042984201DD022353
:10F288003DE70020F9F7CCFB06462846F9F7C8FB0E
:10F2980086427FF435AF002331E794F8388004EBD9
:10F2A800080393F85430002BA1D03421404600F0D5
:10F2B800DFF9342120F48062404600F0A9F994F87F
:10F2C80038300022234490E7FCA9F1D24D629040E7
:10F2D80004000020FA590020F05900205C59002051
:10F2E800E8590020A4490020000402407856002074
:10F2F800085A00208456002098590020FF49002011
:10F3080028B91AF80800012801D10AF8083009F1CB
:10F318000109B9F1080F08F1010884D194F83830CF
:10F3280016F0010104EB030200F0D98092F8631093
:10F3380081B9012182F863108F4A1A4492F8242077
:10F34800D00707D58B408D4A1B33D15C012904BFF8
:10F358000221D15494F83830B00704EB030292F834
:10F36800691040F1CC8091B9012182F86910824A74
:10F378001A4492F82A2012F0010F08D07F4A0E335F
:10F3880012F81310012904BF022102F8131016F015
:10F39800800100F0EC8094F83830784A0333D05C70
:10F3A800012801D10220D0544FB194F83830734A63
:10F3B8000F33D05C012801D10220D05401B3DFF80B
:10F3C800C8E194F838009EF8003043FA00F2D207FA
:10F3D80011D50121DFF8B4C101FA00F28CF8002040
:10F3E800DFF8ACC18CF800106549097819B923EA2F
:10F3F80002038EF800308022352100F009F92FB180
:10F408004022352194F8380000F002F994F83800C9
:10F4180005EB80131B6A23B3770522D4392100F04A
:10F4280027F92121064694F8380000F021F994F8CC
:10F438003830301A05EB83120028126AB8BF4042F0
:10F4480090420ED9184600F013FD012194F8383087
:10F458004C4AD154494A1533D15C012904BF0221D1
:10F46800D15494F8383005EB831292F82400C6067C
:10F4780007D5444A00F00F00D35C002B4CD0F9F7B5
:10F4880091F894F8380005EB801393F82430990626
:10F498000ED53C4B1B5C002B41D000F0E1FC38B989
:10F4A80094F8380000F0E4FC94F83800F9F701FA11
:10F4B80094F8383005EB831595F82420520637D494
:10F4C80094F83800FFF7C8FA94F838300133DBB203
:10F4D800052B4AD884F8383003B0BDE8F08F92F88D
:10F4E800630000283FF436AF82F86310224A1A44BA
:10F4F80092F8242092077FF52DAF5B0023E70029BF
:10F508003FF445AF012182F869101B4A1A4492F86A
:10F518002A2012F0020F30E7F9F72CF8B1E700F0D3
:10F528009FFC0028C4D094F83800F9F7BFF9BFE76A
:10F53800144AD55C75B10025E8B200F091FC28B9F1
:10F54800284600F095FC2846F9F7B3F90135062D51
:10F55800F2D1B5E7E8B200F083FC10B12846F9F71C
:10F56800A5F90135062DF5D1AAE70023B2E7002F4A
:10F578003FF44CAF19E700BF98590020085A002003
:10F5880078590020525600207B5900207A590020D3
:10F59800375A0020000000002DE9F04792469846AF
:10F5A800194B814613F810500C46002241F0800197
:10F5B80028469DF820709DF82460FAF737F9002254
:10F5C80051462846FAF732F9414600222846FAF70A
:10F5D8002DF9394600222846FAF728F93146012242
:10F5E8002846FAF723F9062304F07F0403FB049462
:10F5F80048EA0A2847EA0827044B46EA072643F858
:10F608002460BDE8F08700BF08550108144A0020AF
:10F61800F8B51546144B074613F810600C4600223F
:10F6280041F080013046FAF701F90022290E3046F0
:10F63800FAF7FCF80022C5F307413046FAF7F6F866
:10F648000022C5F307213046FAF7F0F80122E9B2A3
:10F658003046FAF7EBF8062304F07F0403FB047442
:10F66800024B43F82450F8BD08550108144A0020FD
:10F67800294B70B501F07F069A19127B002A43D0F6
:10F6880013F81050002231462846FAF7CFF8002226
:10F6980028461146FAF7CAF8002228461146FAF712
:10F6A800C5F8002228461146FAF7C0F801220021C1
:10F6B8002846FAF7BBF8002228461146FAF7B6F8AA
:10F6C800002228461146FAF7B1F800220402114632
:10F6D8002846FAF7ABF80022044311462846FAF701
:10F6E800A5F824020443012200212846FAF79EF8CF
:10F6F8002402222E40EA040001D0422E0AD103023D
:10F7080008D540F07F4070BD062303FB0606034B77
:10F7180053F8260070BD00BF08550108144A0020A0
:10F7280070B50B4C0546221892F8002C0E465AB9B3
:10F738006C21FFF79DFF06F00F0320F00F021A431C
:10F748006C212846FFF764FF631983F8066C70BDC7
:10F75800144A002038B50C466C210546FFF788FF8F
:10F76800240104F0700420F0700222432846BDE80A
:10F7780038406C21FFF74CBF38B50C466C21054664
:10F78800FFF776FFE40304F4C03420F4C0322243C8
:10F798002846BDE838406C21FFF73ABF38B50C461B
:10F7A8006C210546FFF764FF240504F4700420F477
:10F7B800700222432846BDE838406C21FFF728BF75
:10F7C80038B50C466C210546FFF752FF240604F0B5
:10F7D800706420F0706222432846BDE838406C21EE
:10F7E800FFF716BF38B50D466C210446FFF740FFFA
:10F7F8003DB140F080422046BDE838406C21FFF71B
:10F8080007BF20F08042F6E738B50D466C21044664
:10F81800FFF72EFF3DB140F400222046BDE83840F6
:10F828006C21FFF7F5BE20F40022F6E738B50D4647
:10F838006C210446FFF71CFF3DB140F480222046AE
:10F84800BDE838406C21FFF7E3BE20F48022F6E7DC
:10F8580038B50D466C210446FFF70AFF3DB140F468
:10F8680080422046BDE838406C21FFF7D1BE20F425
:10F878008042F6E738B50D466C210446FFF7F8FEDE
:10F888003DB140F400522046BDE838406C21FFF7F6
:10F89800BFBE20F40052F6E738B50D466C21044689
:10F8A800FFF7E6FE3DB140F480522046BDE83840FF
:10F8B8006C21FFF7ADBE20F48052F6E738B50C4650
:10F8C8006C210546FFF7D4FE230748BF20F07000DF
:10F8D8004FEA04124CBF40F4006020F4076002F0C5
:10F8E800700202436C212846BDE83840FFF790BEFD
:10F8F80038B50C466C210546FFF7BAFEE40104F45E
:10F90800F06420F4F06222432846BDE838406C21B8
:10F91800FFF77EBEFFF7ECBF08B5074B034493F82B
:10F92800002C2AB96C21FFF7A3FE00F00F0008BDD8
:10F9380093F8060C08BD00BF144A002008B56C21D6
:10F94800FFF796FEC0F3021008BD08B56C21FFF75B
:10F958008FFEC0F3C13008BD08B56C21FFF788FEE3
:10F96800C0F3035008BD08B56C21FFF781FEC0F352
:10F97800036008BD08B56C21FFF77AFEC0F38070FC
:10F9880008BD08B56C21FFF773FEC0F3C04008BD81
:10F9980008B56C21FFF76CFEC0F3804008BD08B5C0
:10F9A8006C21FFF765FEC0F3803008BD08B56C21F7
:10F9B800FFF75EFEC0F3403008BD08B56C21FFF7C5
:10F9C80057FEC0F3003008BD08B56C21FFF750FEA4
:10F9D800C0F30213020548BF43F00803184608BDE8
:10F9E80008B56C21FFF744FEC0F3C31008BDFFF74C
:10F9F800F7BF38B50C466D210546FFF739FE64019F
:10FA080004F0600420F0600222432846BDE8384034
:10FA18006D21FFF7FDBD38B50C466D210546FFF792
:10FA280027FE640304F4C04420F4C042224328465D
:10FA3800BDE838406D21FFF7EBBD38B50C466D21A8
:10FA48000546FFF715FE240204F4706420F4706282
:10FA580022432846BDE838406D21FFF7D9BD38B5A7
:10FA68000C466D210546FFF703FE04F00F0420F055
:10FA78000F0222432846BDE838406D21FFF7C8BD74
:10FA880038B50D466D210446FFF7F2FD20F47F00DE
:10FA980040EA05426D212046BDE83840FFF7B8BD71
:10FAA80038B50D466D210446FFF7E2FD3DB140F43F
:10FAB80000422046BDE838406D21FFF7A9BD20F47B
:10FAC8000042F6E738B50D466D210446FFF7D0FD34
:10FAD8003DB140F080722046BDE838406D21FFF707
:10FAE80097BD20F08072F6E708B56D21FFF7C0FDDD
:10FAF800C0F3411008BD08B56D21FFF7B9FDC0F38B
:10FB0800413008BD08B56D21FFF7B2FDC0F30320F1
:10FB180008BD08B56D21FFF7ABFD00F00F0008BD6B
:10FB280008B56D21FFF7A4FD0314D8B21B0648BF22
:10FB380060F0FF0008BD08B56D21FFF799FDC0F31F
:10FB4800C03008BD08B56D21FFF792FDC0F3006015
:10FB580008BD38B50C4670210546FFF789FD04F04D
:10FB6800030420F4401242EA04522846BDE8384013
:10FB78007021FFF74DBD38B50D4670210446FFF7DB
:10FB880077FD3DB140F400222046BDE838407021A1
:10FB9800FFF73EBD20F40022F6E738B50D46702188
:10FBA8000446FFF765FD3DB140F480222046BDE8DC
:10FBB80038407021FFF72CBD20F48022F6E738B5D5
:10FBC8000C4670210546FFF753FD04F0030420F4AA
:10FBD800403242EA04422846BDE838407021FFF727
:10FBE80017BD38B50D4670210446FFF741FD20F4D6
:10FBF8007F4040EA052270212046BDE83840FFF7E3
:10FC080007BD38B50D4670210446FFF731FD20F0D9
:10FC1800FF0045EA000270212046BDE83840FFF7A2
:10FC2800F7BC08B57021FFF723FDC0F3015008BDEC
:10FC380008B57021FFF71CFDC0F3C04008BD08B52A
:10FC48007021FFF715FDC0F3804008BD08B570218D
:10FC5800FFF70EFDC0F3014008BD08B57021FFF79E
:10FC680007FDC0F3072008BD08B57021FFF700FDA8
:10FC7800C0B208BD70B50E466F2115461C46FFF789
:10FC8800F7FC16B1C0F30903336015B1C0F30443A0
:10FC98002B700CB1000E207070BD2DE9F347F8F7FA
:10FCA8000BFB0446F8F708FB001B0028B8BF4042CE
:10FCB8000928F7DD0025554EA9463746DFF858A133
:10FCC800ECB243F2930200212046FFF7A1FC0C237B
:10FCD80001930093002309211A462046FFF75CFC94
:10FCE800022253234FF00A088DE80C006C214123AF
:10FCF80000222046FFF750FC0123002241462046FF
:10FD0800CDF80480CDF80090FFF746FCBB7A1021AF
:10FD1800DB0801937B7A2046DB08009300231A4610
:10FD2800FFF73AFC524670212046FFF771FC204647
:10FD3800FFF7F2FD364B00225855063B05F80390B5
:10FD480020212046FFF764FC00222D212046FFF7E2
:10FD58005FFC002221212046FFF75AFC01222321C3
:10FD68002046FFF755FCDC2224212046FFF750FCF3
:10FD780046F6DB0225212046FFF74AFC40F2B7127F
:10FD880026212046FFF744FC4DF2B71227212046D2
:10FD9800FFF73EFC40F2B71228212046FFF738FC57
:10FDA800DC222A212046FFF733FC42462B2120463D
:10FDB800FFF72EFC0135174A14212046FFF728FCCF
:10FDC800062D07F140077FF47BAFF8F775FA044674
:10FDD800F8F772FA001B0028B8BF40423128F7DD57
:10FDE8000024B37AE0B2DB080193737A0022DB08BF
:10FDF8000093102107230134FFF7CEFB062C06F1F0
:10FE08004006EED102B0BDE8F08700BF845600205E
:10FE18001A560020FFFF0F001E000CC438B5074C0F
:10FE2800044494F8001C41B994F8065CFFF778FC88
:10FE3800012384F8065C84F8003C38BD144A00208D
:10FE4800064B034493F8002C32B1002293F8061CA9
:10FE580083F8002CFFF764BC704700BF144A0020E9
:10FE6800024B184490F8000C704700BF144A002059
:10FE780037B501250C4BC4B21D540C4B00221D5440
:10FE880027212046FFF7C4FB20464FF6FF722621A4
:10FE9800FFF7BEFB0023019500931A462021204658
:10FEA800FFF77AFB03B030BD585600201C580020DD
:10FEB800002808B50BDB04F0D3FA0BA3D3E9002321
:10FEC80004F05EFC05F070FA04F0CAFD08BD04F009
:10FED800C7FA05A3D3E9002304F052FC05F0D4F9CE
:10FEE800F2E700BFAFF3008034F7FFFF7F84EE3FF7
:10FEF80008B504F0B5FA06A3D3E9002304F040FCE2
:10FF080005F052FA04F0ACFD08BD00BFAFF3008065
:10FF1800EB1100A2941A5D40002808B50BDB04F031
:10FF28009FFA0BA3D3E9002304F000FB05F0ACF91A
:10FF380004F096FD08BD04F093FA05A3D3E9002365
:10FF480004F0F4FA05F030FAF2E700BFAFF30080EE
:10FF580034F7FFFF7F84EE3F08B504F063FE04F03A
:10FF680091FA05A3D3E9002304F0E0FA05F08CF92F
:10FF780004F076FD08BD00BFEB1100A2941A5D40A5
:10FF8800704700BF7047FEE7FEE7FEE7FEE77047F1
:10FF9800704770477047000000212E4B82B01A68E6
:10FFA80042F001021A6099601A6822F0847222F401
:10FFB80080321A60284A5A601A6822F480221A602D
:10FFC800D9600091019119461A6842F480321A608A
:10FFD8001A6802F400320192009A01320092019AE2
:10FFE8001AB9009AB2F5A06FF2D10B6813F4003376
:08FFF80018BF01230193019BD6
:020000040801F1
:10000000012B04D0174B184A9A6002B07047134B6B
:100010009A689A609A6842F400429A609A6842F438
:10002000A0529A60114A5A601A6842F080721A60AF
:100030001A689201FCD540F203710D4A11609A686A
:1000400022F003029A609A6842F002029A60034A20
:10005000936803F00C03082BFAD1D3E70038024071
:100060001030002400ED00E000800008081E40056C
:10007000003C0240144A10B59068144900F00C008E
:100080000428134B01D008280AD00B600E4B9B6844
:10009000C3F303130B441A790B68D3400B6010BDF4
:1000A00054685068526800F03F00B3FBF0F3C2F3AD
:1000B00088125343044A5268C2F30142013252008B
:1000C000B3FBF2F3E1E700BF00380240BC000020C0
:1000D0000024F40008B501214FF4807001F0D8F934
:1000E000BDE8084000214FF4807001F0D1B94368A9
:1000F0000A7923F0407323F4807343EA02230A68E9
:1001000010B513434360CA680B69846813438A6857
:100110001343084A224013434A7943EA4203836067
:100120000A7DC36A013A23F47003D2B243EA025350
:10013000C36210BDFDF7FFC000230360037143716C
:100140008360C3600361012303757047074990E82A
:100150000C0010B513434C68054A224013438268D3
:100160001343C26813434B6010BD00BF002301401E
:10017000E030FCFF0023036043608360C36070478E
:10018000836819B143F001038360704723F00103D2
:10019000FAE7436823F4400323F4007319434160F2
:1001A0007047416282627047436823F01F0319431E
:1001B00041607047044B5A6818B142F400025A601B
:1001C000704722F40002FAE700230140044B5A680A
:1001D00018B142F480025A60704722F48002FAE7B4
:1001E00000230140092970B51BD90726A1F10A0493
:1001F000C56804EB4404A64025EA060503FA04F4A6
:100200002C43C460062A18D81F24013A436B02EB22
:100210008202944023EA040301FA02F21A43426381
:1002200070BD0724056901EB4106B44025EA0405C9
:1002300003FA06F42C430461E4E70C2A0CD81F24CB
:10024000073A036B02EB8202944023EA040301FAAB
:1002500002F21A43026370BD1F240D3AC36A02EB17
:100260008202944023EA040391401943C16270BDA5
:10027000836843F0804383607047836819B143F417
:1002800080638360704723F48063FAE7836819B161
:1002900043F002038360704723F00203FAE74368E8
:1002A000013923F4604343EA4133436070474368B4
:1002B00019B143F400634360704723F40063FAE725
:1002C000C06C80B27047014B18687047082301402A
:1002D000836819B143F480738360704723F480739B
:1002E000FAE7836819B143F400738360704723F41D
:1002F0000073FAE7044B5A6818B142F400525A608E
:10030000704722F40052FAE700230140092970B532
:100310001CD90726A1F10A04C56804EB4404A640D1
:1003200025EA060503FA04F42C43C460836B023209
:10033000C3F30154121B1F24D2B202EB8202944079
:1003400023EA040391401943816370BD07240569C2
:1003500001EB4106B44025EA040503FA06F42C43F8
:100360000461E3E7836B013923F4401343EA01534B
:1003700083637047002382B001930190019B19446D
:100380000191019B1A6002B07047836823F47023C7
:10039000194381607047836823F4401319438160D7
:1003A0007047836843F48003836070478068C0F3BC
:1003B00080507047FFF7FABF436819B143F4806378
:1003C0004360704723F48063FAE7436819B143F44C
:1003D00080534360704723F48053FAE7002382B0D0
:1003E00001930190019B283319440191019B1868E6
:1003F00080B202B070470123C9B203FA01F1436829
:1004000012B119434160704723EA0101FAE703681A
:10041000194214BF012000207047C9430160704792
:100420004268006810EA112007D00123C9B203FA1C
:1004300001F1114214BF1846002070476FEA1121E4
:100440000160704708B50B4B012198420AD14FF06B
:10045000007001F011F800214FF00070BDE8084075
:1004600001F00AB84FF0806001F006F800214FF06B
:100470008060F3E700640040036823F00203036038
:10048000036843F0010303604FF480334268D207EE
:1004900001D4013BFAD1436813F0010354D08B79A6
:1004A000012B03680CBF43F0800323F0800303603B
:1004B000CB79012B03680CBF43F0400323F04003CA
:1004C00003600B7A012B03680CBF43F0200323F079
:1004D000200303604B7A012B03680CBF43F0100329
:1004E00023F0100303608B7A012B03680CBF43F0E9
:1004F000080323F008030360CB7A012B03680CBFC9
:1005000043F0040323F004030360CB788A781B06CE
:1005100043EA82730A7943EA02434A7943EA02537F
:100520000A88013A1343C361036823F0010303609F
:100530004FF480334268D20701D5013BFAD14068BD
:10054000C04300F0010070471846704730B50125E0
:10055000837A354A9D40EC43D2F8001241F0010104
:10056000C2F80012D2F81C122140C2F81C12017B02
:10057000002934D1D2F80C12DB002140C2F80C1251
:10058000C288418841EA024103F1804202F5C84233
:10059000C2F840120388818843EA0143C2F844321A
:1005A000C37A2149A3BBD1F804322340C1F80432F5
:1005B00003891D4A83BBD1F814321C40C1F8144290
:1005C000437B012B02BFD2F81C322B43C2F81C32F2
:1005D000D2F8003223F00103C2F8003230BD012905
:1005E000DED1D2F80C12DB002943C2F80C120188CC
:1005F000428803F1804342EA014203F5C843C3F84D
:1006000040228188C28842EA0142C3F84422C7E7F7
:10061000D1F804322B43C9E7012B02BFD2F81432C0
:100620002B43C2F81432CBE70064004000238371EF
:10063000C371037243728372C3728370C3700323E6
:100640000371022343710123038070470D4BD3F8DC
:10065000002242F00102C3F80022D3F8002222F463
:100660007C5222F00E02C3F80022D3F8002242EAA4
:100670000020C3F80002D3F8002222F00102C3F8E0
:100680000022704700640040036819B143F48033CE
:100690000360704723F48033FAE70368A9B143F09D
:1006A00080030360D0F8843143F48073C0F8843150
:1006B000D0F8943143F48073C0F89431D0F8A43169
:1006C00043F48073C0F8A431704723F080030360C3
:1006D000D0F8843123F48073C0F88431D0F8943199
:1006E00023F48073C0F89431D0F8A43123F48073DC
:1006F000E8E78368F0B55C012FD483681A0142D41F
:100700008368DB0041D404252846F0BD0A68D3F88D
:10071000807144EA42523A43C3F880218A7A3044D5
:1007200002F00F028A72D3F8844124F00F04C3F858
:100730008441D3F884412243C3F88421D1F80B20AB
:10074000C0F88821D1F80F20C0F88C21D3F880217F
:1007500042F00102C3F88021D6E700252E0183195B
:10076000D3F8802102F00102C3F880210A7A4C7A82
:10077000002ACBD04F68D3F880E142EAC702224377
:1007800042EA0E02C8E70125E8E70225E6E701296B
:1007900015D003D3022916D002207047836823F0B6
:1007A0007B4323F47F0323F47F4323F0FC030E4AAF
:1007B000934216D00FD8002BEED0002070478268ED
:1007C0000A4B1340F3E7836823F06F4323F47C0361
:1007D0001B0C1B04EBE7054A934202D0044A9342E8
:1007E000EBD10120704700BF0300000400030008A4
:1007F00000000310012908D002D3022909D0704754
:10080000836843F0800383607047836843F4004348
:10081000F9E7836843F40003F5E70B0130B5C4182A
:10082000D4F8B05105F004051572B5BBD4F8B05139
:100830006D0D1560D4F8B051034405F002055572F2
:10084000D4F8B45105F00F059572D4F8B441240AD8
:10085000D474D3F8B841D472D3F8B841240A1473CD
:10086000D3F8B841240C5473D3F8B841240E9473D0
:10087000D3F8BC41D473D3F8BC41240A1474D3F820
:10088000BC41240C5474D3F8BC311B0E937449B989
:10089000C36843F02003C36030BDD4F8B051ED0805
:1008A0005560C7E7036943F02003036130BD21B9F8
:1008B000C36843F02003C3607047036943F020031B
:1008C0000361704719B9C06800F00300704701293F
:1008D00001D10069F8E700207047B1B9036823F03F
:1008E000030343F0010303604FF48033426802F0D6
:1008F0000302012A01D0013BF8D1406800F0030057
:10090000012814BF002001207047012911D103687C
:1009100023F0030303604FF480334268920701D051
:10092000013BFAD1436813F0030F0CBF01200020F4
:100930007047022913D1036823F0030343F0020335
:1009400003604FF48033426802F00302022A01D0B0
:10095000013BF8D1406800F003000228D1E70020F5
:100960007047036823F0030343F002030360406809
:1009700000F00300831E584258417047036823F07B
:10098000020303604FF480334268920701D5013BB4
:10099000FAD1406880F00200C0F3400070478069DF
:1009A00000F0700070478069000E70478069C0F3E6
:1009B00007407047436912B119434161704723EA08
:1009C0000101FAE711F4700F07D08369C3F3130331
:1009D0000B4214BF012000207047CB0101D54368B2
:1009E000F4E70A0101D58368F0E78B014CBFC368C7
:1009F0000369EBE70A4B994202D1002383617047F8
:100A00008A01C1F3130301D5C36070474A0101D5C0
:100A1000036170470A014CBF83604360704700BFA9
:100A20007000F03043690B4009D0402946D012D8FD
:100A300004293BD005D8012929D0022930D0002033
:100A40007047102936D0202936D00829F7D1C06840
:100A5000C0F300107047B1F5006F3DD00CD8B1F570
:100A6000007F31D0B1F5806F32D0B1F5807FE6D113
:100A7000806900F001007047B1F5803F20D0B1F5EA
:100A8000003F1FD0B1F5004FD9D1406821E0806808
:100A900000F0013020F08070003018BF0120704756
:100AA000C06810F0030018BF01207047C068C0F391
:100AB000C00070470069F4E70069F8E70069C7E71C
:100AC0004068F4E74068C3E78069C0F340007047BE
:100AD0008069C0F380007047836913F0700F14BF02
:100AE000012000207047B1F5807F23D00CD8082961
:100AF00028D004D801291FD0042920D070472029EC
:100B000022D0402923D07047B1F5006F10D006D80D
:100B1000B1F5007F0ED0B1F5806F0BD07047B1F505
:100B2000803F16D0B1F5003F16D0B1F5004F12D17D
:100B30000023836104230DE0084B83607047082382
:100B4000C36070471023FBE708230361704710233D
:100B5000FBE70823436070471023FBE70101010016
:100B6000036823F001030360002303604360836094
:100B7000C3600361212343612A4B984203D13D2284
:100B800043F8082C7047284B984204D14FF4746204
:100B900043F8202C7047254B984204D14FF474122F
:100BA00043F8382C7047224B984204D14FF07462BE
:100BB00043F8502C70471F4B984203D11E4A43F80C
:100BC000642C70471D4B984203D11D4A43F87C2C7E
:100BD00070471C4B984203D11B4A43F8942C704732
:100BE0001A4B984204D14FF03D5243F8AC2C17E019
:100BF000174B9842C3D0174B9842C7D0164B984218
:100C0000CCD0164B9842D1D0154B9842D6D0154B2C
:100C10009842DAD0144B9842DED0144B9842E2D07E
:100C2000704700BF106002402860024040600240F0
:100C300058600240706002403D0000208860024021
:100C4000400F0020A060024000003D20B86002403C
:100C5000106402402864024040640240586402402C
:100C60007064024088640240A0640240B86402409C
:100C70000368134A10B51A40CC680B6823434C69CB
:100C800023438C692343CC6923430C6A23434C6A76
:100C900023438C6A23434C6B23438C6B23431343C2
:100CA00003604269CB6A0C6B22F0070223431343B3
:100CB00043610B6943604B6883608B68C36010BD00
:100CC0003F801CF00023036043608360C3600361C6
:100CD00043618361C361036243628362C3620363EE
:100CE000436383637047036819B143F001030360F2
:100CF000704723F00103FAE7036819B143F4004396
:100D00000360704723F40043FAE7036819B143F026
:100D100020030360704723F02003FAE74160704727
:100D2000406880B27047036822B143F40023036037
:100D30000161704723F40023F9E7036819B143F414
:100D400080230360704723F48023FAE70AB101612E
:100D50007047C16070470068C0F3C04070470068CA
:100D600000F001007047406900F0380070470A4BFE
:100D700010B50A4A0A4CA04294BF184610468B0090
:100D80004CBF4368036821F0F02121F08211194221
:100D900014BF0120002010BD00600240006402402A
:100DA0000F6402400B0612D5436952B143F0800331
:100DB0008029436104D0036801F01E0119430160DA
:100DC000704723F080038029436104D17047802954
:100DD000F6D0002AEFD1036801F01E0123EA0101D9
:100DE000EDE7114B10B5114A114CA04288BF1A46CD
:100DF00021F0F02323F0C31393B1006800EAD1205F
:100E000000F01E0388004CBF5068106821F0F021EC
:100E100021F08211084002D0181C18BF012010BD1B
:100E2000436903F08003EDE7006402400060024084
:100E30000F64024010B5084A084B094CA04294BF09
:100E40001846104611F0005F21F0F02121F08211C8
:100E500014BFC160816010BD0064024000600240A8
:100E60000F640240FFF7E6BF0022044B1A605A608D
:100E70009A60DA60024A5A61704700BF003C014044
:100E8000FFFF7F00827930B50168037942B3CC431C
:100E9000184A03F18043156803F59E332540156019
:100EA00055682C4054601C6821431960036894689D
:100EB000D9430C409460D4682140D1604179102915
:100EC00006D1916819439160D1680B43D36030BD5E
:100ED00001F1804202F59E3211680B43136030BD70
:100EE00003F1804303F59E331A6822EA0101196079
:100EF00030BD00BF003C014000230C2203600371A1
:100F0000427183717047024A136918431061704738
:100F1000003C0140034B5B69034214BF01200020E9
:100F2000704700BF003C0140014B5861704700BF53
:100F3000003C0140054B1A685B69034004D0024243
:100F400014BF01200020704718467047003C014044
:100F5000014B5861704700BF003C014008B5304B61
:100F6000984209D10121084600F062FA00210120CF
:100F7000BDE8084000F05CBA2A4B984206D1012136
:100F8000022000F055FA00210220F1E7264B98429A
:100F900006D10121042000F04BFA00210420E7E7EC
:100FA000224B984206D10121082000F041FA00218D
:100FB0000820DDE71E4B984206D10121102000F0E9
:100FC00037FA00211020D3E71A4B984206D10121AD
:100FD000202000F02DFA00212020C9E7164B98426E
:100FE00006D10121402000F023FA00214020BFE774
:100FF000124B984206D10121802000F019FA0021FD
:101000008020B5E70E4B984208D101214FF4807043
:1010100000F00EFA00214FF48070A9E708BD00BF70
:10102000000002400004024000080240000C0240A0
:10103000001002400014024000180240001C024050
:10104000002002402DE9F0430022012603240D6810
:1010500006FA02FC3CEA05033DD1570004FA07F307
:10106000DB43D0F800E00EEA030EC0F800E091F890
:1010700004E0D0F800900EFA07F80EF1FF3E48EABF
:101080000908BEF1010FC0F8008017D8D0F808E0B9
:1010900003EA0E0383604B79D0F808E0BB4043EAD3
:1010A0000E038360436823EA0C0343608B79D0F816
:1010B00004E093409BB243EA0E034360C36804FA22
:1010C00007FE23EA0E03C360CB79D0F80CE0BB40E7
:1010D00043EA0E03C3600132102AB9D1BDE8F083A0
:1010E0004FF6FF7303600023037143718371C37173
:1010F00070474FF4803382B00193019B0B430193FF
:10110000019BC361C161019BC361C3690193C36951
:10111000019302B070470369194214BF01200020F7
:101120007047006980B270474369194214BF0120BB
:1011300000207047406980B2704701837047418347
:1011400070470AB10183704741837047416170471E
:10115000436959404161704710B50F2401F00703FE
:10116000C90800EB8100016A9B009C4021EA040150
:101170000162016A9A400A43026210BD00210A4BD3
:101180001A6842F001021A6099601A6822F08472AB
:1011900022F480321A60054A5A601A6822F48022CA
:1011A0001A60D960704700BF003802401030002438
:1011B0000022024B1A701870704700BF02380240BC
:1011C000034A136823F0F80343EAC0001060704735
:1011D00000380240014B1860704700BF00004742D2
:1011E0000022064B01281A701A7002D0042802D07F
:1011F00070471870704705221A70704770380240A7
:10120000014B1860704700BF800E474210B5029C2A
:101210005B0840EA04600843013B40EA821040EA70
:101220000340014B586010BD00380240014B18606C
:10123000704700BF600047420907034B41EA801135
:10124000C3F88410704700BF00380240014B18609B
:10125000704700BF68004742014B1860704700BFED
:101260004C004742034A936823F0EC63194301435F
:101270009160704700380240034A936823F0784336
:10128000194301439160704700380240034A936854
:1012900023F0030318439060704700BF00380240FA
:1012A000024B986800F00C00704700BF0038024005
:1012B000034A936823F0F00318439060704700BF1F
:1012C00000380240034A936823F4E05318439060C7
:1012D000704700BF00380240034A936823F460431C
:1012E00043EAC00090607047003802401A4A10B5C7
:1012F00091681A4B01F00C01042901D0082917D07C
:10130000154A036093681649C3F30313CC5C036862
:10131000E34043609468C4F382240C5D23FA04F430
:1013200084609268C2F342328A5CD340C36010BDCD
:1013300054685168526801F03F01B3FBF1F3C2F306
:1013400088125343044A5268C2F3014201325200E8
:10135000B3FBF2F3D4E700BF003802400024F400EE
:10136000D000002000F44073B3F5407F084A08D154
:10137000916820F0704321F4F81123F440730B437B
:101380009360136FC0F30B0018431067704700BFE2
:1013900000380240014B1860704700BF3C0E4742C6
:1013A000014B1860704700BF400E4742014B186068
:1013B000704700BF5C014742044B1A6B11B11043E8
:1013C0001863704722EA0000FAE700BF00380240C5
:1013D000044B5A6B11B110435863704722EA000066
:1013E000FAE700BF00380240044B9A6B11B110437A
:1013F0009863704722EA0000FAE700BF0038024015
:10140000044B1A6C11B110431864704722EA0000B3
:10141000FAE700BF00380240044B5A6C11B1104388
:101420005864704722EA0000FAE700BF0038024023
:10143000044B1A6911B110431861704722EA000089
:10144000FAE700BF00380240044B5A6911B110435B
:101450005861704722EA0000FAE700BF00380240F6
:10146000044B9A6911B110439861704722EA000059
:10147000FAE700BF00380240044B1A6A11B110436A
:101480001862704722EA0000FAE700BF0038024005
:10149000044B5A6A11B110435862704722EA0000A7
:1014A000FAE700BF00380240044B1A6D11B1104337
:1014B0001865704722EA0000FAE700BF00380240D2
:1014C000044B5A6D11B110435865704722EA000071
:1014D000FAE700BF00380240044B9A6D11B1104387
:1014E0009865704722EA0000FAE700BF0038024022
:1014F000044B1A6E11B110431866704722EA0000BF
:10150000FAE700BF00380240044B5A6E11B1104395
:101510005866704722EA0000FAE700BF0038024030
:10152000044B1A7811B110431870704722EA00007A
:10153000FAE700BF0D3802404209012A074B07D1E4
:101540001B6800F01F0023FA00F000F00100704754
:10155000022A0CBF1B6F5B6FF3E700BF003802402D
:10156000002307B501933120FFF7E6FF019B01330C
:101570000193019BB3F5A06F01D00028F3D0312077
:10158000FFF7DAFF003018BF012003B05DF804FB5D
:10159000024A536F43F0807353677047003802402C
:1015A000034BDB68184214BF01200020704700BFC6
:1015B00000380240014B1870704700BF0E380240DF
:1015C00008B5154B98420BD101214FF48050FFF71D
:1015D0005FFFBDE8084000214FF48050FFF758BF7F
:1015E0000E4B98420BD101214FF48040FFF744FF8E
:1015F00000214FF48040BDE80840FFF73DBF084B95
:10160000984208D101214FF40040FFF735FF002137
:101610004FF40040EFE708BD0030014000380040C3
:10162000003C0040038810B503F441524C880B88FD
:1016300023438C882343CC8823430C8923434C8940
:1016400023438C892343CC89234313439BB20380D8
:10165000838B23F400631B041B0C83830B8A03829C
:1016600010BD838BF0B523F47B6323F00F031B04C1
:101670001B0C8383022303848B68848B022BA4B20C
:101680004ED0284E8A88002AB26814BF022701274C
:10169000120242BFB26822F40002B260D6F884207F
:1016A000D6F88450D6F804E0C2F388161E4A0EF02D
:1016B0003F0EB2FBFEF27243C5F30275B2FBF5F5C5
:1016C000CA88B2F5007F18BF7E014FF00A0214BF2E
:1016D000B5FBF6F52D0A6A43B2FBF3F30A22053394
:1016E0009BB2B3FBF2F303F001021202C3F34F0308
:1016F0009D1EADB2FE2D24BF002202231343CA88D3
:1017000013439BB24A8803840B8813438A8843F4AB
:10171000006313438A8913431C43A4B28483F0BD3E
:101720000022E5E7003802400024F4000023038093
:1017300043808380C380038143818381C3810723E6
:101740000382704700230222038043808380C3808A
:10175000826083817047038821B19BB243F04003CC
:101760000380704723F040031B041B0CF8E7838BB6
:1017700021B19BB243F480638383704723F4806379
:101780001B041B0CF8E7038823F400631B041B0CE9
:10179000038003889BB21943018070470388B1F529
:1017A000804F15BF23F480439BB21B0443F4804356
:1017B00018BF1B0C038070474FF6FF6399420388E4
:1017C0000BBF23F480739BB21B0443F4807308BFE8
:1017D0001B0C03807047838821B19BB243F0040344
:1017E0008380704723F004031B041B0CF8E78388F5
:1017F00021B19BB243F010038380704723F01003A4
:101800001B041B0CF8E7808980B270478181704708
:10181000038821B19BB243F400530380704723F443
:1018200000531B041B0CF8E703889BB243F480535E
:1018300003807047012914BF008B808A80B27047F3
:10184000008A80B2704783889BB212B119438180AD
:10185000704723EA0101FAE70B09012199408388C7
:1018600089B29BB212B119438180704723EA01010A
:10187000FAE70389194214BF012000207047C943C9
:1018800089B201817047012310B58488008901F075
:101890000F0280B203FA02F21040A4B205D0090987
:1018A0008B401C4214BF0120002010BD01F00F032B
:1018B00001219940C94389B20181704730B5048C38
:1018C00042EA031324F001042404240C0484048B4E
:1018D000058C24F0F3042404240C1C4325F00A0393
:1018E0001B041B0C41F00101A4B20B4304830384CD
:1018F00030BD30B5048C120224F010042404240CF2
:101900000484058B048C42EA033324F0A00225F4FE
:10191000407512042D05120C2D0D42EA01111D43D4
:1019200041F01001ADB289B20583018430BD08B524
:101930004D4B984209D101210846FFF7A9FD00212E
:101940000120BDE80840FFF7A3BDB0F1804F09D1E9
:1019500001210846FFF790FD00210120BDE8084065
:10196000FFF78ABD414B984206D101210220FFF7C3
:1019700083FD00210220F1E73D4B984206D1012171
:101980000420FFF779FD00210420E7E7394B984256
:1019900006D101210820FFF76FFD00210820DDE7B7
:1019A000354B984206D101211020FFF765FD00213B
:1019B0001020D3E7314B984206D101212020FFF7B8
:1019C0005BFD00212020C9E72D4B984206D1012163
:1019D0000220FFF75DFD00210220B2E7294B98426B
:1019E00008D101214FF48030FFF752FD00214FF460
:1019F0008030A6E7244B984208D101214FF40030F3
:101A0000FFF746FD00214FF400309AE71F4B984244
:101A100008D101214FF48020FFF73AFD00214FF457
:101A200080208EE71A4B984206D101214020FFF713
:101A300023FD0021402091E7164B984206D1012159
:101A40008020FFF719FD0021802087E7124B984284
:101A500008D101214FF48070FFF70EFD00214FF4F3
:101A600080707BE708BD00BF00000140000400401B
:101A700000080040000C004000100040001400402E
:101A80000004014000400140004401400048014082
:101A900000180040001C0040002000401C4A038841
:101AA00090429BB212D002F5806290420ED0B0F10B
:101AB000804F0BD0A2F58032904207D002F58062B1
:101AC000904203D002F58062904203D14A8823F00D
:101AD000700313430F4A904208D002F5806290428F
:101AE0001FBF23F440730A899BB2134303804B68E2
:101AF000C3620B880385064B984203D003F58063CD
:101B0000984201D18B7A038601238382704700BFFC
:101B100000000140001000404FF0FF3343600023FD
:101B200003800381438083727047018582827047FE
:101B3000038823F070031B041B0C194301807047BA
:101B400041627047C1627047406A7047008D80B241
:101B50007047038821B19BB243F0020303807047B2
:101B600023F002031B041B0CF8E7038821B19BB28E
:101B700043F004030380704723F004031B041B0C91
:101B8000F8E7038821B19BB243F0800303807047DC
:101B900023F080031B041B0CF8E7038823F00803E1
:101BA0001B041B0C038003889BB219430180704700
:101BB000038823F440731B041B0C038003889BB22F
:101BC000194301807047038821B19BB243F00103A0
:101BD0000380704723F001031B041B0CF8E7038C00
:101BE00070B523F001031B041B0C0384038C828853
:101BF000048B0D8824F073042404240C2C4323F05C
:101C000002038D894E881B0435431B0C2B430F4D5B
:101C100092B2A8429BB203D005F58065A8420ED1CE
:101C2000CD8923F008032B438D8823F004032B4335
:101C30004E8A0D8A22F4407235432A4392B2828042
:101C40008A6804834263038470BD00BF00000140C2
:101C5000038C70B523F010031B041B0C0384038C4E
:101C60008488028B0D8822F4E6421204120C42EAA8
:101C7000052223F020038D894E881B0435431B0C5D
:101C800043EA0513114DA4B2A84292B29BB203D00D
:101C900005F58065A84213D1CD8923F0800343EA7E
:101CA00005134FF6BF751D408B884E8A45EA031316
:101CB0000D8A24F44064354344EA85049BB2A4B2FF
:101CC000848002838A688263038470BD00000140BF
:101CD000038C70B523F480731B041B0C0384038CEA
:101CE0008288848B0D8824F073042404240C2C43F4
:101CF00023F400738D894E881B0435431B0C43EA83
:101D00000523114D92B2A8429BB203D005F5806520
:101D1000A84213D1CD8923F4006343EA05234FF68B
:101D2000FF351D408B884E8A45EA03230D8A22F435
:101D30004052354342EA05129BB292B282808A68D1
:101D40008483C263038470BD00000140038C70B5BE
:101D500023F480531B041B0C0384038C8488828B24
:101D60000D8822F4E6421204120C42EA052223F402
:101D700000538D894E881B0435431B0C43EA053301
:101D80000A4DA4B2A84292B29BB203D005F5806579
:101D9000A84205D10D8A24F4804444EA8514A4B2F3
:101DA000848082838A680264038470BD00000140DD
:101DB000002303804380838083608381C381038207
:101DC0004382704730B50125048C8D40A4B224EACB
:101DD000050400F11803048421F0080050B94908F3
:101DE000C85820F070000004000CC850C8580243C6
:101DF000CA5030BD0439C1F34E01C858120220F454
:101E0000E0400004000CC850C85892B2EFE74163AC
:101E1000704781637047C163704701647047038BEB
:101E200023F070031B041B0C194301837047038BC1
:101E300023F4E0431B041B0C43EA012189B2018314
:101E40007047838B23F070031B041B0C19438183A1
:101E50007047838B23F4E0431B041B0C43EA0121EE
:101E600089B281837047038B23F008031B041B0C8A
:101E7000194301837047038B23F400631B041B0C7D
:101E800043EA012189B201837047838B23F0080361
:101E90001B041B0C194381837047838B23F400635D
:101EA0001B041B0C43EA012189B281837047038B19
:101EB00023F004031B041B0C194301837047038B9D
:101EC00023F480631B041B0C43EA012189B20183C4
:101ED0007047838B23F004031B041B0C194381837D
:101EE0007047838B23F480631B041B0C43EA01219E
:101EF00089B281837047038B23F080031B041B0C82
:101F0000194301837047038BC3F30E0343EA012196
:101F100089B201837047838B23F080031B041B0C61
:101F2000194381837047838BC3F30E0343EA012176
:101F300089B281837047038C23F002031B041B0CBE
:101F4000194301847047038C23F008031B041B0C06
:101F5000194301847047038C23F020031B041B0CDE
:101F600043EA011189B201847047038C23F0800396
:101F70001B041B0C43EA011189B201847047038CD6
:101F800023F400731B041B0C43EA012189B2018472
:101F90007047038C23F400631B041B0C43EA0121EC
:101FA00089B201847047038C23F400531B041B0C7B
:101FB00043EA013189B20184704710B50124038CD2
:101FC0008C409BB223EA04030384038C02FA01F1E0
:101FD000194389B2018410BD10B50424038C8C40D0
:101FE0009BB223EA04030384038C02FA01F1194330
:101FF00089B2018410BD00230122038043808280C6
:10200000C38003817047406B7047806B7047C06B23
:102010007047006C7047038B23F00C031B041B0CF0
:102020000383038B9BB2194301837047038B23F413
:1020300040631B041B0C0383038B9BB243EA012107
:1020400089B201837047F8B50C464988A2880029F7
:10205000B4F800E00CBF02260026012A0CBF0227BC
:1020600001272389BEF1000F0ED1FFF727FCE1887D
:10207000FFF7D1FF314623893A46FFF73AFCE18862
:10208000BDE8F840FFF7D2BFFFF733FCE188FFF768
:10209000CDFF314623893A46FFF710FCE188BDE8C1
:1020A000F840FFF7B8BF838B23F00C031B041B0C15
:1020B0008383838B9BB2194381837047838B23F483
:1020C00040631B041B0C8383838B9BB243EA012177
:1020D00089B281837047F8B50E880D460B898A88CE
:1020E000498836B9FFF7EAFBE988BDE8F840FFF711
:1020F00092BF042E06D1FFF7FCFBE988BDE8F8404B
:10210000FFF794BF082EEF88058C1CD125F480754D
:102110002D042D0C0584868B058CB6B226F0F306B3
:102120003243ADB242EA031325F4206242F48072D6
:1021300042EA01229BB292B283833946BDE8F8405D
:102140000284FFF7B0BF1B0343EA022345F6FF7288
:1021500025F480552D042D0C0584868B058C26F4E2
:1021600040762A403605360D42F48052334342EA27
:1021700001329BB292B283833946BDE8F8400284B3
:10218000FFF79CBF4A880B8813438A881343CA8889
:1021900013430A8913434A8913438A8913439BB221
:1021A000A0F8443070470023038043808380C380BD
:1021B0000381438183817047B0F8443039B16FEABD
:1021C00043436FEA53439BB2A0F844307047C3F3D4
:1021D0000E03F9E7838821B19BB243F004038380A7
:1021E000704723F004031B041B0CF8E7838821B11C
:1021F0009BB243F001038380704723F001031B046B
:102200001B0CF8E781827047038A194214BF012032
:1022100000207047C94389B201827047038A8289CE
:1022200011EA030092B203D0114214BF0120002032
:102230007047C94389B2018270470A43A0F8482019
:10224000704783899BB212B119438181704723EA99
:102250000101FAE7FFF7F5BF838821B19BB243F094
:1022600008038380704723F008031B041B0CF8E766
:10227000038923F007031B041B0C038170470389A8
:1022800023F070031B041B0C1943018103899BB2CB
:1022900043F007030381704738B50D46602D1146A2
:1022A00004464FF001020ED1FFF723FB218921F0F4
:1022B00070010904090C2943218123899BB243F051
:1022C0000703238138BDFFF7F9FAEFE7038923F00D
:1022D00070031B041B0C194301817047838823F092
:1022E00070031B041B0C838083889BB2194381807D
:1022F0007047038923F007031B041B0C0381038928
:102300009BB2194301817047038923F080031B04AA
:102310001B0C038103899BB219430181704710B5DF
:1023200004890A43E4B242EA03231C43A4B20481B1
:1023300010BD10B5FFF7F3FF038923F077031B04EB
:102340001B0C43F07703038110BD10B5FFF7E7FFC7
:1023500003899BB243F48043038110BD70B50689A5
:10236000048B058C24F4407424F0030425F022052A
:1023700026F0070624042D043604240C2D0C42EA12
:102380000313360C44F480741D43314344F00104BC
:10239000ADB201810483058470BD838821B19BB2F5
:1023A00043F080038380704723F080031B041B0CE1
:1023B000F8E7A0F85010704708B5254B984209D1AE
:1023C00001211020FFF764F800211020BDE808402B
:1023D000FFF75EB81F4B98420BD101214FF400303C
:1023E000FFF74AF800214FF40030BDE80840FFF73E
:1023F00043B8194B984208D101214FF48020FFF7D0
:102400003BF800214FF48020EFE7144B984208D1AD
:1024100001214FF40020FFF72FF800214FF4002096
:10242000E3E70F4B984208D101214FF48010FFF7EA
:1024300023F800214FF48010D7E70A4B984206D1C9
:1024400001212020FFF724F800212020BEE708BD4D
:10245000001001400044004000480040004C004093
:10246000005000400014014030B50D460446028A79
:10247000EB8892B222F440521A43898902828389FE
:10248000288923F4B052AB8822F00C0203436889F8
:1024900012040343120C9BB21343A381A38A85B099
:1024A0009BB223F440730B43A3826846FEF71EFFE2
:1024B000194B9C4203D003F580639C4221D10399C0
:1024C0001922A3894A4313F4004F2B684FF0640587
:1024D00014BF5B009B00B2FBF3F1B1FBF5F3A289E3
:1024E0001801120405FB13130DD5DA003232B2FBCA
:1024F000F5F202F0070242EA00039BB2238105B025
:1025000030BD0299DCE71B013233B3FBF5F303F076
:102510000F030343F1E700BF001001404FF41653CF
:102520000C220360002342818380C3800381838166
:102530007047038A10B59BB24C8823F470620B88F5
:1025400023438C88C98823430B439BB213430382E4
:1025500010BD0023038043808380C380704783893C
:1025600021B19BB243F400538381704723F400539D
:102570001B041B0CF8E7038B03F47F430383038BDB
:102580009BB2194301837047838931B16FEA43439A
:102590006FEA53439BB283817047C3F30E03FAE79C
:1025A000838A21B19BB243F400638382704723F492
:1025B00000631B041B0CF8E7C1F30801818070471E
:1025C0008088C0F308007047038A23F00F031B04C0
:1025D0001B0C0382038A9BB21943018270478389D3
:1025E00021B19BB243F002038381704723F00203C1
:1025F0001B041B0CF8E7838923F400631B041B0CEA
:10260000838183899BB2194381817047038A23F0B8
:1026100020031B041B0C0382038A9BB21943018213
:102620007047038A21B19BB243F480430382704711
:1026300023F480431B041B0CF8E783899BB243F00F
:10264000010383817047838A21B19BB243F0080361
:102650008382704723F008031B041B0CF8E7038BED
:10266000DBB20383038B9BB243EA012101837047F2
:10267000838A21B19BB243F020038382704723F009
:1026800020031B041B0CF8E7838A21B19BB243F0A3
:1026900010038382704723F010031B041B0CF8E720
:1026A000838A23F004031B041B0C8382838A9BB25E
:1026B000194381827047838A21B19BB243F00203A0
:1026C0008382704723F002031B041B0CF8E7838A04
:1026D0009BB212B119438182704723EA0101FAE7E4
:1026E00001F01F0310B5C1F342140121012C01FABE
:1026F00003F105D10C3003683AB11943016010BDF4
:10270000022C0CBF10301430F5E723EA0101F5E785
:102710000388194214BF012000207047C94389B2C1
:10272000018070470123C1F3421210B5012A01F064
:102730001F0403FA04F30ED1828992B21340028877
:1027400092B26BB10123090A03FA01F10A4214BFE4
:102750001846002010BD022A0CBF028A828AECE7CC
:10276000184610BD0B0A01219940C94389B2018066
:10277000704700BF40F0BF60024B40F40030D860AB
:10278000704700BF00ED00E010B5C3780278FBB1E0
:10279000154BD9684378C943C1F30221C1F1040440
:1027A000E4B2A3400F24807844FA01F10140DBB287
:1027B0000B430E491B018818DBB280F8003301235C
:1027C000500902F01F0203FA02F241F8202010BD66
:1027D0000121530902F01F0201FA02F203492033DA
:1027E00041F8232010BD00BF00ED00E000E100E053
:1027F00021F0604121F07F01014B01439960704756
:1028000000ED00E0044B1A6911B1104318617047E4
:1028100022EA0000FAE700BF00ED00E0044B0428C4
:102820001A680CBF42F0040222F004021A607047DA
:1028300010E000E0D0F8E83510B51B690446984771
:10284000032384F81231002010BD08B590F812312E
:1028500080F81331042380F81231D0F8E835DB68B2
:102860009847002008BD08B5D0F8E435DB6903B10E
:102870009847002008BD08B5D0F8E4351B6A984792
:10288000002008BD08B5D0F8E4355B6A9847002001
:1028900008BDD0F8E83510B55B69044698470123B8
:1028A00084F81531002010BD10B50446D0F8E83585
:1028B0009B699847D4F8E43500215B682046984727
:1028C000002084F8150110BD002310B504461946F8
:1028D000402201F02BF9402280210023204601F004
:1028E00025F9012384F81231D4F8E835A0785B6823
:1028F0009847002010BD13B56946044600F010FC4F
:102900009DF8001001F01F03012B0FD007D3022BFD
:1029100011D001F08001204601F086F903E06946FC
:10292000204600F06BFA002002B010BD6946204638
:1029300000F080FBF7E76946204600F093FBF2E7E2
:1029400038B50446002948D190F81131022B16D130
:10295000D0F83821D0F824319A421DD9C178D21A42
:10296000012908BFD0F82811C0F8382104BF5B182E
:10297000C0F8283192B2D0F8281100F0EDF994F89F
:102980001631012B06D11A4A236912685A600023B6
:1029900084F81631002038BDD0F83C21B2FBF3F5A5
:1029A00003FB15255DB9934209D8D0F840319A420E
:1029B00005D22A4600F0D0F9C4F84051DFE7D4F838
:1029C000E435DB682BB194F81221032A01D12046AB
:1029D0009847204600F0EFF9D1E7D0F8E4355B697D
:1029E000002BD7D090F81221032AD3D19847D1E7F2
:1029F0005466002010B5044661BB90F81131032BDA
:102A000019D1D0F89033D0F87C23934215D9C178EE
:102A10009B1A012908BFD0F88013C0F8903304BF77
:102A20008918C0F880139A4228BF1A46D0F880133C
:102A300092B200F0A9F9002010BDD0F8E4351B696E
:102A400023B190F81221032A00D19847204600F0C4
:102A5000A3F9F0E7D0F8E4359B69002BEBD090F8B0
:102A60001221032AE7D19847E5E72DE9F041044612
:102A7000164698460D46069FF7F769FB20462946FD
:102A8000C4F8E485C4F8E875C4F8EC6501F000F812
:102A9000D4F8E8351B6898472046BDE8F041F7F7C1
:102AA000A9BB0020704710B50446D0F8E4351B6878
:102AB0009847D4F8E8359B689847002010BD08B5C2
:102AC000D0F8E4355B689847002008BD10B5074C86
:102AD0002068FF2807D0064B064A9B681268064903
:102AE0009847FF232360002010BD00BF1001002085
:102AF000A800002020560020DB6600204323014868
:102B00000B8070471401002038B51B4B5A681946DA
:102B1000052A02F1010402D05C60002038BD0023C8
:102B20000A7A4B60012AF8D0CA68B2F5006F08BF74
:102B3000CB60CC680B699C4202D100230B72ECE79E
:102B40008CBFC4F500631B1B4B614D69A2B2402DC5
:102B50000CD940234034403DCC604D6101240C72BF
:102B600006490A44812101F03FF8D6E72C44CC60A5
:102B70000024ABB24C61F1E720560020E366002050
:102B800038B52823044603FB0101074D074BB1F874
:102B90008C131B692846984740232A46012120466A
:102BA00000F0FCFF002038BD9B660020A80000203C
:102BB000F8B50A78064612F060040D4628D0202C9D
:102BC00022D1CC884B78C4B112060BD5214A2249B8
:102BD000976818462246B847EA881F49304600F0F1
:102BE000ABF807E01D4A1C4913601D4B22461C60D0
:102BF00000F0BAF800242046F8BD164A2146956830
:102C000018462246A847F6E700F0ACFA0224F2E79D
:102C10004B780A2B10D00B2B13D0062BEBD14B8803
:102C20001B0A212B05D1CA880E493A2A28BF3A220D
:102C3000D4E70D493A22D1E701220C4900F07CF893
:102C4000D9E78B7813B9064A9361D3E700F08AFA83
:102C5000D1E700BFA8000020DB66002010010020A3
:102C600020560020260100201D010020385600209B
:102C700010B50446812100F07BFF0121204600F0C1
:102C800077FF8221204600F073FF024B5B68984774
:102C9000002010BDA800002038B5044602234022C1
:102CA000812100F043FF022340220121204600F051
:102CB0003DFF822103230822204600F037FF002534
:102CC0000222074B1A715D71064B1B68984740231F
:102CD000054A0121204600F061FF284638BD00BFAB
:102CE00044000020A80000209B66002038B5104C4E
:102CF000237A012B02D1616911B92172002038BDFC
:102D000040290CD9E36840399AB24033E36040234C
:102D1000616108490A44812100F066FFEEE7E56839
:102D20008BB22944E1600021AAB26161F1E700BFE2
:102D300020560020E366002010B504461346C4F870
:102D40003C21C4F83821022280F811210A460021D2
:102D500000F04AFF002010BD08B513460A460021C6
:102D600000F042FF002008BD10B504461346C4F829
:102D70009423C4F89023032280F811210A460021ED
:102D800000F00CFF002010BD08B513460A460021D4
:102D900000F004FF002008BD042310B580F81131B5
:102DA000002304461A46194600F01EFF204600F094
:102DB0009BFD002010BD052310B580F811310023C4
:102DC00004461A46194600F0E9FE204600F08CFD44
:102DD000002010BD282303FB0101B1F88C037047CC
:102DE00010B50446802100F01FFF2046002100F0AE
:102DF0001BFF2046BDE8104000F076BD37B54B788C
:102E000004460D46092B73D8DFE813F0C200000119
:102E10007200D200720067000A007200B4008700DE
:102E20004B881A0A013A062A62D8DFE802F0042623
:102E3000326161616100D0F8EC350DF106011B686B
:102E400080789847EB88402B03D094F81231012BFF
:102E500002D10823ADF80630BDF80620002A57D06D
:102E6000EB88002B54D09A4228BF1A460146ADF891
:102E700006202046FFF760FF4AE0D0F8E4350DF168
:102E800006019B6A8078984702234370C4F8F005D6
:102E9000E2E7DBB2052B2BD8DFE803F0030B0F13BF
:102EA000171BD0F8EC355B680DF10601A078984748
:102EB000D2E7D0F8EC359B68F6E7D0F8EC35DB6864
:102EC000F2E7D0F8EC351B69EEE7D0F8EC355B693A
:102ED000EAE7D0F8EC359B69E6E78B8843B9CB8805
:102EE00033B990F812318D78032B05F07F0503D1AB
:102EF0002046FFF775FF0BE080F81451294600F0DB
:102F0000D1FE2046FFF748FF2DB1022384F812318D
:102F1000002003B030BD0123F8E78978414D012935
:102F20002970E5D890F81231022B0DD0032BDFD198
:102F3000B1B9022380F8101180F81231FFF7BFFDFC
:102F40002046FFF729FFE3E70029F9D001210323F9
:102F500080F8101180F812312046FFF7A4FDEFE74A
:102F600090F810110129EBD0FFF7A9FD297884F81A
:102F70001011F1E7CA88012ABAD190F81231022B58
:102F800004D0032BB4D100F5887172E7264970E7AD
:102F900090F81231023B012BAAD80122214B9A60F2
:102FA000D0F818210AB103229A6002221F4960E773
:102FB0004B88012B08D1C4F81831D4F8E4352946E0
:102FC0009B6820469847BBE7022BA1D18B8813F062
:102FD000FF0F9DD102691B0A013B5268042B07D8E1
:102FE000DFE803F0030C0E101200012363F3061256
:102FF0000F4B1A60012384F81631A1E70223F5E78D
:103000000323F3E70423F1E70523EFE790F81231F8
:10301000023B012B3FF66CAF4B88012B7FF478AF5E
:103020000023C8E73C5600204056002044560020AC
:103030005466002038B590F812310446032B0D4633
:103040000DD10B79012B0AD8D0F8E4359B6898474D
:10305000EB8813B92046FFF79FFE002038BDFFF72D
:10306000BFFEFAE738B50D466A788B88012A044618
:10307000D9B21CD029D3032A17D190F81231022BD0
:103080003ED0032B02D0FFF7ABFE0EE06B881BB9DE
:103090004B0601D000F0C8FDD4F8E43529469B6802
:1030A000204698472046FFF777FE002038BD90F86D
:1030B0001231022B24D0032BE5D16B88002BF4D1E5
:1030C0004A06EFD000F0CAFDE6E790F81221022A86
:1030D00016D0032AD7D113F0800F4FF028020E4BE1
:1030E00015D001F07F0102FB010191F81E2162B1B0
:1030F0000122DA60094902222046FFF71DFED4E7CB
:103100004B06D2D000F090FDCFE70022F1E702FBA2
:10311000010191F87623EAE73C560020485600204A
:1031200090F8CC350B7090F8CD354B7090F8CF25DA
:1031300090F8CE3503EB02234B8090F8D12590F820
:10314000D03503EB02238B8090F8D32590F8D2354D
:1031500003EB02239BB2CB80C0F84031012380F8FF
:103160001131704710B50446802100F05DFD204606
:10317000002100F059FD2046BDE8104000F0B4BB2E
:1031800030B588B105462B1A15F8014BDBB2002C7F
:10319000F9D15B00023313800B7003234B700223C1
:1031A000013810F8015F05B930BD5A1CCD54D2B2B8
:1031B0000233DBB28C54F4E7002337B50546104CDC
:1031C00001930320F7F728F82B68013C1A69019254
:1031D00013D0019A002AF4DA019A42F00102019216
:1031E000019A1A61064A1969013A019102D00199BE
:1031F000C907F8D40320F7F70FF8002003B030BD5B
:10320000410D030010B5C47844B900EB820022469A
:103210000333D0F8D0009B10934201D1002010BDA1
:1032200051F8224001320460F6E7D0F8D030002097
:1032300010B503329210904202D101EB800010BD14
:103240001C6841F820400130F5E7012230B5002329
:10325000827040220129C37082803CD10823037010
:10326000042343704FF4A073C380022303724FF012
:10327000A043C17203F5006202614278C36003EBB0
:10328000421203F5106100F1180402F51062914238
:103290002DD1044603F58062426103F58862C0F8CF
:1032A000CC2014F8902B03F5A06103EB421505F533
:1032B000A065A94222D103EB023203F5805100F14F
:1032C000D00402F5805291421CD103F56063C0F82E
:1032D0000C31002030BD0029CCD10C230370062313
:1032E00043704FF4A063C172C380094BC2E744F836
:1032F000041B01F50075A5632031C8E744F8041BE1
:103300002031D6E744F8041B01F58051DBE700BF0C
:103310000000044038B5037A0546012B4FF0000445
:1033200050F80C2F2AD1936B697A64F3104309B1DA
:1033300043F480139363D3686FF386136FF396534C
:103340006FF351436FF3D343D360FFF735FFEB784F
:10335000012B06D1052363F34404EB6844F02004F9
:103360009C60EB78012B07D10522EB689C6862F327
:10337000440444F020049C60002038BDD36843F02E
:103380004003D360FFF718FF6B7AEA68002B0CBF8D
:103390004FF450234FF4E81314209363F6F746FFDD
:1033A000DFE7C2680020936843F001039360704731
:1033B000C2680020936823F00103936070470023E4
:1033C00007B50193019B43F020030193019B61F337
:1033D0008A130193019BC2681361074B1169013B7A
:1033E000019102D001998906F8D40320F6F714FF61
:1033F000002003B05DF804FB410D0300002307B576
:103400000193019B43F010030193019BC268136178
:10341000074B1169013B019102D00199C906F8D40B
:103420000320F6F7F9FE002003B05DF804FB00BFAF
:10343000410D0300C26808B5D36801296FF35D73BD
:103440006FF39E7307D143F00053D3603220F6F739
:10345000EDFE002008BD0029F7D143F08043F4E7DA
:10346000C368586900F001007047C3685869C043D9
:1034700000F001007047C368586900F00100704710
:10348000C36858699B6918407047C368586870479B
:103490000269136861F301031360704710B50023DC
:1034A0006FF080414FF0FF34C26893615161546006
:1034B000516109499161C1780020994208BF1023E8
:1034C00043F0804343F47013916943F4605343F035
:1034D0000C030B43936110BD00080080F8B5002673
:1034E000D0F80C3102691E601368044666F3CC23E1
:1034F0001360C37A3546012B374622D10321FFF7EB
:10350000C7FF2021C368A020802261F31F4660F31B
:103510000F055A6262F31F4562F30F064FF4907273
:103520009E62C3F8045162F30F054FF4A07261F379
:103530001F45C3F8085162F30F0567F31F45C3F831
:103540000C5110212046FFF73AFF2046FFF756FFA7
:1035500000234FF0FF311F464FF0FF0E226904F1A8
:103560001805136153619161D36166782169B34293
:1035700018D30023FF271E4604F1540562789342B6
:103580001ED30B69204643F480730B61E378012B53
:1035900001BF4022114B62F359430B63FFF77EFFDB
:1035A0000020F8BD55F8042B013310680028ACBF8B
:1035B00000204FF0904010601761C2F808E0D6E795
:1035C00055F8042B013310680028ACBF00204FF0E1
:1035D0009040106016619760D0E700BF03010100C2
:1035E00003699B68C3F34103022B04D001D8012B6C
:1035F00003D1022070470120704703207047036900
:10360000806999680268C1F3410102290ABF032158
:103610006FF30A0261F30A0202605A68002042F462
:1036200080725A60704730B54C780022012C0B78BC
:103630001DD100EB8305AD6904FA03F363F30F02B8
:103640002B681C040DD48C6864F30A03CC78C988F9
:1036500064F3934361F3995343F0805343F400437D
:103660002B6003690020D9690A43DA6130BD00EBA1
:103670008304656D012404FA03F363F31F42DFE75B
:1036800030B500254A782C46012A0B7810D100EB82
:103690008301896902FA03F363F30F0402696FF38C
:1036A000CF350D60D369002023EA0403D36130BD18
:1036B00000EB8302516D012202FA03F363F31F440E
:1036C000ECE7F8B54F780A78012F4B6942D100EB4F
:1036D0008204A6693468356963F31205EBB967F3B0
:1036E000DC453561C578012D26D10D697561CD7830
:1036F000012D07D10769BF68FF0554BF44F000548E
:1037000044F0805444F00444012D346003D19BB252
:10371000C968FFF777FD0020F8BDD1F808E003EB9A
:103720000E07013FB7FBFEF767F3DC45CF78012FAB
:1037300008BF67F35E75D4E7CD78012DD7D0002B95
:10374000D5D0012507699540D7F834E045EA0E0544
:103750007D63CCE700EB8202566D8A683468356978
:10376000ABB9012362F3120563F3DC453561C3781D
:10377000012B04BF0B697361CB78012B03D14B790B
:103780008BB144F0005444F004443460C3E7134464
:10379000013BB3FBF2F363F3DC45C3F3090353438B
:1037A00063F31205E2E744F08054ECE7F7B54F7895
:1037B0004E69012F3AD185692C682B690093DAB2E2
:1037C000C3F3074316BB66F306028DF8002067F3C8
:1037D000C4038DF80230009B2B61C278012A05D109
:1037E0000B780E6900EB83039B695E6144F004442F
:1037F0002C6042B94B6933B1012302690978506BDF
:103800008B4003435363002003B0F0BD8F68BE427A
:103810008CBF67F3060266F306028DF800204FF0B6
:10382000010288BF4F6162F3C403D2E70B788F684F
:1038300000EB83035D6D2C682B690093DAB2C3F350
:1038400007439EB967F306028DF80020012262F358
:10385000C4038DF80230009B44F004442B61C3780C
:10386000012B04BF0B696B612C60CCE74F61E9E76A
:103870004B78012B0B7800EB83000AD18269136827
:10388000002B01DA43F0804343F40013136000205F
:103890007047426D1368F7E74B78012B0B78C978B6
:1038A00000EB83000CBF8269426D02391368012965
:1038B0006FF3555398BF43F0805313600020704757
:1038C00003699869DB691840000C704700EB8101BF
:1038D0004B6D9A680369586910407047036998698D
:1038E000DB69184080B27047002382B00093C02388
:1038F00001228DF803304FF0000362F3C4038DF80A
:10390000023018238DF80030009A436D1A61C27896
:10391000012A06D100F2CC5058611A684FF080227B
:103920001A6002B07047D0F8183110B50446D3B110
:1039300002699368DB0716D5837A43B1D0F80C315E
:10394000D0F80C116FF341036FF300030B60536861
:10395000052043F001035360F6F768FC22695368C1
:1039600023F00103536010BD837A63B103699B6840
:10397000DB0708D5D0F80C31D0F80C216FF34103E8
:103980006FF300031360704738B50123044680F8D5
:103990001231FF210023407804F11802834210D332
:1039A0000022236920461A615A61DA614FF0FF3222
:1039B0009A61FFF723FD2046BDE838401021FFF74C
:1039C000FEBC52F8045B0133A960956BA960E5E782
:1039D0004B78012B0B7800EB83000BD183691B68BC
:1039E000C3F30743990613D413F0020F14BF20202A
:1039F00030207047436D1B68C3F307439A0609D410
:103A000013F0020F14BF4FF400504FF440507047B2
:103A1000102070474FF48050704770B44B780646C2
:103A2000012B0B780D4600EB830316D19C69102AFD
:103A3000236802D170BCFFF71BBF202A02D143F0DC
:103A4000006311E0302A1DD19A0216D500232946C1
:103A50006B71304670BCFFF71FBF5C6DB2F5805FC5
:103A6000236804D143F40013236070BC7047B2F59F
:103A7000005FE4D0B2F5405FE5E743F0044343F470
:103A80000043F1E7002AEFD162F3CF33ECE700BF48
:103A900070B50446FFF7D9FB0023012118464026E4
:103AA000657884F8121184F8143104F58E72AB42F3
:103AB00002F128021AD300224020114604F55D735A
:103AC000AA4203F1280321D32046FFF771FC2046C8
:103AD000FFF720FC00212046FFF7ACFC2046FFF753
:103AE000FDFC2046BDE87040FFF75BBC02F8283CB7
:103AF00022F8223C02F8271C02F8250C42F8206C20
:103B000042F81C0C42F8140C0133D0E703F8282CBF
:103B100023F8222C03F8271C03F8251C43F8200C5B
:103B200043F81C1C43F8141C0132C9E770B5282562
:103B30004EB201F07F04002EB5BF05FB040105FB6A
:103B4000010101F58E7101F55D71E4B2002EB8BF7F
:103B5000CC80022BCB7008BF00234FEAD6750C70C7
:103B60004D708A6008BF0B71FFF75DFD002070BDCE
:103B700028224BB2002B10B501F07F04B5BF02FB29
:103B8000040102FB010101F58E7101F55D71DB0F8E
:103B90000C704B70FFF774FD002010BD70B5282627
:103BA00001F07F0506FB05F404F55D710444C4F8DB
:103BB0008833002384F87453C4F88023C4F88C330A
:103BC00084F87533C37806FB0505012B08BFC4F8DC
:103BD000842395F8743301441BB9FFF7E7FD0020F7
:103BE00070BDFFF76EFDFAE770B52825044601F0B9
:103BF0007F0675432C4405F58E71C4F828210125F4
:103C0000C4F82C210022014484F81D5184F81C6161
:103C1000C4F83421C4F830311EB9FFF7C7FD0020C5
:103C200070BDFFF74EFDFAE728224BB2002B10B50E
:103C300001F07F04B4BF02FB040102FB01014FF05D
:103C40000102B4BF01F58E7101F55D71DB0F8A7061
:103C50000C704B70FFF70CFE002010BD282238B509
:103C600000244BB2002B01F07F05B5BF02FB05011C
:103C700002FB010101F58E7101F55D71DB0F8C70A6
:103C80000D704B70FFF708FE204638BD08B50B06D7
:103C900005D501F07F01FFF792FB002008BDFFF77B
:103CA000ADFBFAE70023026961F30A1311680B43C5
:103CB000136070470269032053686FF34103536038
:103CC000F6F7B4BA02690320536843F00203536065
:103CD000F6F7ACBA282311F0800F1BBF01F07F016B
:103CE00003FB010103FB010101F58E7108BF01F522
:103CF0005D71FFF76DBE282311F0800F1BBF01F02F
:103D00007F0103FB010103FB010101F58E7108BF77
:103D100001F55D71FFF781BE2DE9F04F85B00446D6
:103D2000FFF7A3FB18B9002005B0BDE8F08F2046CF
:103D3000FFF7A6FB05460028F5D0C0F3074A1AF0A6
:103D400008000ED02046FFF7BBFD4FF0000881466B
:103D5000DFF8B8B204F15407B9F1000F40F00E815A
:103D600001201AF0040F0DD02046FFF7B7FD2646BC
:103D700082464FF0000904F11807BAF1000F40F035
:103D800049810120EEB2B70742BF0222E3685A61BF
:103D9000002D19DAA37A43B1D4F80C31D4F80C21F0
:103DA0006FF341036FF300031360226920465368E9
:103DB00023F001035360954B1B689B6998474FF0B4
:103DC00000420120E3685A61C5F3072739072DD562
:103DD00000238DF80F3094F8123120468DF80F3003
:103DE0008A4B1B685B6998474FF400612369E2685E
:103DF0009B685161A27AC2B1DA0716D594F81531E1
:103E0000012B12D19DF80F30032B0ED1D4F80C31B9
:103E10001A6842F001021A601A6842F003021A603E
:103E20007B4A136943F0060313610120330708D569
:103E3000764B20461B68DB68984708220120E36820
:103E40005A61F10615D5E3689A6922F010029A6169
:103E50001E6AC6F34343022B06F00F0900F0798176
:103E6000062B00F092810120E268936943F0100371
:103E70009361FA0631D54FF0000822694146536834
:103E8000204623F001035360FFF799FA4346FF21D0
:103E9000667804F11802B342C0F084814FF0FF321B
:103EA000236901269A610B2266F30F0866F31F4807
:103EB000C3F81C805A611A611A6820466FF30A120F
:103EC0001A60FFF711FD4FF48052E36820465A61F3
:103ED0004E4B1B681B6998473046BB0618D52046D9
:103EE000FFF78DFBE3682046DE68FFF779FB0328C8
:103EF00040F05F810023A3704FF40073A380092377
:103F00004FF40052012063F38D26E368DE605A61AE
:103F1000C5F30746F70609D53C4B20461B68DB690D
:103F200098474FF480120120E3685A61B60609D51C
:103F3000364B20461B681B6A98474FF4001201203D
:103F4000E3685A61690009D5304B20461B685B6AFB
:103F500098474FF080420120E3685A616A077FF575
:103F6000E3AEE3685D686B0704D5284B20461B6809
:103F70009B6A9847E36801205D60D5E619F0010F60
:103F80003ED05FFA88F3194620460193FFF79EFC66
:103F9000C107064624D501263A68019B9660E17860
:103FA000B1420AD11069282202FB0842D2F87C13E0
:103FB000C0F31200091AC2F88C13DBF8002019466E
:103FC000126820469047E378012B09D1B8F1000F21
:103FD00006D194F81131052B02D12046FFF784FC5D
:103FE000B20741BF022632463B689A60330707D5C5
:103FF000DBF8003020469B68984708223B689A60AF
:1040000008F101084FEA59090437A5E6E00000204D
:1040100000ED00E01AF0010F76D023695FFA89FB0A
:104020001969586B04EB8B02926920FA0BF84FEA7E
:10403000C81892685FFA88F848EA010808EA020896
:1040400018F0010F1ED001214FF001085A6B01FA40
:1040500009F122EA01025A633B685946C3F8088015
:10406000574B20461B685B689847E378434509D166
:10407000B9F1000F06D194F81131042B02D120467A
:10408000FFF732FC18F0080F1EBF4FF008083B681E
:10409000C3F8088018F0100F1EBF4FF010083B68DF
:1040A000C3F8088018F0400F1EBF4FF040083B686F
:1040B000C3F8088018F0020F1EBF4FF002083B68DB
:1040C000C3F8088018F0800F1ED0D6F83421D6F837
:1040D00030319B1AD6F82421934228BF134603336C
:1040E0009B0801933B68019A9B699BB2934206D956
:1040F000D6F83421D6F83031934200D95BB94FF06D
:1041000080083B68C3F8088009F101094FEA5A0AA0
:104110000437283631E6A3EB0208D6F824315A4694
:10412000984528BF984608F103039B080193D6F8E9
:1041300028111FFA88F32046FFF764F8D6F82831D3
:104140004344C6F82831D6F834314344C6F83431F4
:10415000C8E747F6F07333423FF485AE4FF02808C6
:1041600008FB0948C6F30A163246D8F880132046E1
:10417000FFF75BF8D8F880333344C8F88033D8F8B9
:104180008C331E44C8F88C636DE64FF02808082273
:1041900004F2CC512046FFF748F808FB0948C6F363
:1041A0000A16ECE752F8040B01338160906B8160D2
:1041B00071E60123A3704023A3800523A0E600BF7E
:1041C000E000002081F0004102E000BF83F00043E6
:1041D00030B54FEA41044FEA430594EA050F08BFA2
:1041E00090EA020F1FBF54EA000C55EA020C7FEA66
:1041F000645C7FEA655C00F0E2804FEA5454D4EBE3
:104200005555B8BF6D420CDD2C4480EA020281EAAC
:10421000030382EA000083EA010180EA020281EAE4
:104220000303362D88BF30BD11F0004F4FEA013136
:104230004FF4801C4CEA113102D0404261EB410145
:1042400013F0004F4FEA03334CEA133302D05242CB
:1042500063EB430394EA050F00F0A780A4F1010487
:10426000D5F1200E0DDB02FA0EFC22FA05F28018C1
:1042700041F1000103FA0EF2801843FA05F35941A7
:104280000EE0A5F120050EF1200E012A03FA0EFC26
:1042900028BF4CF0020C43FA05F3C01851EBE37150
:1042A00001F0004507D54FF0000EDCF1000C7EEB6D
:1042B00000006EEB0101B1F5801F1BD3B1F5001FAB
:1042C0000CD349085FEA30004FEA3C0C04F10104CA
:1042D0004FEA445212F5800F80F09A80BCF1004FF3
:1042E00008BF5FEA500C50F1000041EB045141EA75
:1042F000050130BD5FEA4C0C404141EB010111F476
:10430000801FA4F10104E9D191F0000F04BF014620
:104310000020B1FA81F308BF2033A3F10B03B3F1FE
:1043200020020CDA0C3208DD02F1140CC2F10C028E
:1043300001FA0CF021FA02F10CE002F11402D8BFEC
:10434000C2F1200C01FA02F120FA0CFCDCBF41EAB8
:104350000C019040E41AA2BF01EB0451294330BD87
:104360006FEA04041F3C1CDA0C340EDC04F1140464
:10437000C4F1200220FA04F001FA02F340EA03003B
:1043800021FA04F345EA030130BDC4F10C04C4F181
:10439000200220FA02F001FA04F340EA0300294661
:1043A00030BD21FA04F0294630BD94F0000F83F4AB
:1043B000801306BF81F480110134013D4EE77FEA8E
:1043C000645C18BF7FEA655C29D094EA050F08BFDA
:1043D00090EA020F05D054EA000C04BF19461046BB
:1043E00030BD91EA030F1EBF0021002030BD5FEAFF
:1043F000545C05D14000494128BF41F0004130BD27
:1044000014F580043CBF01F5801130BD01F000457A
:1044100045F0FE4141F470014FF0000030BD7FEAED
:10442000645C1ABF194610467FEA655C1CBF0B46E8
:10443000024650EA013406BF52EA033591EA030FFF
:1044400041F4002130BD00BF90F0000F04BF0021F7
:10445000704730B54FF4806404F132044FF000052A
:104460004FF0000150E700BF90F0000F04BF0021A3
:10447000704730B54FF4806404F1320410F0004509
:1044800048BF40424FF000013EE700BF42004FEA04
:10449000E2014FEA31014FEA02701FBF12F07F4381
:1044A00093F07F4F81F06051704792F0000F14BF7E
:1044B00093F07F4F704730B54FF4607401F00045C2
:1044C00021F0004120E700BF50EA010208BF704719
:1044D00030B54FF000050AE050EA010208BF70470E
:1044E00030B511F0004502D5404261EB41014FF477
:1044F000806404F132045FEA915C3FF4DCAE4FF07B
:1045000003025FEADC0C18BF03325FEADC0C18BF61
:10451000033202EBDC02C2F1200300FA03FC20FAB2
:1045200002F001FA03FE40EA0E0021FA02F11444FF
:10453000C1E600BF70B54FF0FF0C4CF4E06C1CEA14
:1045400011541DBF1CEA135594EA0C0F95EA0C0F89
:1045500000F0DEF82C4481EA030621EA4C5123EAFC
:104560004C5350EA013518BF52EA033541F480112B
:1045700043F4801338D0A0FB02CE4FF00005E1FBDE
:1045800002E506F00042E0FB03E54FF00006E1FB28
:1045900003569CF0000F18BF4EF0010EA4F1FF046B
:1045A000B6F5007F64F5407404D25FEA4E0E6D41AB
:1045B00046EB060642EAC62141EA55514FEAC520BC
:1045C00040EA5E504FEACE2EB4F1FD0C88BFBCF538
:1045D000E06F1ED8BEF1004F08BF5FEA500E50F1E9
:1045E000000041EB045170BD06F0004646EA0101AF
:1045F00040EA020081EA0301B4EB5C04C2BFD4EBE1
:104600000C0541EA045170BD41F480114FF0000ED9
:10461000013C00F3AB8014F1360FDEBF002001F047
:10462000004170BDC4F10004203C35DA0C341BDCC1
:1046300004F11404C4F1200500FA05F320FA04F093
:1046400001FA05F240EA020001F0004221F00041C7
:1046500010EBD37021FA04F642EB06015EEA430E3A
:1046600008BF20EAD37070BDC4F10C04C4F120056A
:1046700000FA04F320FA05F001FA04F240EA02001D
:1046800001F0004110EBD37041F100015EEA430EEE
:1046900008BF20EAD37070BDC4F1200500FA05F20E
:1046A0004EEA020E20FA04F301FA05F243EA02038D
:1046B00021FA04F001F0004121FA04F220EA02009C
:1046C00000EBD3705EEA430E08BF20EAD37070BDE2
:1046D00094F0000F0FD101F00046400041EB0101C2
:1046E00011F4801F08BF013CF7D041EA060195F0A4
:1046F000000F18BF704703F00046520043EB03035E
:1047000013F4801F08BF013DF7D043EA060370474A
:1047100094EA0C0F0CEA135518BF95EA0C0F0CD055
:1047200050EA410618BF52EA4306D1D181EA03019B
:1047300001F000414FF0000070BD50EA410606BF95
:104740001046194652EA430619D094EA0C0F02D1DA
:1047500050EA013613D195EA0C0F05D152EA03361F
:104760001CBF104619460AD181EA030101F000413D
:1047700041F0FE4141F470014FF0000070BD41F086
:10478000FE4141F4780170BD70B54FF0FF0C4CF460
:10479000E06C1CEA11541DBF1CEA135594EA0C0F7F
:1047A00095EA0C0F00F0A7F8A4EB050481EA030ECC
:1047B00052EA03354FEA013100F088804FEA0333B3
:1047C0004FF0805545EA131343EA12634FEA022281
:1047D00045EA111545EA10654FEA00260EF0004142
:1047E0009D4208BF964244F1FD0404F5407402D294
:1047F0005B084FEA3202B61A65EB03055B084FEA25
:1048000032024FF480104FF4002CB6EB020E75EB21
:10481000030E22BFB61A754640EA0C005B084FEA49
:104820003202B6EB020E75EB030E22BFB61A7546C6
:1048300040EA5C005B084FEA3202B6EB020E75EB11
:10484000030E22BFB61A754640EA9C005B084FEA89
:104850003202B6EB020E75EB030E22BFB61A754696
:1048600040EADC0055EA060E18D04FEA051545EA85
:1048700016754FEA06164FEAC30343EA52734FEA2E
:10488000C2025FEA1C1CC0D111F4801F0BD141EAA7
:1048900000014FF000004FF0004CB6E711F4801F0C
:1048A00004BF01430020B4F1FD0C88BFBCF5E06FEC
:1048B0003FF6AFAEB5EB030C04BFB6EB020C5FEAFC
:1048C000500C50F1000041EB045170BD0EF0004E51
:1048D0004EEA113114EB5C04C2BFD4EB0C0541EA83
:1048E000045170BD41F480114FF0000E013C90E680
:1048F00045EA060E8DE60CEA135594EA0C0F08BF44
:1049000095EA0C0F3FF43BAF94EA0C0F0AD150EA42
:1049100001347FF434AF95EA0C0F7FF425AF1046D5
:1049200019462CE795EA0C0F06D152EA03353FF4FD
:10493000FDAE1046194622E750EA410618BF52EA7A
:1049400043067FF4C5AE50EA41047FF40DAF52EA4E
:1049500043057FF4EBAE12E74FF0FF3C06E000BFEB
:104960004FF0010C02E000BF4FF0010C4DF804CDF8
:104970004FEA410C7FEA6C5C4FEA430C18BF7FEAB8
:104980006C5C1BD001B050EA410C0CBF52EA430CE6
:1049900091EA030F02BF90EA020F0020704710F166
:1049A000000F91EA030F58BF994208BF90422CBFF5
:1049B000D8176FEAE37040F0010070474FEA410CEE
:1049C0007FEA6C5C02D150EA013C07D14FEA430C0C
:1049D0007FEA6C5CD6D152EA033CD3D05DF8040B7D
:1049E000704700BF8446104662468C4619466346AF
:1049F00000E000BF01B5FFF7B7FF002848BF10F186
:104A0000000F01BD4DF808EDFFF7F4FF0CBF0120CA
:104A100000205DF808FB00BF4DF808EDFFF7EAFF46
:104A200034BF012000205DF808FB00BF4DF808ED01
:104A3000FFF7E0FF94BF012000205DF808FB00BFF6
:104A40004DF808EDFFF7CEFF94BF012000205DF880
:104A500008FB00BF4DF808EDFFF7C4FF34BF01208D
:104A600000205DF808FB00BF4FEA410212F500127A
:104A700015D211D56FF47873B3EB625212D94FEAA5
:104A8000C12343F0004343EA505311F0004F23FA8F
:104A900002F018BF404270474FF00000704750EAE4
:104AA000013005D111F0004008BF6FF000407047A1
:104AB0004FF00000704700BF80F0004002E000BFF0
:104AC00081F0004142001FBF5FEA410392EA030FF9
:104AD0007FEA226C7FEA236C6AD04FEA1262D2EB43
:104AE0001363C1BFD218414048404140B8BF5B4248
:104AF000192B88BF704710F0004F40F4000020F0E1
:104B00007F4018BF404211F0004F41F4000121F0F6
:104B10007F4118BF494292EA030F3FD0A2F1010240
:104B200041FA03FC10EB0C00C3F1200301FA03F17E
:104B300000F0004302D5494260EB4000B0F5000FA1
:104B400013D3B0F1807F06D340084FEA310102F160
:104B50000102FE2A51D2B1F1004F40EBC25008BF12
:104B600020F0010040EA03007047490040EB0000DC
:104B700010F4000FA2F10102EDD1B0FA80FCACF10B
:104B8000080CB2EB0C0200FA0CF0AABF00EBC2500A
:104B900052421843BCBFD0401843704792F0000FF8
:104BA00081F4000106BF80F400000132013BB5E74B
:104BB0004FEA41037FEA226C18BF7FEA236C21D0C1
:104BC00092EA030F04D092F0000F08BF0846704726
:104BD00090EA010F1CBF0020704712F07F4F04D1F4
:104BE000400028BF40F00040704712F100723CBF07
:104BF00000F50000704700F0004343F0FE4040F431
:104C0000000070477FEA226216BF08467FEA2363EE
:104C10000146420206BF5FEA412390EA010F40F4D9
:104C2000800070474FF0000304E000BF10F0004325
:104C300048BF40425FEA000C08BF704743F096430C
:104C400001464FF000001CE050EA010208BF704727
:104C50004FF000030AE000BF50EA010208BF7047AE
:104C600011F0004302D5404261EB41015FEA010CC3
:104C700002BF84460146002043F0B64308BFA3F1BB
:104C80008053A3F50003BCFA8CF2083AA3EBC2539D
:104C900010DB01FA02FC634400FA02FCC2F12002BC
:104CA000BCF1004F20FA02F243EB020008BF20F0F3
:104CB0000100704702F1200201FA02FCC2F1200259
:104CC00050EA4C0021FA02F243EB020008BF20EA4E
:104CD000DC7070474FF0FF0C1CEAD0521EBF1CEA7C
:104CE000D15392EA0C0F93EA0C0F6FD01A4480EA6A
:104CF000010C400218BF5FEA41211ED04FF0006353
:104D000043EA501043EA5111A0FB01310CF000407E
:104D1000B1F5000F3EBF490041EAD3715B0040EAA4
:104D2000010062F17F02FD2A1DD8B3F1004F40EB74
:104D3000C25008BF20F00100704790F0000F0CF047
:104D4000004C08BF49024CEA502040EA51207F3A0B
:104D5000C2BFD2F1FF0340EAC250704740F40000E6
:104D60004FF00003013A5DDC12F1190FDCBF00F0D7
:104D700000407047C2F10002410021FA02F1C2F185
:104D8000200200FA02FC5FEA310040F1000053EA21
:104D90004C0308BF20EADC70704792F0000F00F06F
:104DA000004C02BF400010F4000F013AF9D040EA75
:104DB0000C0093F0000F01F0004C02BF490011F409
:104DC000000F013BF9D041EA0C018FE70CEAD15307
:104DD00092EA0C0F18BF93EA0C0F0AD030F0004C87
:104DE00018BF31F0004CD8D180EA010000F000403B
:104DF000704790F0000F17BF90F0004F084691F0F9
:104E0000000F91F0004F14D092EA0C0F01D1420232
:104E10000FD193EA0C0F03D14B0218BF084608D1FB
:104E200080EA010000F0004040F0FE4040F4000045
:104E3000704740F0FE4040F4400070474FF0FF0CD8
:104E40001CEAD0521EBF1CEAD15392EA0C0F93EA1F
:104E50000C0F69D0A2EB030280EA010C49024FEA71
:104E6000402037D04FF0805343EA111143EA10132A
:104E70000CF000408B4238BF5B0042F17D024FF4E2
:104E8000000C8B4224BF5B1A40EA0C00B3EB510FBD
:104E900024BFA3EB510340EA5C00B3EB910F24BFA6
:104EA000A3EB910340EA9C00B3EBD10F24BFA3EB2B
:104EB000D10340EADC001B0118BF5FEA1C1CE0D1F3
:104EC000FD2A3FF650AF8B4240EBC25008BF20F0A6
:104ED000010070470CF0004C4CEA50207F32C2BFFA
:104EE000D2F1FF0340EAC250704740F400004FF097
:104EF0000003013A37E792F0000F00F0004C02BFC8
:104F0000400010F4000F013AF9D040EA0C0093F091
:104F1000000F01F0004C02BF490011F4000F013BEB
:104F2000F9D041EA0C0195E70CEAD15392EA0C0F53
:104F300008D142027FF47DAF93EA0C0F7FF470AF8B
:104F4000084676E793EA0C0F04D14B023FF44CAFCE
:104F500008466EE730F0004C18BF31F0004CCAD163
:104F600030F000427FF45CAF31F000437FF43CAF9F
:104F70005FE700BF4FEA4002B2F1FE4F0FD34FF0A0
:104F80009E03B3EB12620DD94FEA002343F00043B6
:104F900010F0004F23FA02F018BF404270474FF064
:104FA0000000704712F1610F01D1420205D110F0EB
:104FB000004008BF6FF0004070474FF0000070479E
:104FC000002103E00A4B5B584350043109480A4B67
:104FD00042189A42F6D3094A02E0002342F8043B01
:104FE000074B9A42F9D3FAF7DBFF00F00DF8704750
:104FF0001056010800000020B4050020B405002070
:1050000008700020FEE7000008B54FF44070FDF77F
:10501000B1FB62B601214FF48040FCF7FDF9F3F7D4
:1050200057F9F4F727FBF3F731F9F4F7D9FCF4F764
:1050300057FFF3F765FAF3F78BFAF3F7E1FB1B4C35
:1050400028B1F3F7DDFB6070F3F7DAFBA06020789E
:10505000F3F748FDE078F3F787FE2078F3F7A9FE31
:10506000E078F4F705F82269A1686079F4F736F979
:10507000F5F72EF9FAF715FEF3F7C1FCF8F74EFE37
:10508000F9F798FC80220A4B1A83F8F7C7FFF9F763
:1050900092FCF9F7DFFFF3F75FFBF3F77DFB0028E6
:1050A000F3D0FAF7FEFDF8F739FEEEE70400002032
:1050B000000402402DE9F843C1F30A57A7F2FF3577
:1050C000132D0B460446864611DC002D42DB264F8D
:1050D00047FA05F501EA050757EA000E1DD101F070
:1050E0000045C2E9000170462946BDE8F883332D2A
:1050F0001FDC4FF0FF35A7F2134725FA07F710EA38
:10510000070C1FD00D4620EA0704C2E900450B46F4
:105110002246FFF75BF8BDE8F8834FF0000821EA6C
:105120000509C2E900894B464246FFF74FF8BDE842
:10513000F883002401F00045C2E900012046294619
:10514000BDE8F88301F00045C2E900016046294648
:10515000BDE8F883002001F0004106460F462046D6
:105160001946C2E90067C0E7FFFF0F00024B13B109
:10517000024800F005B87047000000008D5101089A
:10518000002301461A46184600F01EB838B50A4CEE
:105190000A4D641BA4100AD004F18043013B05EBC7
:1051A0008305013C55F804399847002CF9D1BDE836
:1051B000384000F021BA00BF105601080C56010813
:1051C000704700BF704700BF2DE9F8432C4D0646DD
:1051D000286898460F469146FFF7F2FF294B1C6856
:1051E000D4F84831002B3ED05A681F2A1CDC02F14B
:1051F000010E76B1012103EB8204C4F88890D3F844
:10520000880191400843022EC3F88801C4F8088140
:1052100023D00232C3F804E0286843F82270FFF775
:10522000D1FF0020BDE8F883174B0BB34FF4C870D3
:10523000AFF300800346D8B10020D4F848114FF0F6
:10524000010E586019600246C4F84831C3F888015D
:10525000C3F88C01002EDCD0CCE7D3F88C010143DD
:10526000C3F88C11D5E704F5A673C4F84831BBE741
:105270002868FFF7A7FF4FF0FF30BDE8F88300BFB5
:10528000B0050020E8550108000000000000000003
:10529000C1F30A522DE9F047A2F2FF36132E0B4656
:1052A00004460D4607468846824622DC002E4FDB28
:1052B0003D4A42FA06F901EA090202431ED038A328
:1052C000D3E90023FEF784FF00220023FFF7C2FB8F
:1052D00050B1002D04DD4FF4801343FA06F6B044BC
:1052E0004FF0000A28EA0905544629462046BDE841
:1052F000F087332E06DDB6F5806F3DD01946204687
:10530000BDE8F0874FF0FF39A2F2134229FA02F903
:1053100010EA090FF2D022A3D3E90023FEF758FFC9
:1053200000220023FFF796FB0028DDD0002D09DDC9
:10533000142E2FD00123C6F1340603FA06F63719CE
:1053400028BF9844454627EA090A54462946CDE72E
:1053500013A3D3E90023FEF73BFF00220023FFF74E
:1053600079FB0028C0D0002D0FDB55EA040709D0D7
:105370004FF0000A0D4DB7E702460B46FEF728FF37
:105380000446BCE7BA463D46AEE74FF0000A4FF090
:105390000045A9E705F10108D4E700BFAFF300809D
:1053A0009C7500883CE4377EFFFF0F000000F03F53
:1053B000C1F30A522DE9F843A2F2FF36132E0B4631
:1053C00004460D46884607461DDC002E40DB3C4A5D
:1053D000864642FA06F901EA0902024318D036A3CA
:1053E000D3E90023FEF7F4FE00220023FFF732FB8F
:1053F00020B1002D42DB002728EA09053C4629465A
:105400002046BDE8F883332E06DDB6F5806F2FD039
:1054100019462046BDE8F8834FF0FF39A2F2134247
:1054200029FA02F910EA090FF2D023A3D3E90023E5
:10543000FEF7CEFE00220023FFF70CFB0028DDD094
:10544000002D21DB454627EA09073C462946D7E7D8
:1054500019A3D3E90023FEF7BBFE00220023FFF7C8
:10546000F9FA0028CAD0002D19DB00273D46C5E710
:1054700002460B46FEF7ACFE0446CAE74FF4801323
:1054800043FA06F6B044B6E7142E10D00123C6F155
:10549000340603FA06F6371928BF9844D2E725F0F8
:1054A0000042084B224318BF1D460027A6E705F11E
:1054B0000108C7E7AFF300809C7500883CE4377EA5
:1054C000FFFF0F000000F0BF50C300008813000072
:1054D000018008080000000000000000C800000073
:1054E0000100C80000800000000000000000000073
:1054F00000000000000000000000000000000000AC
:105500000000000000000000010002000300040091
:10551000050006000101010001000000010000007B
:105520000100000000000100000000000000000079
:105530000000000001010100000000000000000068
:105540000001000000000000010101000101000154
:10555000010000000000000000000000000000004A
:10556000000000000000000000000000000000003B
:105570000000000000000000000000000000010129
:105580000100000100010101000000000000000016
:105590000000000036323134563131350053746525
:1055A0007070657220446576696365005472696E37
:1055B000616D6963204D6F74696F6E20436F6E7407
:1055C000726F6C00544D4353544550005643502065
:1055D000436F6E6669670056435020496E7465726A
:1055E000666163650000000088010020F8B500BF17
:1055F000F8BC08BC9E467047F8B500BFF8BC08BCB4
:045600009E4670470B
:085604006D510108AD810008A1
:04560C008981000888
:10561000945501080001020000080000010000008C
:105620000200000000000000000000000000000078
:10563000000000000000000000000000000000006A
:10564000000000000000000000000000000000005A
:105650000000000012010002020000403C2A00018C
:1056600000020102030104030904000000C201005A
:105670000000080025A0000831A000088DA0000847
:1056800071A00008A9A00008C5A00008E1A00008BA
:1056900045A1000821A0000847A1000849A1000871
:1056A0004BA100084DA1000823A000080A06000233
:1056B000000000400100000041A100083DA00008DA
:1056C000FDA0000841A0000845A00008000E270723
:1056D00000000000000000000102030406070809A2
:1056E0000000000001020304010203040607080988
:1056F000E4000020F529010841290108F7280108E4
:1057000067280108C92801084B2801083528010825
:10571000772801088528010893280108A92801088D
:10572000FF00000009024300020100C0320904002A
:1057300000010202010005240010010524010001FE
:10574000042402020524060001070582030800FF65
:1057500009040100020A00000007050102400000E0
:105760000705810240000000992C0108712C0108F6
:10577000B12B010800000000CD2A0108ED2C010822
:10578000812B0108092B0108000000000000000027
:10579000FD2A010800000000000000007404002041
:1057A000DC04002044050020000000000000000090
:1057B00000000000000000000000000000000000E9
:1057C00000000000000000000000000000000000D9
:1057D00000000000000000000000000000000000C9
:1057E00000000000000000000000000000000000B9
:1057F00000000000000000000000000000000000A9
:105800000000000000000000000000000000000098
:105810000000000000000000000000000000000088
:105820000000000000000000000000000000000078
:105830000000000000000000000000000000000068
:1058400001000000000000000E33CDAB34126DE605
:10585000ECDE05000B00000000000000000000006E
:105860000000000000000000000000000000000038
:105870000000000000000000000000000000000028
:105880000000000000000000000000000000000018
:105890000000000000000000000000000000000008
:045BC000E46F00206E
:0400000508014FC1DE
:00000001FF
